:020000040000FA
:080000000002040000000000F2
:020000040000FA
:100400002F8B21000E7F22000E01880000000000CB
:100410000C000700C0B12C000100200011000700F3
:10042000000020000000E000020032000000020096
:100430000000000036D10200000000000040DA0099
:100440000000FE004440A900C06221000000E0005E
:100450000300320000002000A00188004440A800F2
:100460000000060091018800800078000000EB0089
:1004700015003700E280400032A0B4009101BA00BC
:10048000E280400032A0B4009102BA00E280400055
:1004900032A0B4000002EB00472BDE00F507B200EB
:1004A000602CE10004003A000059EB008301E900F0
:1004B000FDFF3E00040037006128E100010032002A
:1004C0000082EB00040007001101BA000200E00006
:1004D000E8FF3A00000006003159BA008301E90044
:1004E0000C0032002159BA008301E90008003200F3
:1004F0000400E00003003A00E280400032A0B400B3
:10050000F5FF370011D9BA008301E900FAFF3A007C
:100510008100E800E180400032A0B4000000060045
:100520000040DA000000FE006900E1000400350030
:100530006D00E100030034000002B1000100320050
:1005400000000500100005001004B1000700350090
:100550009001B100040034007000B10003003500C8
:100560009001B10001003C001000050000000500F2
:10057000800078001106B100030035009101B10040
:1005800001003C000050A100000006001004B10072
:10059000030035009001B10001003C00100005008F
:1005A00000000500800078001104B1000300350050
:1005B0009101B10001003C000050A00000000600C5
:1005C0000A00FA0080017800E20F500028003E0087
:1005D00080C58000E10F5000080032008023200019
:1005E0000000E00005003200042320002523200045
:1005F00046232000800178000400370004222000F8
:100600002522200046222000832220001440900052
:100610000004E000040035008009EB001440900065
:100620000074A00010429800154090000028A3001C
:1006300003003A00154090000024A000904298006A
:100640008001EB0007003700154090000008A30070
:10065000FDFF320063C078000000FB00000B780053
:100660008301E800828F5100F7FF3A00080037004D
:1006700030002000B0BF9F00C3BF9F00D1BF9F00CC
:10068000E2BF9F006A80570000C0DA006FB9970090
:10069000020078000080FA00000006000A00FA005C
:1006A000881F7800800178000000E00029003A00EF
:1006B00080C58000E10F5000080032008023200038
:1006C0000000E00005003200042320002523200064
:1006D00067232000800178000400370004222000F6
:1006E0002522200067222000832220001440900051
:1006F0000004E000040035008009EB001440900085
:100700000074A000104298000002EB000C003700BB
:10071000130A2000154478006140640002003A008A
:100720008301E900FBFF3A000402E80095417800EC
:1007300061C0610005003200170078008058780021
:1007400004035100820F5200F1FF3A0006005100ED
:100750000800370020002000A0BF9F00B3BF9F000B
:10076000C1BF9F00D2BF9F006C80570000C0DA005D
:100770005FB897004F0478000080FA000000060080
:10078000020AB900001BB9000200B8008100420053
:100790008100430000000600889FBE008A9FBE00C3
:1007A000010578000100E0000400350008003C006D
:1007B0000000E0002000320005003700600010005B
:1007C000E080180002003B0001F02C001A00370006
:1007D0000004BE006011B8006B0920000982CF0040
:1007E000020039000882CF000441B0006942520083
:1007F0000E00320008003B0082817100610164003C
:100800008904D1000884D3008B05E8000442E80085
:10081000F9FF3A00050037000804440089844C00C1
:100820008B05E9000442E900FBFF3A007202070071
:100830000AF0A70001F0A0004F05BE004F04BE0063
:1008400000000600889FBE008A9FBE008C1F7800B3
:100850008F0207009602330003866C006450E100AB
:100860002E0032006420E100330032006150E100CC
:100870002F0032006120E1003100320085855500F3
:10088000EB07B00009002000080420000500370035
:100890000804440089844C000A0031000603430028
:1008A00087834B000001530081815B00F8FF330018
:1008B0000203BE000800A0000804440089844C0024
:1008C000F6FF3900C639DD008301730001003200F4
:1008D000130020008904D1000884D3000998A300E4
:1008E000050032000800A7000300A0008904D10021
:1008F0000884D3008B05E8008904D1000884D30064
:100900000001EB000281D2003B02070001F0A100D0
:100910000CF0A70001F0A0006E0237006420E10097
:10092000700232000801BE000200BE00F7FF37006F
:100930006120E1006B0232006000B800F3FF370075
:100940000000200001F82700F0FF370003F0A200AC
:10095000889FBE008A9FBE008C1F78004C02070053
:10096000530233006450E1004F0032006420E10084
:100970005200320003826C0007003B000905D000E2
:100980000306D000820F54000C065D0002003900FF
:100990000200320089017800030678008582550044
:1009A00004003D000003FD008103FD008502EA0014
:1009B0008B854200840F720002003B006000100033
:1009C000E08018006011B8000005EB007A28E10013
:1009D0000A00390006007800C75DDD00F707B200A5
:1009E000878075002D003700828171000A01780030
:1009F000610560008180D1000080D3008502E9009C
:100A0000F9FF3B00060440008784480002003B00D9
:100A100060041400E0841C000988A3000700320071
:100A20008A81710082817100610164008904D100B2
:100A30000884D3008B05E800170037000978A3006D
:100A400013003A000B00E000130034008B05E900AE
:100A50000804440089844C000A4474000978A30007
:100A60000D003A000B00E000070034008B05E900A0
:100A70000804440089844C0001003A000B00200067
:100A80000978A300F7FF32000001EB0002003700F5
:100A9000828171000A017800D70107000CF0A700DD
:100AA00001F0A0000B0237006420E10002003A00D0
:100AB000838F6C000B0233000801BE000200BE00F1
:100AC00004023700020007000400BE000000060018
:100AD0006022B800060220000000D0008180D20011
:100AE0000482D2008582D2000000A00002025200DF
:100AF00083825A00030031000202420083824A00CE
:100B00000000A1000603E900F3FF3A000000060020
:100B1000839F68000100E00002003D0060001000BB
:100B2000E08018000300E00002003D0060011100B9
:100B3000E0811900E6FF07004F00E00002003B00E3
:100B400060001000E0801800000006000400200093
:100B5000E7013700889FBE008A9FBE008C1F780087
:100B6000CB010700D201330003866C006450E10022
:100B7000240032006420E100270032006150E100CF
:100B8000220032006120E100210032008B8542000A
:100B9000EB07B1000134B800003AB8000804420085
:100BA00089844A00013AB8000030B80088804000CB
:100BB00009014A0004003300000040008180480021
:100BC000020149008B05E900C909DD0083017000BD
:100BD0000100320013002000C814DE004814DD00BC
:100BE0004709DE001200B200C808DE000884700069
:100BF0008101070001F0A1000CF0A70001F0A000A6
:100C0000B40137006120E100B60132000801BE00E6
:100C10000200BE00F7FF37006150E100FCFF3A0020
:100C2000B00137000001BE00CC0107000470A7002E
:100C300003F0A10003F8A30013003A006509B10016
:100C400010003200090035006928E100020035007B
:100C500001002800000005000000400081804800DD
:100C60008502E900FCFF3A0000000600F88F420010
:100C7000050035008100D1000080D3008502E80026
:100C8000FCFF3A00000006008000EB0000000500B9
:100C90000001BE00B10107000470A70003F0A1002D
:100CA0006509B100160032000D0035006828E1002A
:100CB00006003500F0FF2F00F1FF27000300E000E1
:100CC00013003B0001002800000005000000400068
:100CD000818048008502E900FCFF3A0008003700E7
:100CE000F88F420002003C008000EB00000005008D
:100CF0008100D1000080D3008502E800FCFF3A00AB
:100D00000300E00002003B0060001000E0801800DB
:100D100000000600889FBE008A9FBE008C1F7800DE
:100D20000205BE000004BE000006EB00E00F50000C
:100D3000E08F5800E00F5900E08F590007003D0098
:100D40006000B8006011B8000804500089845800A1
:100D50000A0559008B8559001C002000E00F520045
:100D6000E08F5A00E00F5B00E08F5B0002003D0067
:100D70000F0007000C00A2000800BE000A01BE0020
:100D80008B0107000203BE000002BE000C00E00061
:100D900001003200060007000400BE000601BE008C
:100DA0004F0678004F05BE004F04BE00000006004D
:100DB0006000B8006011B80004025000858258003D
:100DC000060359008783590000000600881F780039
:100DD000000478005001BE004000BE000400400046
:100DE000858048000601490087814900009CBE00BB
:100DF0000294BE000400E1000588E1000690E100D5
:100E00000798E10002003100680044001008E80083
:100E10004F04780000000600F4874700889FBE005A
:100E20008A9FBE008C9FBE008E1F78000205BE0008
:100E30000004BE00D4B79F00E5B79F00F6B79F003F
:100E400087BF9F000000EB00C0B79F00B0B79F00B6
:100E5000A0B79F0090B79F0080B79F000D042000AF
:100E6000BFB097004FB09700000140000000E000C5
:100E70000F003D004F08DE0000007100C0B79F006A
:100E80009E00070001003D0012002000A1000700A5
:100E900001003D0012002000A6000700B10007007D
:100EA000B60007000F004000C8FF0700220037000F
:100EB0004F08DE0000067100CCB79F008F000700CE
:100EC00001003D00120020009200070001003D00DB
:100ED0001200200097000700A20007000FB2970041
:100EE0009FB297002FB39700BFB39700A9000700E8
:100EF0000000520081805A0002015B0083815B0088
:100F000080B79F0091B79F00A2B79F00B3B79F0023
:100F10000007EB009F0007000020E10001A8E100AE
:100F200002B0E10003B8E100010031001E00200022
:100F30000E005600C0B79F004FB297000400E000BB
:100F40000700350010002000010020006011B800EB
:100F500008047000898470000A0571008B85710097
:100F60008D06E900BEFF3A000400E00003003D00EA
:100F7000820007000F00400094FF07004FA8970071
:100F80000000E00004003A000FB497009FB49700FF
:100F90002FB59700BFB59700940007004F07780062
:100FA0004F06BE004F05BE004F04BE004F01B1000A
:100FB00000000600881F780018002000881F7800B5
:100FC00095FF07008F87E9004F04780000000600B6
:100FD000801FEB0090FF07008F87E90000000600EC
:100FE000889FBE008A9FBE008C1F78006E0007009D
:100FF00007003D0073000700E00F5B00E08F5B001F
:1010000007003D00320007000006EB000400370037
:101010003400070002003D002A0007001C002000E9
:1010200072000700E3FF07000203BE000002BE00DB
:101030000C00E00001003200220007000400BE00A6
:101040000601BE004F0678004F05BE004F04BE00EB
:1010500000000600889FBE008A9FBE008C1F78009B
:101060005100070005003D0056000700E00F5B003F
:10107000E08F5B0006003D00040037001900070008
:1010800003003D006000B8006011B80010000700C8
:1010900056000700CEFF07000203BE000002BE009C
:1010A0000C00E00001003200060007000400BE0052
:1010B0000601BE004F0678004F05BE004F04BE007B
:1010C000000006006000B8006011B80000003700A2
:1010D0000402500085825800060359008783590096
:1010E000000006000006EB00E00F5200E08F5A00FF
:1010F000E00F5B00E08F5B00000006000180400015
:1011000090B79F000001EB008FB097000100E00056
:10111000000006000200700090B79F0001804000B0
:1011200080B79F000001EB00FFA897000100E000DE
:10113000000006000200700080B79F0001804000A0
:101140006FAA9700CF20DE0001007000F0AF9F0073
:1011500004024200250007004F18DE000002720062
:1011600000000600E4AF9F000804440089844C009E
:101170000A054D008B854D00000006003FB2970028
:10118000CFB297005FB39700EFB3970000FE2F0038
:10119000000006003FB09700CFB097005FB1970006
:1011A000EFB19700000006000205BE000004BE007B
:1011B000E00F5000E08F5800E00F5900E08F590019
:1011C000000006006000B8006011B800080450007C
:1011D000898458000A0559008B8559001C0020009D
:1011E000E00F5200E08F5A00000006000800BE0029
:1011F0000A01BE0000000600810020006180550049
:101200000B003D000B00200061FE2F000100E100FB
:101210001D00340082817100610164008904D100E5
:101220000884D3000000E800FAFF3A0071002000B3
:1012300061006400030070000200600009003200D9
:1012400061044400E0844C000988A50005003200D8
:101250008B05E8006808E10002003A008904D1002B
:101260000884D300F20F20000258E10005003D0081
:10127000C75DDD00F907B2008980750008007800BD
:10128000000006000BF827008B0078000000050026
:101290000004BE00310007000003BE000405BE00CC
:1012A0000200BE002D000700844F750000000600FC
:1012B0000200BE006450E100050036006420E10039
:1012C000020036000968A30001003A000800BE00D1
:1012D0000160A0004F0678004F05BE004F04BE001D
:1012E00000000600F0FF2F00F1FF2700F9FF370094
:1012F000889FBE008A9FBE00841F7800E4FF07001D
:101300004F00780011003300F0FF2F00838F6C0036
:1013100006003B00040565000A00A700080037002E
:1013200009F0A6001000200008003700820F5400CA
:10133000838F5C00030039001000200001003E0094
:101340000000200009F0A7000000EA004F05BE00E1
:101350004F04BE000000E00000000600C70ADE00E7
:10136000F107B200F50FB20008003200E1CF4200F1
:10137000020032000170A00024000500810F7000FF
:10138000010032000408050044000500810F7000D0
:1013900002003A00140005008502E9000000400048
:1013A00081C04800FCFF3B000170A0002400050044
:1013B000889FBE008A9FBE008C9FBE000404B800B8
:1013C0000506B8008904460060854E000606B80090
:1013D0000A054600E0854E000706B8008B0546006A
:1013E000040EB800890446000A854E00E0854D00D1
:1013F000050EB8000A0546008B854E00060EB800A3
:101400008B0546000416B8000A0546008B854E0081
:101410000516B8008B054600041EB8008B05460073
:101420000800BE000A01BE004F06BE004F05BE0008
:101430004F04BE0000000600800178000001780023
:1014400031407800005978000004E000FCFF3A00C9
:1014500003007800000006008001EB000200370066
:10146000817178008301E800828F5100FCFF3A000F
:10147000000006000400FA00E0BF9F00E48157006E
:10148000812978000002EB000F0037006FB8970049
:10149000904078007FB89700104078000402E80080
:1014A00080CF5000040032008180FB000080FB00F0
:1014B00000805000070037006FB897000000E80078
:1014C000E0BF9F009309E800820F5200EFFF3A004F
:1014D0000000EB000080FA000000060010417800D8
:1014E000B141510003003A000000E8000204E000AE
:1014F000FAFF3A000300FB0000000600889FBE00D0
:101500008A9FBE008C9FBE00800478000205BE004A
:10151000010478000200BE006146B9000C01BE0063
:101520006BFD07000901E800E00F5000E08F580054
:101530000200320082047800F7FF37000049EB0018
:101540000C01BE000A00BE005EFD070000447800EA
:101550000C01BE000A00BE005DFD07000005BE00D4
:10156000E94F5400010034006744440002C3B30053
:1015700082544400E00F5000E08F5800F0FF3A0022
:10158000090078004F06BE004F05BE004F04BE00A4
:1015900000000600881F780000047800E00F51006A
:1015A000E08F590002003500000278000500370086
:1015B00000027800D0C2B300005A78006001110028
:1015C000E081190004007800CCFF070008007800D3
:1015D0004F047800000006000003780080027800C5
:1015E000020278008001EB00080037000402E900E5
:1015F00063C07800805A78008301E8000004E000AE
:1016000002003A008000EB0006003700828F510094
:10161000F6FF3A00FBFF37000040EB0080F07A0055
:101620008100E800848F5000FBFF3A00060078003C
:1016300000000600800178000001780001003700FA
:101640000201E8001204E000FDFF3A00314078009A
:10165000005978000004E000FCFF3A000300780025
:1016600000000600810178000002EB000B0037004B
:10167000E44078000104E000030032000402E800C6
:1016800093CF5000040032008180FB001380FB00E8
:1016900000805000000006008301E800820F520025
:1016A000F3FF3A0000000500800078003004E000FD
:1016B000FEFF3A00010050000000E90000000600B3
:1016C0008001EB000200370061F079008301E8003F
:1016D000828F5100FCFF3A00000006000C00FA0067
:1016E000A0BF9F00C0BF9F00EFFF0700B0BF9F00DB
:1016F000F0BF9F00100C2000D0BF9F0074815700E6
:10170000EFB097006C805700580107000080FA0086
:1017100000000600E4874700889FBE008A9FBE0045
:101720008C9FBE008E1F78000005780001077800AE
:10173000820578000000EB0070C588000100E00021
:10174000010032008A0878000A047800B844780062
:101750000900FB0074FB07000000E00002003200FB
:1017600008057800F8FF3700D0C2B30080CF5400DE
:1017700005003A00984478000A84E80010C0B300DD
:1017800090F79F00070037000041EB0092F79F00A1
:10179000B0C2B30080CF540002003A0098447800F1
:1017A0000A84E80000C3B30080CF540017003A0059
:1017B00008057800BA4478000B00E000020032000F
:1017C000F08F550009003A0080C7B30080CF540065
:1017D0000300320080C5B30080CF540007003A00F8
:1017E0009A4478000885E8000B0120006066B80084
:1017F0000040EB0080F79F00100037000B00E00076
:10180000FAFF3A008B002000F8FF37000B00E000E1
:1018100003003A0008057800AB002000F3FF370012
:1018200008057800F1FF37002002200070C588000D
:101830000205780012C0B300240037000904FB0041
:101840000800780040FB07000000E00005003200BF
:101850000800780046FB070091CCB300014440002B
:101860000500370001FD2F0001004400E90F500082
:1018700015003E0001C444000800FB008B0F50001F
:1018800011003D006159B9000C00BE00BCFB07000F
:101890000801FB00CF91DE0000004100818049007B
:1018A0000A01E800800F5600818F5E00DEFF3E00D7
:1018B0009A4478000205780012C0B30082F79F00B6
:1018C0000006BE00DDFF37000041EB000E00E00027
:1018D000030032000FF097000004E00004003A001B
:1018E0009E00780000C3B300914F100001003A0041
:1018F0000A0FE900E14F510003003A000086EB00B7
:101900008086EB00050037001FF197000204E0001D
:101910000200320060061600E0861E000C00BE00C9
:101920004F0778004F06BE004F05BE004F04BE00B3
:101930004F00B10000000600889FBE008A9FBE00D5
:101940008C1F780080057800010578000206780079
:101950000000EB0070C588000B0478000100370020
:101960000804E800984478000900FB00EEFA07003C
:101970000000E000FAFF3A00D0C2B30080CF54006C
:101980000500320000C0E90080CF540002003200A0
:1019900080447800010037000804E8000C0178005A
:1019A0008A007800080078005AFF07000001BE0096
:1019B0009A0F540001003A000B0D78009A8F5500E1
:1019C00003003A00E00F5100E08F59000F003A0089
:1019D000B0C2B30080CF540004003A00E00F5100C1
:1019E000E08F590015003D0008003700D0C2B30059
:1019F00080CF540011003A000000200001002800B0
:101A0000800F5100818F59000A003600200220000B
:101A100070C5880002002000030028006B404000D1
:101A200080CF540005003200F2FF2F00F3FF2700A3
:101A30000200370060011100E08119000200BE00C1
:101A40004F0678004F05BE004F04BE0000000600A0
:101A50008002780080017800010037008301E800EF
:101A60001304E000FDFF3A000002EB00820F520079
:101A70000600320064C07800805978000402E80053
:101A80000004E00002003200F8FF37008049EB005C
:101A900005007800000006000C00FA00889FBE00D8
:101AA00000047800CFB09700F0FF2700D0BF9F0060
:101AB0008004EB0099BF9F0088BF9F00A8BF9F00D4
:101AC000200C2000B0BF9F00788157007080570025
:101AD000870107000FB89700094878000FB89700F2
:101AE00008045000080078004F04BE000080FA008F
:101AF00000000600889FBE008A9FBE00800078001C
:101B000000C2B3000100370089007800810478002A
:101B100039447800804F5400FBFF3200E94F5400F5
:101B2000F9FF3200D0C2B300804F540004003A00E5
:101B3000194478008184E8001AC0B3000600370019
:101B40000045EB00B0C2B300804F540002003A00E1
:101B5000194478008184E8006022B8000A00370048
:101B6000A2002000030020000400BE0004FB0700C8
:101B70000B4144000281FB000300200000024100F1
:101B800081824900394478000880FB000BFD2F005A
:101B90000B004000E90F5000F1FF36000A04E0009E
:101BA0000200320060021200E0821A000400BE004F
:101BB0004F05BE004F04BE0000000600889FBE0017
:101BC000000478008144780000FD2F0000004400EC
:101BD000E90F500002003E00000178000D003700C0
:101BE0000800780069FA07000000E00003003200F6
:101BF000080078006BFA07000004780008007800FD
:101C000051FA07000000E0000700320090FA2F00B0
:101C1000000144000980FB00800F510002003D00DC
:101C20000280FB0001003700F00F20004F04BE00CF
:101C300000000600881F780060C58000E1030700EF
:101C40000004780038FA07000000E000FAFF3A00CC
:101C5000E10F44000300320061C5800008007800F5
:101C60000C0407004F04780000000600EC874700D2
:101C7000889FBE008A9FBE008C9FBE008E1F78008A
:101C800081BF9F000207780060C588008046EB0096
:101C9000040137008884FB000900780022FA07005D
:101CA000800078000000E00002003200E1FF070041
:101CB000FC00370050C2B300804F5400F0003A00DF
:101CC0000FBD970020C0B300C0EF9F00D1EF9F0071
:101CD00081EF9F000300370040C0B300C0EF9F00BA
:101CE0000FBD97000FB99700B240780082BF9F00E8
:101CF0008184FB0090C6B30080CF500035003200D5
:101D000017003E006640500080CF50006200320055
:101D10000C003E007740500080CF50002800320079
:101D200006003E000104E0009B003200A0C2B300A8
:101D300080CF50006E003A001D00370080C5B30010
:101D40001600370040C6B30080CF5000210032009B
:101D50006440400080CF500065003A001200370018
:101D600030C7B30080CF50001E00320007003E0095
:101D70006740500080CF50001100320063404000A7
:101D800080CF50005A003A001400370050C7B3000B
:101D900080CF50000F0032006340400080CF5000E1
:101DA00053003A006500370020C0B300CBFF370076
:101DB000DFE897008140E800D1EF9F00C8FF3700BF
:101DC0004FE9970080C0B300E24F5100C3FF3A00D3
:101DD000C1FF3700ACC0B300590037008CC0B3005E
:101DE0005700370093FF0700DFE897000104E00089
:101DF00002003A004E017800D2B79F0060C5800013
:101E00007003070000047800E10F4000A2003200D8
:101E10008FEC9700120037000A85E8008ABF9F0008
:101E2000160037008FB897001100FB00800F540098
:101E3000F9FF32005FE997000204E00003003A0076
:101E40005FB0970008587800D0B79F008944E90038
:101E50000A00320060C580005A03070000047800C1
:101E60000800E800E10F5000040036000800780088
:101E7000ADF907000000E000EAFF3200DFE897005C
:101E80000104E00087003A008D46E8005FB197004A
:101E900001497800830037005FE897000004E00004
:101EA00003003A008D46E800CE007800D1B79F00CD
:101EB00060C5800043030700E10F40007600320058
:101EC0005FE997000204E00003003A00DFB09700EA
:101ED00080587800D1B79F000FE997000241E900D0
:101EE00082EF9F004240A9006E003400F0FF3700EF
:101EF0000180FB0008FD2F0008004000E90F5000A2
:101F00005F003E000A0078007F03070080EF9F001B
:101F100088007800030037000FB897000000E80041
:101F200080BF9F000FB997001200FB000100400026
:101F3000E90F5000F8FF360069FF37000CC1B3000D
:101F40003CFF070060C580001E0307000005780005
:101F50000040EB00E0EF9F00D0022000800F550012
:101F600005003A0060C580001603070000057800F0
:101F700011C0B300E1EF9F008C4078000A007800A8
:101F80000EFF0700E14F40000A003A0061C58000E3
:101F90000A0078003F0307000D04E0004B003A0000
:101FA00060C58000300090000048A300430032006C
:101FB000480037008FED97006044B8000C81FB00AB
:101FC000030020000800BE00EDF907000004BE0079
:101FD0008C4078000A007800F8FE07000080FB00C3
:101FE0000100200008044000898448008B45E90076
:101FF0000700320060C58000F2020700000578008B
:102000008C407800EDFE0700E14F4000EBFF3A0006
:102010008C4078000A007800E8FE0700E14F40009D
:1020200003003A0061C580000A0078001903070028
:102030006FE997000204E00002003200600414001F
:10204000E0841C005FE897000004E00015003A00FF
:102050008D46E800CFE89700E4CF500003003A0037
:102060004E0078000888BE000E0037000E81E9009F
:10207000020778001200780008087800090037008D
:1020800060C58000CF020700808F54000500320039
:10209000E10F40000B003A000D04E0000D0032009B
:1020A0000A0037008FB897003144780081BF9F0045
:1020B0000804E000F7FE3A00040037000000EB00DF
:1020C0000500370061C58000F20207000D80FB00AB
:1020D000010037000080EB004F0778004F06BE007C
:1020E0004F05BE004F04BE00CF00B1000000060047
:1020F000FE874700889FBE008A9FBE008C9FBE005F
:102100008E1F7800F0B79F000107780082BF9F0004
:102110000000EB00A0B79F009F0237008006EB0095
:1021200050C2B30080CF5000090032000100FB0014
:10213000FFB0970018030700E10F4000960232003D
:10214000AFB097008100E800A1B79F00920237006E
:102150009E407800D0C2B30080CF50000C00320007
:1021600007003C006D40500080CF50000A00320054
:102170006B40400080CF50000E003A00080037004E
:1021800000C3B30080CF50000A003A0006003700B9
:102190000D30A000050037000D00A000030037003F
:1021A0000D10A000010037000D20A0000E07E80070
:1021B000E7FF37000D18A300010032000D00A10059
:1021C0000D38A300010032000D20A1000100FB002A
:1021D00002FD2F0002004000E90F50000E003E00FB
:1021E0000002EB00C4B79F0082017800CFB29700D5
:1021F0006A28B9001E01FB000001410003014100F3
:10220000C2B79F005E00FB0003004000E90F5000D2
:102210000B003E00F5FF37000006EB00CCB79F0037
:10222000A0C2B30080CF500005003A000FB897005D
:10223000C000780080BF9F00C1B79F000E07E80074
:102240000001EB00B2B79F00E0C2B3009E4F100048
:1022500018003A000DE0A0008E00E8006440500035
:10226000914F100002003200010778000C00370087
:102270000FBA9700C402780084BF9F00B5B79F00D3
:102280000E87E8000B0037003FB697006A60B90080
:102290000000410003004000B0B79F000E07E800B7
:1022A0001E01FB0003FD2F0003004100E90F500059
:1022B000F5FF3600BE407800E1D79F00C0C6B300EE
:1022C00080CF5000220032000F003C0069405000D7
:1022D00080CF50007700320004003C000104E00091
:1022E000310232006B4050000F00370040C6B3008F
:1022F00080CF5000930032006540400080CF5000F6
:102300008B003A008F00370030C7B30080CF5000F9
:102310001A00320007003C006440500080CF50009B
:10232000110032000040E80080CF500080003A00E9
:102330000F00370050C7B30080CF5000800032003C
:102340006340400080CF500079003A000900370018
:10235000000028000D48A30001003A000001200001
:1023600080867600D3FF37000D60A000750037002F
:102370000D50A0000D70A000720037008FB89700BC
:102380004100780081BF9F00000478000000E00059
:1023900001003A00688521008004EB00010037004D
:1023A0008104E80089007800088044001004E000FF
:1023B000FBFF3A003FB197000200E000030032004B
:1023C000890F510001003100820478000002EB0007
:1023D000E4AF9F00CFB29700898F52000200360011
:1023E00009805200E0AF9F004368DE00E106600014
:1023F0001B003A000D06780009003700FFB0970077
:102400000002200064020700E10F400003003200D8
:102410002FB097000000E800A0B79F000C06E8006E
:10242000EFA89700810F5600F4FF3A000081EB00FF
:10243000E2AF9F000A003700880078003100FB00FF
:1024400001047800FFB0970053020700E10F40003D
:10245000030032002FB297000402E800A4B79F00E7
:102460000900E90080047800E10F4000F2FF3A0023
:102470000006EB000D00E0000A003A00C60137003C
:10248000FFB097000002200043020700E10F400068
:1024900003003200AFB297008502E800A5B79F00A5
:1024A0000C06E8006FA89700800F5600F4FF3A0072
:1024B000B90137008FB897004100780081BF9F00B5
:1024C000CF80DE0001017800820178000205BE00A5
:1024D0000004BE000203BE000002BE004822DE006F
:1024E000482EDD0004027600E4D79F000D48A300CB
:1024F0000A0032000404E00008003200E14F42000C
:102500000600320071FD2F0001804700044878006A
:10251000184098002900200002003700F0D79F00E3
:102520001900200072FD2F0002844700A1FF370030
:1025300064FD2F0004844700190020009DFF370030
:102540000D0CB3000D007800000CB20028003A001A
:102550000D00E00005003D008FBA97004505BE0064
:102560004504BE0085BF9F00140037000D48A3003E
:102570000B0032000FBE97004C00BE008CBF9F00C6
:102580004F89DE00CF91DE000002BE00020378001A
:10259000820378000605BE000404BE000700370071
:1025A0008FB897004100780081BF9F000004780039
:1025B000CFC4DE00090578008A057800E00F5400DA
:1025C000E08F5C00E00F5D00E08F5D001F003D00CC
:1025D0003D00B3006000B8006011B800080450006E
:1025E000898458000A0559008B8559001700370067
:1025F0000D00E00005003D000FB997004205BE0048
:102600004204BE0082BF9F00100037000D48A300A7
:10261000070032000FBA97004400BE0084BF9F003D
:102620006011B8000205BE000004BE0007003700BC
:102630008FBA97004500780085BF9F00000478009E
:10264000090020000A0020000B0020003FB6970080
:102650000C00E00007003A00E00F5400E08F5C003F
:10266000E00F5D00E08F5D0002003A0010002000E6
:10267000B0B79F008D007800010CB200E1B79F0059
:1026800000042000808F50003000320003003C0026
:102690000100E00008003200400037000008200080
:1026A0006FB19700800F510014003200000C200021
:1026B000800F510039003A0014C0B300657B21003F
:1026C0000B0037000400FB004300DD000500400064
:1026D0005001BE004000BE000040E10001C8E10022
:1026E00002D0E10003D8E1002B0039000442E800E9
:1026F000F44F5200F3FF3A0027003700000120009A
:10270000010020006011B80014C0B3000040E100D7
:1027100001C8E10002D0E10003D8E1001E00390049
:10272000450020000000D0008180D2000281D2004C
:102730008381D2008502E900FAFF3A000442E800F2
:10274000F04F5200F1FF3A001300370080002000E4
:10275000010020006011B80014C0B3000040E10087
:1027600001C8E10002D0E10003D8E1000A0039000D
:102770003C0020000000D0008180D2000281D20005
:102780008381D2000C06E900FAFF3A000442E80017
:10279000F54F5200F1FF3A00E4D79F00EFD09700C9
:1027A0000100FB003FB19700820F500002003D0086
:1027B000E2D79F00040037003FB29700800F52001D
:1027C00001003D00B0B79F00CFB297000500E000C8
:1027D0000400320063806600020032008502E900D6
:1027E000C5B79F000DE8A3000B0032004FB697005D
:1027F0003FB09700800F560003003C008000EB00C4
:10280000C1B79F00040037004FB197003FB2970057
:1028100004015100C2B79F00EFD297000500FB00F2
:102820000006EB00DCAF9F00CFB09700808F500018
:102830000200340000805000D0AF9F000D28A3009C
:1028400037003200E18066000D18A3000C00320052
:10285000D00220000100E00001003A000080E90001
:10286000FFB097004C010700E10F40000E0032005E
:102870002FB197000201E800A2B79F000A003700BD
:102880000100E00008003200FFB0970000022000C5
:1028900041010700E10F4000030032002FB2970012
:1028A0000402E800A4B79F00DFAA97000500E0003B
:1028B0000F0032000006EB00FFB09700000320007D
:1028C00035010700E10F4000030032002FB09700F0
:1028D0000000E800A0B79F000C06E800DFA8970002
:1028E000810F5600F4FF3A000001EB00D2AF9F00C9
:1028F0003FB29700C320DD00E07A210080804000D5
:1029000091B79F004220DD006400500080B79F0017
:102910006320B900F0AF9F006306500084003700C9
:10292000DFAA97000500E000110032006880660011
:102930000F003A0000067800FFB097000002200068
:1029400015010700E10F4000030032002FB097008F
:102950000000E800A0B79F000C06E800DFA8970081
:10296000810F5600F4FF3A000001EB00D2AF9F0048
:10297000E18066000D18A3000C003200D002200098
:102980000100E00001003A000080E900FFB097007C
:1029900001010700E10F4000D5FF32002FB2970080
:1029A0000402E800A4B79F00D1FF37000100E00057
:1029B000CFFF3200FFB0970000022000F6000700B2
:1029C000E10F4000CAFF3200AFB297008502E80075
:1029D000A5B79F00C6FF370000042000EFB09700A6
:1029E000808F50003100320003003C000100E00005
:1029F000080032003E003700000820006FB1970049
:102A0000800F510011003200000C2000800F510097
:102A100037003A001FB097003002BE002003BE000E
:102A20000800BE000A01BE0062F90700A4002000F1
:102A3000050020006033B80065F9070004C3B30047
:102A400004424000E4D79F0029003700D5852100CB
:102A5000D5B79F000D58A30002003A00E086210080
:102A6000D0B79F0014002000050020006033B8009C
:102A70008FB097008100E900050033000402D00008
:102A80008582D2000683D2008783D200F9FF370007
:102A90000800BE000A01BE0046F907006F00600092
:102AA0005FB19700624078001000370014002000EA
:102AB000050020006033B8000C0078000000E90039
:102AC000050033000402D0008582D2000683D200C4
:102AD0008783D200F9FF37000800BE000A01BE005C
:102AE00034F90700674060000043B000E0D79F0062
:102AF000EFD097000100FB00FFB09700A600070091
:102B0000E10F4000030032002FB197000201E800FE
:102B1000A2B79F001FB297006802520094B79F00AF
:102B20008FB29700E482520085B79F00630656007B
:102B3000D0FF2F003FB197000090B9007FAA970007
:102B40000000420063005000800F5600A2FF3A00D0
:102B50000D38A30010003200DFAA97000500E00046
:102B60000D0034000006EB00FFB0970000022000CB
:102B700089000700E10F4000030032002FB09700EA
:102B80000000E800A0B79F000C06E800DFA897004F
:102B9000810F5600F4FF3A00BE407800E1D79F0055
:102BA0000104E0005DFD3A002FB097004F07780068
:102BB0004F06BE004F05BE004F04BE00EF01B1003E
:102BC00000000600881F780000047800B000900024
:102BD0000148A30007003A000108A30005003200E5
:102BE0000198A30008003200100090000000E000EF
:102BF00005003200380090000040A000300498002A
:102C00008080EB00200037000190A1003104980083
:102C1000180090000000E000060034000000E90009
:102C20001004980018007800B080FB00000C7800B9
:102C300006003700380090000068A300EDFF3A005E
:102C4000080078009B0007008000780038009000A2
:102C50000078A3000C003A00FA8F500008003A00F8
:102C6000280090000000E000E2FF32001800900011
:102C70000000E80010049800180CE900DDFF3700A0
:102C8000ED8F5000E2FF3200010078004F04780021
:102C90000000060080017800E10F400017003200BC
:102CA000310090000008A300140032000098A30037
:102CB00012003A00210290000400E0000F003200F0
:102CC0001101900051009000800F51000B00320064
:102CD00011007800840F500002003A008008E800DC
:102CE000020037000200E800900098001100E9009F
:102CF0008008780003487800010037008081EB00ED
:102D000003007800000006000001780000C2B30054
:102D1000010037000201E8009240780080CF5000A7
:102D2000FCFF3200E9CF5000FAFF3200D0C2B300FE
:102D300080CF500003003A000201E80014C0B30045
:102D4000050037000042EB00B0C2B30080CF500056
:102D500001003A000201E8008000EB0005FD2F00B1
:102D6000040037006A08B900008041008500400077
:102D70000201E8009201FB0005804100E90F5000CC
:102D8000F8FF36000404E000010032008100EA0090
:102D90000100780000000600889FBE000001780056
:102DA00001047800B10090000118A3003D0032003A
:102DB0000198A30003003A00180090000000E00012
:102DC00038003A000190A000310498008204780095
:102DD000F90FB200180090000000E00002003A0075
:102DE00028009000000C7800EA8F540006003A009A
:102DF000380090000078A30003003A0088007800B3
:102E0000D0002000E4FF07009800900058009000D8
:102E1000808F50000B0032000100E8001004980081
:102E20001800780009587800000C780011C0B30031
:102E3000A08A210001487800EA8F54000600320081
:102E40001900370088007800094078006700070003
:102E50008004780014003700380090000088A30038
:102E60001100320018019000A80090004800900066
:102E7000D3F5070098009000810F50000400320045
:102E8000380090000003B300300498008084EB0009
:102E90000000EB001004980028009000000C78005F
:102EA000010037008084EB00090078004F04BE0069
:102EB000000006000200FA00889FBE008A1F78000A
:102EC000000478000000EB00100498003800900027
:102ED0008080EB000008A3003F003200A08A2100A0
:102EE0001004E00010003200298821008A882100A7
:102EF0001A0078006C0545002010B2002110200057
:102F0000810F500002003A00090078007A000700A3
:102F1000EC844400608A2100808F5400F4FF3A0062
:102F2000A08A21000048EB00480090005801900062
:102F30000200E0000D003A00120498001200200088
:102F4000E8805700D5F50700E10F500003003A0074
:102F50000FF897008080FB001F00370038009000BA
:102F60000040A0003004980012003700A800900034
:102F7000CAF50700100498000000E00003003200CA
:102F8000E10F40000D003A000300370038009000C8
:102F90000040A00002003700380090000003B3009A
:102FA00030049800A8009000010C78000000EB00AD
:102FB000100498008080EB0007003700A800900004
:102FC000010C78000000E90010049800010078006E
:102FD000B080FB00000C7800010078004F057800FD
:102FE0004F04BE000080FA00000006000200FA0054
:102FF000889FBE00A0FF9F0001047800B1009000F0
:10300000810478000904B200020032000000FB00D5
:10301000360037000118A30005003A000103B30091
:1030200031049800190498000080EB002F0037004D
:10303000580090000000E00006003A0048009000B0
:1030400012002000E68057005DF507001904980083
:1030500024003700280090000000E00008003A003B
:10306000608A210020049800000C780020002000D5
:1030700050049800100498000130A000310498001A
:1030800018019000A8009000480090004CF507003F
:1030900028009000000C78000080EB0010049800DD
:1030A00018007800AFF8970001587800000C7800FD
:1030B0002FF89700EA4F50000A003A0038009000BD
:1030C0000088A3000700320018019000A8009000BB
:1030D000480090003AF5070019049800A8009000F5
:1030E000010C7800AFF897000100FB004F04BE0010
:1030F0000080FA0000000600881F780000047800B5
:10310000300090000008A300070032008000780023
:103110000120B20004003A0011049800A8009000B9
:10312000010C7800170037000018A30019003200C6
:103130000098A30017003200A80090000100E000F2
:1031400014003200180190000200E000110032006B
:10315000480090001AF5070098009000810F500079
:1031600003003200380090000003B30030049800E0
:103170000000EB001004980028009000000C78007C
:10318000380090000058A300020032000080EB00DD
:10319000010037000000EB004F047800000006003B
:020000040000FA
:0200000401F009
:04000C00FBFF0000F6
:020000040000FA
:0200000401F009
:04001000FDFF0000F0
:020000040000FA
:0200000401F009
:040014007FFF00006A
:020000040000FA
:1000080090020000900200002AD1000030D10000C8
:100018009002000090020000900200009002000090
:10002800900200001CD4000090020000F0ED0000D7
:100038009002000064D400009002000090020000CA
:1000480090020000900200009002000012E30000FD
:100058009002000090020000900200009002000050
:100068009002000090020000900200009002000040
:100078009002000090020000900200009002000030
:10008800900200009002000090020000A2D9000037
:100098004ADA000090020000DEE40000900200004E
:1000A8009002000090020000900200009002000000
:1000B80090020000900200009002000090020000F0
:1000C80090020000900200009002000090020000E0
:1000D80090020000900200009002000090020000D0
:1000E80090020000900200009002000090020000C0
:1000F80090020000900200009002000090020000B0
:10010800900200009002000090020000900200009F
:10011800900200009002000090020000900200008F
:10012800900200009002000090020000900200007F
:10013800900200009002000090020000900200006F
:10014800900200009002000090020000900200005F
:10015800900200009002000090020000900200004F
:10016800900200009002000090020000900200003F
:10017800900200009002000090020000900200002F
:10018800900200009002000090020000900200001F
:10019800900200009002000090020000900200000F
:1001A80090020000900200009002000090020000FF
:1001B80090020000900200009002000090020000EF
:1001C80090020000900200009002000090020000DF
:1001D80090020000900200009002000090020000CF
:1001E80090020000900200009002000090020000BF
:0801F8009002000090020000DB
:020000040000FA
:1002080090020000900200002AD1000030D10000C6
:10021800900200009002000090020000900200008E
:10022800900200001CD4000090020000F0ED0000D5
:100238009002000064D400009002000090020000C8
:1002480090020000900200009002000012E30000FB
:10025800900200009002000090020000900200004E
:10026800900200009002000090020000900200003E
:10027800900200009002000090020000900200002E
:10028800900200009002000090020000A2D9000035
:100298004ADA000090020000DEE40000900200004C
:1002A80090020000900200009002000090020000FE
:1002B80090020000900200009002000090020000EE
:1002C80090020000900200009002000090020000DE
:1002D80090020000900200009002000090020000CE
:1002E80090020000900200009002000090020000BE
:1002F80090020000900200009002000090020000AE
:10030800900200009002000090020000900200009D
:10031800900200009002000090020000900200008D
:10032800900200009002000090020000900200007D
:10033800900200009002000090020000900200006D
:10034800900200009002000090020000900200005D
:10035800900200009002000090020000900200004D
:10036800900200009002000090020000900200003D
:10037800900200009002000090020000900200002D
:10038800900200009002000090020000900200001D
:10039800900200009002000090020000900200000D
:1003A80090020000900200009002000090020000FD
:1003B80090020000900200009002000090020000ED
:1003C80090020000900200009002000090020000DD
:1003D80090020000900200009002000090020000CD
:1003E80090020000900200009002000090020000BD
:0803F8009002000090020000D9
:020000040000FA
:1031A0003078000000000000000000000000000077
:1031B000000000000000000000000000000000000F
:1031C00000000000000000000000000000000000FF
:1031D00000000000000000000000000000000000EF
:1031E00000000000000000000000000000000000DF
:1034000000450000523D0000313000002044000023
:1034100065760000696300006520000054790000B3
:103420007065000020490000732000005365000013
:1034300074200000496E0000636F0000727200008B
:1034400065630000746C00007900000045520000C4
:103450003D310000205500006E61000063630000F4
:103460006570000074610000626C0000652000005F
:1034700050610000726100006D650000746500001D
:10348000722000005265000063650000697600004C
:1034900065640000204900006E200000436F0000BA
:1034A0006D6D0000616E00006400000048000000C7
:1034B000455200003D36000020430000616E0000D0
:1034C0006E6F000074200000457800006563000006
:1034D0007574000065200000436F00006D6D0000F2
:1034E000616E00006420000057680000696C0000F5
:1034F00065200000446500007669000063650000F7
:103500002049000073200000536C00006565000036
:10351000706900006E670000004D00000048000068
:10352000414C00005445000044000000535400008A
:103530004F5000005045000044000000455200007C
:103540003D32000020520000656300006569000004
:103550007665000064200000436F00006D6D000080
:10356000616E0000642000005761000073200000BD
:10357000546F00006F2000004C6F00006E67000069
:10358000005300004554000000450000523D00007B
:1035900037200000436100006E6E00006F74000071
:1035A0002045000078650000637500007465000028
:1035B000204300006F6D00006D6100006E6400002C
:1035C0002057000069740000686F000075740000E7
:1035D00020540000656D0000702000005072000053
:1035E0006F620000652000004174000074610000FB
:1035F000636800006564000000450000523D000063
:1036000039200000436100006E6E00006F740000FE
:103610002050000075730000682000005365000012
:1036200074740000696E0000677300002E200000B3
:103630004E65000063650000737300006172000056
:10364000792000005365000074740000696E00006A
:10365000677300002041000072650000204D0000EB
:1036600069730000736900006E670000005300007A
:10367000544F00005245000000450000523D00003C
:1036800038200000436F00006D6D0000756E000073
:103690006963000061740000696F00006E20000023
:1036A000707200006F6200006C6500006D20000009
:1036B000776900007468000020570000692D000041
:1036C00046690000204200006F6100007264000043
:1036D0000044000045460000415500004C540000E5
:1036E0005300000052450000534500005400000004
:1036F00053430000414E000000450000523D0000D1
:1037000031310000204900006E6300006F6D000041
:103710007061000074690000626C000065200000A8
:1037200046690000726D000077610000726500005C
:103730002056000065720000736900006F6E000083
:103740000025000064000000257500000045000011
:10375000523D000033200000556E00006B6E0000EB
:103760006F7700006E200000436F00006D6D000059
:10377000616E000064200000526500006365000077
:103780006976000065640000002500006C7500008B
:1037900000450000523D000035200000436100005C
:1037A0006E6E00006F740000204500007865000018
:1037B0006375000074650000204300006F6D000019
:1037C0006D6100006E640000202D000020440000A8
:1037D0006576000069630000652000004973000001
:1037E000204E00006F740000204800006F6D000044
:1037F0006564000000000000000000000000000000
:1038000000000000434F00004E4600004947000002
:10381000004E0000696300006B6E0000616D0000E7
:10382000652000003D200000004D00006178000090
:10383000205000006F730000202000003D20000099
:1038400000440000657600002054000079700000FC
:10385000202000003D20000000540000436F0000C5
:103860006D700000204F00004E2000003D20000041
:1038700000540000656D0000704300006F200000E0
:10388000412000003D20000000540000656D000054
:10389000704300006F200000422000003D20000027
:1038A00000540000656D0000704300006F200000B0
:1038B000432000003D20000000540000656D000022
:1038C000704300006F200000442000003D200000F5
:1038D00000540000656D0000704300006F20000080
:1038E000452000003D20000000540000432000005F
:1038F0004D6F000064650000202000003D200000A6
:10390000004200004C430000204500006E200000F3
:10391000202000003D200000004200004C43000039
:103920002053000074700000732000003D20000050
:10393000004C00004544000020420000727400006A
:10394000202000003D200000005400004340000003
:103950005374000061720000742000003D200000DC
:10396000004500004E440000000000000000000080
:103970000000000000000000000000000000000047
:103980000053000054410000545500005300000053
:10399000546500006D7000002843000029200000DD
:1039A000203D0000200000004375000072720000FE
:1039B000205000006F730000203D00002000000038
:1039C0005461000072670000205000006F73000017
:1039D000203D000020000000497300004D6F0000F2
:1039E000766900006E670000203D000020000000A6
:1039F00049730000486F00006D6900006E670000A9
:103A0000203D00002000000049730000486F0000C6
:103A10006D65000064200000203D000020000000D3
:103A200046460000446500007465000063740000B1
:103A3000203D000020000000546D00007050000088
:103A4000726F000062650000203D00002000000051
:103A5000526500006D6F000074650000494F000062
:103A6000203D000020000000486E0000642000009F
:103A7000437400006C720000203D00002000000034
:103A8000526500007665000072730000652000003A
:103A9000203D00002000000053430000414E000084
:103AA000204900004E4600004F0000005363000014
:103AB000616E00002020000049440000203D00000D
:103AC000202500006400000053430000204900004E
:103AD0006E64000065780000203D00002025000095
:103AE000640000004E650000744300006F75000024
:103AF0006E740000203D00002025000064000000DE
:103B000053630000616E00005353000049440000FD
:103B1000203D0000200000005365000063200000ED
:103B20004D6F000064650000203D0000202500006E
:103B3000640000004E65000074200000547900000D
:103B400070650000203D000020250000640000009A
:103B500053690000672000002053000074720000C9
:103B6000203D000020250000640000004C6F000094
:103B700061640000446F00006E650000203D00009D
:103B80002025000064000000322E0000332E0000CB
:103B900030000000000000000000000000000000F5
:103BA0000000000000000000485500004220000016
:103BB000494E0000464F00000048000075620000BA
:103BC0002046000056650000722000003D200000E5
:103BD000005300006C65000065700000696E000015
:103BE000672000003D2000000057000069720000BF
:103BF0006564000020490000502000003D200000C6
:103C0000004400004843000050690000734F00006A
:103C10006E2000003D2000000057000046200000FC
:103C20004174000063680000642000003D20000033
:103C30000057000046200000436F00006E6E000039
:103C4000202000003D20000000570000462000001A
:103C50004656000065720000202000003D20000054
:103C6000005700004620000046560000204F00008C
:103C70004B2000003D2000000057000046200000BF
:103C80005353000049440000202000003D20000064
:103C9000005700004620000049500000202000008E
:103CA000202000003D2000000057000046200000BA
:103CB00053650000634D0000642000003D200000BB
:103CC000005700004620000053650000634B0000D1
:103CD000792000003D200000005700004620000031
:103CE00057650000704B0000492000003D20000097
:103CF0000044000049410000472E0000205200000F
:103D0000455000004F520000540000005065000074
:103D1000726900006F640000203100002C20000058
:103D2000322000003D200000256400002C2000000F
:103D3000256400000050000065720000696F0000FB
:103D4000642D00004F200000312C000020320000C4
:103D5000203D000020250000642C000020250000EC
:103D600064000000507200006573000073200000C2
:103D7000312C000020320000203D000020250000F2
:103D8000642C00002025000064000000436F000048
:103D90006E200000312C000020320000203D000089
:103DA00020250000642C0000202500006400000095
:103DB000526F00006C6C0000204F00007665000020
:103DC000722000003D200000256400000054000027
:103DD000696D000065720000203D00002025000094
:103DE0006C75000000530000454300002E200000C9
:103DF00052450000504F0000525400000054000093
:103E0000696D000065730000746100006D70000052
:103E1000203D0000202500006C6C000075000000B3
:103E2000484D000041430000203D000020000000FC
:103E30002530000032580000005200006576000076
:103E400069730000696F00006E2000003D200000D3
:103E500025750000004C00006F6300006B2000001F
:103E60003D2000002575000000560000657200002E
:103E7000736900006F6E0000203D000020250000E7
:103E800075000000426C00006F6300006B200000B2
:103E90003D200000256C0000750000004843000034
:103EA0002053000045540000544900004E470000D4
:103EB000530000005363000072650000656E00004F
:103EC00073200000203D0000202500007500000048
:103ED000484300002046000057560000657200006D
:103EE000203D000020000000000000000000000055
:103EF0000000000000540000454D0000502000006C
:103F0000434F00004D50000000540000656D00005C
:103F1000704900006E200000412000003D2000009C
:103F200000540000656D0000704900006E20000024
:103F3000422000003D20000000540000656D00009C
:103F4000704900006E200000432000003D2000006A
:103F500000540000656D0000704900006E200000F4
:103F6000442000003D20000000540000656D00006A
:103F7000704900006E200000452000003D20000038
:103F8000005300007465000070530000697A00005F
:103F9000652000003D20000000000000000000003F
:103FA0000000000000000000000000000000000011
:103FB0000000000000000000000000000000000001
:103FC00000000000000000000000000000000000F1
:103FD00000000000000000000000000000000000E1
:103FE00000000000000000000000000000000000D1
:103FF00000000000000000000000000000000000C1
:1040000000000000000000000000000000000000B0
:1040100000000000000000000000000000000000A0
:104020000000000000000000000000000000000090
:1040300000000000000000000048000055420000A1
:104040002049000050200000494E0000464F00006B
:104050000043000075720000722E0000204900002D
:10406000502000003D200000256400002E250000A7
:10407000642E0000256400002E250000640000006E
:1040800043750000722000004D610000736B00005A
:10409000203D000020250000642E00002564000063
:1040A0002E250000642E000025640000004700005B
:1040B0006174000065770000617900002020000035
:1040C0003D200000256400002E250000642E000025
:1040D000256400002E2500006400000050720000DE
:1040E000692E0000204400004E530000203D0000D7
:1040F00020250000642E0000256400002E2500000D
:10410000642E000025640000005300006563000079
:104110002E200000444E0000532000003D200000EF
:10412000256400002E250000642E00002564000098
:104130002E2500006400000044650000662E00008B
:104140002049000050200000203D000020250000F4
:10415000642E0000256400002E250000642E00005F
:104160002564000000440000656600002E4D00003C
:10417000617300006B2000003D20000025640000FA
:104180002E250000642E0000256400002E2500006E
:10419000640000004448000043500000202000005C
:1041A0004F6E0000203D000020250000640000004C
:1041B0004E65000074420000494F0000532000008B
:1041C000203D000020250000730000004D4100004C
:1041D000432000004164000064720000203D0000A4
:1041E0002025000073000000000000000000000017
:1041F00000000000000000000000000000000000BF
:1042000000000000000000000000000000000000AE
:10421000000000000000000000000000000000009E
:10422000000000000000000000000000000000008E
:10423000000000000000000000000000000000007E
:10424000000000000000000000000000000000006E
:10425000000000000000000000000000000000005E
:10426000000000000000000000000000000000004E
:10427000000000000000000000000000000000003E
:1042800000000000000000005749000046490000FF
:104290002049000050200000494E0000464F000019
:1042A000004300006F6E0000666900006720000098
:1042B0004D2000003D2000002564000000000000AB
:1042C00000000000000000000000000000000000EE
:1042D00000000000000000000000000000000000DE
:1042E00000000000000000000000000000000000CE
:1042F00000000000000000000000000000000000BE
:1043000000000000000000000000000000000000AD
:10431000000000000000000000000000000000009D
:10432000000000000000000000000000000000008D
:1043300000000000004E00006577000020480000EB
:104340007562000020490000502000003D20000060
:10435000256400002E250000642E00002564000066
:104360002E250000640000004E650000772000004C
:1043700048750000622000004D610000736B000072
:10438000203D000020250000642E00002564000070
:104390002E250000642E000025640000004E000061
:1043A000657700002048000075620000204700008B
:1043B000572000003D200000256400002E2500004D
:1043C000642E0000256400002E250000640000001B
:1043D0004E65000077200000487500006220000054
:1043E0004448000043500000203D0000202500000C
:1043F000640000004E65000077200000576900004F
:104400004669000020490000502000003D200000C7
:10441000256400002E250000642E000025640000A5
:104420002E250000640000004E650000772000008B
:104430005769000046690000204D000061730000CC
:104440006B2000003D200000256400002E250000A8
:10445000642E0000256400002E250000640000008A
:104460004E65000077200000576900004669000093
:1044700020470000572000003D2000002564000078
:104480002E250000642E0000256400002E2500006B
:10449000640000004E6500007720000057690000AE
:1044A00046690000204400004843000050200000FE
:1044B0003D20000025640000000000006865000049
:1044C00061640000657200002E6900006E630000E8
:1044D000006600006F6F000074650000722E00001F
:1044E000696E0000630000002144000045460000A2
:1044F000000D00000A000000747800007400000045
:10450000687400006D000000687400006D6C0000AD
:104510000063000067690000007800006D6C000017
:10452000006300007373000000670000696600000C
:10453000007000006E670000006A000070670000F5
:10454000006300006C6100000077000061760000ED
:104550000000000000000000000000007CA200003D
:1045600080A2000084A2000089A200008DA20000A9
:1045700091A2000095A2000099A200009DA2000057
:10458000A1A20000A5A20000A9A20000746500007D
:10459000787400002F7000006C610000696E0000EC
:1045A0000074000065780000742F0000687400003B
:1045B0006D6C00000074000065780000742F00002E
:1045C000786D00006C0000007465000078740000D5
:1045D0002F63000073730000006900006D6100002C
:1045E000676500002F670000696600000069000031
:1045F0006D610000676500002F7000006E670000AD
:10460000006900006D610000676500002F6A00000E
:10461000706500006700000061700000706C0000B1
:104620006963000061740000696F00006E2F000074
:104630006A610000766100002D7600006D000000C8
:1046400061750000646900006F2F0000782D000084
:10465000776100007665000000000000C6A200003F
:10466000D1A20000D1A20000D1A20000DBA2000074
:10467000E4A20000EDA20000F7A2000001A30000E8
:104680000CA3000020A300002DA30000485400004C
:10469000545000002F3100002E3100002032000065
:1046A00030300000204F00004B0D00000A43000096
:1046B0006F6E00006E65000063740000696F00009B
:1046C0006E3A0000206300006C6F0000736500000C
:1046D0000D0A00000048000054540000502F000054
:1046E000312E000031200000343000003020000066
:1046F00042610000642000005265000071750000F6
:1047000065730000740D00000A4300006F6E000026
:104710006E65000063740000696F00006E3A00006F
:10472000206300006C6F0000736500000D0A00003C
:104730000D0A00003430000030200000426100000B
:104740006420000052650000717500006573000070
:10475000743A000020630000616E000027740000BE
:1047600020680000616E0000646C0000652000009D
:10477000436F00006E740000656E0000742D000031
:104780004C6500006E670000746800000D0A0000B0
:104790000048000054540000502F0000312E00004B
:1047A000312000003430000031200000556E000040
:1047B00061750000746800006F720000697A000083
:1047C000656400000D0A000057570000572D0000D7
:1047D0004175000074680000656E00007469000097
:1047E00063610000746500003A200000426100002F
:1047F000736900006320000072650000616C0000B6
:104800006D3D000022500000726F000074650000D2
:104810006374000065640000220D00000A4300007C
:104820006F6E00006E65000063740000696F000029
:104830006E3A0000206300006C6F0000736500009A
:104840000D0A00000D0A0000343000003120000085
:10485000556E000061750000746800006F72000002
:10486000697A0000656400003A2000005061000091
:1048700073730000776F0000726400002072000004
:10488000657100007569000072650000640D00002C
:104890000A00000048540000545000002F3100006E
:1048A0002E3100002034000030340000204E000083
:1048B0006F740000206600006F7500006E640000D9
:1048C0000D0A0000436F00006E6E0000656300007B
:1048D000746900006F6E00003A200000636C0000F5
:1048E0006F730000650D00000A4300006F6E00004A
:1048F000746500006E7400002D5400007970000093
:10490000653A00002074000065780000742F0000F4
:10491000687400006D6C00000D0A00000D0A0000B4
:1049200034300000343A000020460000696C00007A
:10493000652000006E6F000074200000666F0000AC
:10494000756E0000643C0000627200003E5500007D
:1049500073650000203C00006120000068720000C8
:10496000656600003D2200002F750000706C00009D
:104970006F610000642200003E4D000050460000C0
:1049800053200000557000006C6F0000616400004F
:104990003C2F0000613E0000207400006F200000EA
:1049A000707200006F670000726100006D200000EF
:1049B00077650000622000007061000067650000FC
:1049C000730D00000A00000048540000545000001D
:1049D0002F3100002E31000020340000313400005F
:1049E00020520000657100007565000073740000BE
:1049F0002D55000052490000205400006F6F000048
:104A0000204C00006F6E0000670D00000A4300009C
:104A10006F6E00006E65000063740000696F000037
:104A20006E3A0000206300006C6F000073650000A8
:104A30000D0A00000D0A000034310000342000008F
:104A4000526500007175000065730000742D000050
:104A50005552000049200000546F00006F200000F4
:104A60004C6F00006E6700003A20000042750000A5
:104A70006666000065720000206F00007665000029
:104A8000726600006C6F0000772000006465000013
:104A90007465000063740000656400000D0A000086
:104AA0000048000054540000502F0000312E000038
:104AB000312000003530000030200000496E000039
:104AC00074650000726E0000616C000020530000ED
:104AD00065720000766500007220000045720000DB
:104AE000726F0000720D00000A4300006F6E00003C
:104AF0006E65000063740000696F00006E3A00008C
:104B0000206300006C6F0000736500000D0A000058
:104B10000D0A00003530000030200000496E000012
:104B200074650000726E0000616C0000205300008C
:104B3000657200007665000072200000457200007A
:104B4000726F0000723A000020450000787000008B
:104B5000656300007465000064200000646100006B
:104B600074610000206E00006F740000207000006F
:104B700072650000736500006E7400000D0A00008D
:104B80000048000054540000502F0000312E000057
:104B90003120000035300000312000004E6F000051
:104BA00074200000496D0000706C0000656D00000D
:104BB000656E000074650000640D00000A4300008B
:104BC0006F6E00006E65000063740000696F000086
:104BD0006E3A0000206300006C6F000073650000F7
:104BE0000D0A00000D0A00003530000031200000E1
:104BF0004E6F000074200000496D0000706C0000D2
:104C0000656D0000656E000074650000643A000088
:104C1000204F00006E6C0000792000004745000026
:104C200054200000616E000064200000504F00001E
:104C3000535400002073000075700000706F000076
:104C400072740000656400000D0A00000048000056
:104C500054540000502F0000312E0000312000007D
:104C600032300000302000004F4B00000D0A0000E1
:104C7000436F00006E6E0000656300007469000001
:104C80006F6E00003A200000636C00006F7300003C
:104C9000650D00000A4300006F6E0000746500009F
:104CA0006E7400002D54000079700000653A000019
:104CB0002074000065780000742F00006874000004
:104CC0006D6C00000D0A00000D0A00003C68000039
:104CD000746D00006C3E00003C6200006F640000D8
:104CE0007920000073740000796C0000653D0000BD
:104CF000226D000061720000676900006E3A0000DA
:104D00003130000030700000782200003E3C00008E
:104D1000666F0000726D0000206D00006574000079
:104D2000686F0000643D0000706F00007374000045
:104D30002061000063740000696F00006E3D000098
:104D4000222F0000757000006C6F0000616400008D
:104D500022200000656E000063740000797000007E
:104D6000653D0000226D0000756C00007469000054
:104D700070610000727400002F6600006F72000006
:104D80006D2D00006461000074610000223E00008F
:104D90003C6200003E4D00005046000053200000E1
:104DA000496D00006167000065200000557000003B
:104DB0006C6F0000616400003C2F0000623E000048
:104DC0003C7000003E3C0000696E00007075000001
:104DD0007420000074790000706500003D660000DA
:104DE000696C0000652000006E6100006D650000C8
:104DF0003D69000020730000697A0000653D0000F5
:104E0000343000003E200000266E00006273000077
:104E1000703B0000203C0000696E000070750000CF
:104E20007420000074790000706500003D7300007C
:104E3000756200006D69000074200000766100005A
:104E40006C750000653D000022550000706C00008C
:104E50006F610000642200003E3C00002F660000ED
:104E60006F7200006D3E00003C2F0000626F00007A
:104E7000647900003E3C00002F680000746D000063
:104E80006C3E00000048000054540000502F000009
:104E9000312E0000312000003230000030200000B0
:104EA0004F4B00000D0A0000436F00006E6E0000C3
:104EB00065630000746900006F6E00003A20000016
:104EC000636C00006F730000650D00000A43000072
:104ED0006F6E0000746500006E7400002D540000B9
:104EE00079700000653A00002074000065780000C9
:104EF000742F0000687400006D6C00000D0A000043
:104F00000D0A00003C680000746D00006C3E00005B
:104F10003C6200006F6400007920000073740000A0
:104F2000796C0000653D0000226D00006172000098
:104F3000676900006E3A00003130000030700000F8
:104F4000782200003E3C0000623E00004D50000010
:104F5000465300002055000070640000617400009A
:104F60006520000053750000636300006573000056
:104F700073660000756C00003C2F0000623E00006C
:104F80003C7000003E3C00006120000068720000A0
:104F9000656600003D2200002F2200003E53000005
:104FA00069740000652000006D610000696E0000FA
:104FB0002070000061670000653C00002F61000068
:104FC0003E3C00002F6200006F640000793E00004C
:104FD0003C2F0000687400006D6C00003E00000073
:104FE00048540000545000002F3100002E310000C2
:104FF0002035000030300000204900006E740000B1
:10500000657200006E6100006C20000053650000B6
:105010007276000065720000204500007272000088
:105020006F7200000D0A0000436F00006E6E0000FA
:1050300065630000746900006F6E00003A20000094
:10504000636C00006F730000650D00000A430000F0
:105050006F6E0000746500006E7400002D54000037
:1050600079700000653A0000207400006578000047
:10507000742F0000687400006D6C00000D0A0000C1
:105080000D0A00003C680000746D00006C3E0000DA
:105090003C6200006F64000079200000737400001F
:1050A000796C0000653D0000226D00006172000017
:1050B000676900006E3A0000313000003070000077
:1050C000782200003E3C0000623E00004D5000008F
:1050D00046530000204900006D6100006765000034
:1050E000204300006F7200007275000070740000B1
:1050F000206F000072200000577200006F6E0000E9
:10510000672000005665000072730000696F0000A0
:105110006E3C00002F6200003E3C0000703E00002C
:105120003C6100002068000072650000663D0000E0
:10513000222F0000757000006C6F00006164000099
:10514000223E0000547200007920000061670000D8
:10515000616900006E3F00003C2F0000613E0000CE
:105160003C2F0000626F0000647900003E3C0000AC
:105170002F680000746D00006C3E000000480000C5
:1051800054540000502F0000312E00003120000048
:105190003330000032200000466F0000756E0000C2
:1051A000640D00000A4300006F6E00006E65000091
:1051B00063740000696F00006E3A00002063000015
:1051C0006C6F0000736500000D0A00004C6F00005A
:1051D00063610000746900006F6E00003A200000F7
:1051E0000048000054540000502F0000312E0000F1
:1051F000312000003430000033200000466F0000F2
:105200007262000069640000646500006E0D0000B9
:105210000A4300006F6E00006E65000063740000BA
:10522000696F00006E3A0000206300006C6F0000A0
:10523000736500000D0A00000D0A00003430000004
:1052400033200000466F00007262000069640000B5
:10525000646500006E3A000020530000534C0000CB
:105260002052000065710000756900007265000041
:10527000642000002D2000007573000065200000F0
:105280004854000054500000530D00000A00000074
:1052900046A3000046A300006BA30000C9A30000C2
:1052A0004AA40000E4A4000051A50000C1A500002C
:1052B00027A600002DA3000043A70000F0A70000D0
:1052C000BFA80000F1A80000436F00006F6B000052
:1052D000696500003A000000417500007468000034
:1052E0006F720000697A000061740000696F00004D
:1052F0006E3A0000004300006F6E0000746500000D
:105300006E7400002D4C0000656E00006774000094
:10531000683A00000000000064A900006CA90000C9
:105320007BA900004745000054000000504F0000DA
:105330005354000000750000706C00006F610000A5
:1053400064000000666F0000637500007365000074
:10535000723100002E680000746D0000000D000026
:105360000A0D00000A330000303400002052000013
:10537000656400006972000065630000743A000013
:1053800020000000436F00006E740000656E000096
:10539000742D000054790000706500003A20000070
:1053A000004300006F6E0000746500006E74000022
:1053B0002D4500006E6300006F640000696E000000
:1053C000673A0000206700007A690000700D000055
:1053D0000A0000004361000063680000652D0000C2
:1053E000436F00006E740000726F00006C3A0000A2
:1053F000200000006E6F00002D630000616300005C
:1054000068650000006D0000617800002D610000FB
:10541000676500003D0000003630000030000000ED
:1054200053650000742D0000436F00006F6B000097
:10543000696500003A200000000D00000A0D000020
:105440000A0000000D0A00000D0A00004D50000087
:105450004653000002010000000000004845000023
:105460004C4C00004F000000484100004C5400002C
:10547000004800004F4D000045000000434500007B
:105480004E54000045520000004D0000314900001C
:10549000004D0000314F0000004D00004F52000051
:1054A000004D000049520000004D00004100000086
:1054B000455200004D000000534C000045450000DF
:1054C00050000000574100004B450000004700001D
:1054D000455400005354000041540000555300004F
:1054E0000047000045540000434F00004E460000B6
:1054F00049470000005300004344000054000000EE
:105500005343000054430000005300004354000084
:105510004D000000534300005445000000530000BC
:105520004354000053000000534300004E4E00005F
:1055300000530000434200005300000053430000AA
:105540004245000000530000434C000042000000B0
:105550005343000043500000004700004554000042
:1055600048550000424900004E4600004F00000030
:1055700052450000534500005400000053570000FE
:105580005353000000530000575300004D0000002B
:1055900053570000534B00000053000057570000C2
:1055A000490000005357000050530000005700000E
:1055B0004946000049520000455300004554000090
:1055C00000570000494600004944000045460000DD
:1055D000415500004C5400005300000044490000B5
:1055E00041470000005300004950000048000000FF
:1055F00047490000504800000053000041490000A6
:10560000505300004F460000460000005341000088
:1056100049500000534F00004E000000534D000061
:1056200056480000004700004D56000048000000AA
:10563000474100004950000000530000495000005D
:105640005300000052450000564500005253000030
:105650004500000053450000544D00004158000033
:105660000053000045540000494E00005400000063
:105670004745000054540000434900000053000017
:1056800045540000465300005300000057490000F5
:105690004649000053430000414E0000004700000F
:1056A000455400004E450000540000004C4F0000DF
:1056B000414400004E4500005400000052450000E7
:1056C000424F00004F5400000047000045540000C6
:1056D00048490000500000004745000054570000B2
:1056E00049500000004700004554000050490000A8
:1056F000500000005345000054570000495000007E
:105700000053000045540000575300004D000000B6
:105710005345000054570000534700000053000059
:10572000455400005753000044000000534100005E
:105730005645000057460000005300004554000045
:105740005349000050000000534500005448000039
:10575000534D000000530000455400004853000022
:105760004700000053450000544800005344000027
:105770000053000041560000454900005000000061
:1057800053490000505200005354000000470000ED
:1057900045540000484300005300000053450000FA
:1057A00054480000535300000053000045540000CB
:1057B0004843000056000000534B000045590000CC
:1057C0000053000045540000465400005300000000
:1057D00053450000544600004353000000530000AE
:1057E00041560000455300004300000047450000BB
:1057F000545300004543000000530000455400008E
:105800005454000053000000707200006F740000D8
:105810006563000074000000736E00006D7000008E
:1058200000610000646D0000696E0000006D000002
:1058300069630000726F0000636800006970000017
:105840000000000000000000000000000000000058
:105850000000000000000000000000000000000048
:105860000000000000000000000000000000000038
:10587000736500006E640000436D0000640000006A
:10588000455200003D330000205500006E6B0000C3
:105890006E6F0000776E0000204300006F6D000007
:1058A0006D6100006E64000020520000656300001E
:1058B000656900007665000064000000666F000006
:1058C0006375000073650000723100002E680000EF
:1058D000746D000000700000726F000074650000BD
:1058E000637400002F6300006F6E000066690000A3
:1058F000672E0000687400006D00000069700000F1
:10590000006700007700000073750000620000006F
:10591000646E000073310000006400006E730000CC
:10592000320000006D61000063000000686F00003D
:1059300073740000006400006863000070000000E1
:105940002F700000726F0000746500006374000027
:105950002F720000656200006F6F0000742E00005F
:10596000687400006D3F0000002F0000707200009E
:105970006F74000065630000742F0000636F000007
:105980006E660000696700002E680000746D0000FC
:105990000046000065620000203100003220000057
:1059A000323000003138000020310000313A000070
:1059B000303800003A320000340000007635000034
:1059C0002E340000320000006E6100006D650000A2
:1059D000006E00006F74000020730000657400000A
:1059E000003C0000623E0000557000006C6F00003B
:1059F000616400002061000020460000696C000026
:105A0000653C00002F6200003E000000636800005B
:105A1000656300006B6500006400000066610000C3
:105A2000696C00000054000068650000204400001C
:105A3000796E0000616D0000696300002044000081
:105A40004E530000204300006C690000656E0000AA
:105A50007420000069730000206E00006F74000065
:105A6000206500006E610000626C0000656400004B
:105A70002E0000006E6F00006E65000000620000E6
:105A80006C6F0000636B000000000000000000006D
:105A90000000000000000000000000000000000006
:105AA00000000000000000000000000000000000F6
:105AB00000000000000000000000000000000000E6
:105AC00000000000000000000000000000000000D6
:105AD00000000000000000000000000000000000C6
:105AE00000000000000000000000000000000000B6
:105AF00000000000000000000000000000000000A6
:105B00000000000000000000000000000000000095
:105B100000000000000000003130000032310000C1
:105B2000313000003232000030450000523D0000AC
:105B300033200000556E00006B6E00006F77000090
:105B40006E200000436F00006D6D0000616E00006C
:105B50006420000052650000636500006976000063
:105B60006564000000450000523D00003220000046
:105B700052650000636500006976000065640000FE
:105B8000204300006F6D00006D6100006E64000036
:105B90002057000061730000205400006F6F000068
:105BA000204C00006F6E0000670000002100000024
:105BB000455200003D330000205500006E6B000090
:105BC0006E6F0000776E0000204300006F6D0000D4
:105BD0006D6100006E6400002052000065630000EB
:105BE0006569000076650000640000004552000011
:105BF0003D3200002052000065630000656900002E
:105C00007665000064200000436F00006D6D0000A9
:105C1000616E0000642000005761000073200000E6
:105C2000546F00006F2000004C6F00006E67000092
:105C30000021000000000000455200003D3300003C
:105C4000205500006E6B00006E6F0000776E000044
:105C5000204300006F6D00006D6100006E64000065
:105C60002052000065630000656900007665000051
:105C700064000000455200003D3200002052000048
:105C8000656300006569000076650000642000001F
:105C9000436F00006D6D0000616E00006420000025
:105CA0005761000073200000546F00006F20000057
:105CB0004C6F00006E670000002100000000000033
:105CC000455200003D330000205500006E6B00007F
:105CD0006E6F0000776E0000204300006F6D0000C3
:105CE0006D6100006E6400002052000065630000DA
:105CF0006569000076650000640000004552000000
:105D00003D3200002052000065630000656900001C
:105D10007665000064200000436F00006D6D000098
:105D2000616E0000642000005761000073200000D5
:105D3000546F00006F2000004C6F00006E67000081
:105D4000002100000000000008000000C800000062
:105D50002C01000008000000C80000002C01000019
:105D600008000000C80000002C0100000A0000002C
:105D700000020000800000000A0000000002000095
:105D8000800000000A000000000200008000000007
:105D90000D0A000044480000435000002F5000004E
:105DA0006F770000657200002065000076650000D6
:105DB0006E740000206F00006363000075720000C5
:105DC000726500006400000000040000A3000000F1
:105DD00000000000464F000043550000534C0000F7
:105DE000594E0000580000004D500000465300007E
:085DF0000201000000000000A8
:020000040000FA
:105DF8000000FA00889FBE0029C3B300090078009C
:105E0800C2E9B70030C3B300C3E9B70008C3B300A1
:105E180008007800C4E9B7000303200062B8200036
:105E28000004200001002000F0E002000000000053
:105E38007B0E0700B05D8800C15D8800C969EF006E
:105E48000004FD00DAE9B700DBE9B700DCE9B700D8
:105E5800C5E9B700C6E9B7000004FD0008007800EE
:105E6800C7E9B70010C3B300E0E8B700090078003D
:105E7800C0E9B70010C0B3002CE8B70040C6B300B3
:105E88000CE9B700A0112000E0438800C0112000F1
:105E9800E04A880000182000F043880060182000BD
:105EA800F04A8800208020004B000700208E200048
:105EB80049000700DED30200000000002AD90200D2
:105EC800000000000F0EB00001F22F000180470013
:105ED800228E20006F00090032187800000EB100F1
:105EE8000F0EB00001804700218020006F000900DC
:105EF80031187800000EB10042E6020000000000F0
:105F080000E42F0080874700E2000700208020007F
:105F1800C6140700208E2000C414070086C8BF00DE
:105F28000038A300040032002080200006B30200DD
:105F380000000000040037002D08AB00020032000A
:105F480010C0B30054E8B70066C9BF000038A3000A
:105F580004003200208E200006B30200000000007A
:105F6800040037000D09AB000200320010C0B30076
:105F780034E9B700504E8000E50F400001003E00B4
:105F8800CAA9EF00C1478000A0A52500808F500056
:105F980002003A000040EB00B400070092ED020056
:105FA8000000000060BA880071BA880092ED020013
:105FB80000000000E0468800F146880092ED0200EB
:105FC80000000000E04D8800F14D88004F04BE003D
:105FD8000080FA00000006000000FA00889FBE005A
:105FE8008A1F78008004780060D891005ADB02008C
:105FF800000000000040EB00D0F498006000B800FA
:1060080090049800A1049800B0049800C104980076
:10601800495090000004A100441607000014A10094
:10602800421607000024A100401607000064A100E2
:106038003E1607000074A1003C1607000044A100AA
:10604800C054980010C0B300E0CC98000900780054
:1060580008BF0200000000000004E00002003A004F
:106068000045780046003700E0C4B300805C980023
:10607800F0C6B300905C980002C2B300A25C98001E
:1060880040C4B300B05C980051C6B300C15C98002E
:1060980060C7B300D05C98006D405000E05C980089
:1060A80066405000F05C9800816498009264980003
:1060B80069D89100A06498008040EB00B164980012
:1060C800C1649800D1649800591090000080A10024
:1060D800D0149800A0C5B300E0549800F05498007C
:1060E800A14C9800A1D4980060052000E014980005
:1060F800F0149800801C9800901C9800A01C980030
:10610800C0DA2000B01C9800C01C9800D01C980071
:10611800E01C9800F01C980010C4B30080C49800DC
:1061280079405000E0F49800494091000004A10033
:10613800C0449900B0C4B300906C980049409100E5
:106148000044A100C04499006000B800C02C980029
:10615800D12C98000F0EB00000F22F0000844700E9
:106168006F000900391C7800080EB100090EB10053
:106178007AC00200000000001AC0B3008807780047
:106188008A407800090078004CDE02000000000018
:10619800494091000038A30009003A0049289000BE
:1061A800D9289000E00F5000E08F5800040032001A
:1061B80049289000D9289000A02C9800B12C98006C
:1061C8000A04E0000E003A00494091000038A3009C
:1061D8000B003A0069009000F900900090049800C4
:1061E800A104980069009000F9009000B00498009C
:1061F800C1049800495090000024A000C0549800A1
:1062080069D8910068DB0200000000004F057800A3
:106218004F04BE000080FA0000000600881F7800C6
:10622800D8D5BF0001C4B3000144600007003A009C
:1062380008407800DC9B020000000000084078005D
:1062480046CA020000000000060037000040EB00CC
:10625800EC9B0200000000000040EB0054CA020062
:10626800000000004F047800000006000004E00071
:1062780002003A00CA29A90005003700514E8000E3
:106288000180EA006200600080806800514E88004A
:106298000000060090C1BF0081CFB300014060003C
:1062A8006040B30090E1B7009061A8002BC8BF0020
:1062B8000080FB00600C88000000060000417800A8
:1062C8008101780010C3B300804F51000D003A00DF
:1062D80010BA80007600B900A2BB20007D15070027
:1062E80010BA800003BA8000801507000100320050
:1062F8004237EC0010BA80008F15070011BA8800E9
:106308001F00370020C3B300804F51000D003A0032
:1063180030BA80007600B900A2D120006D150700C0
:1063280030BA800023BA80007015070001003200DF
:106338004637EC0030BA80007F15070031BA880074
:106348000F00370080C4B300804F51000C003A00A2
:1063580050BA80007600B900A2E720005D1507005A
:1063680050BA800043BA800060150700010032006F
:106378004A37EC0050BA80006F15070051BA880000
:10638800000006001600FA00881F780001BA800095
:1063980010BA8000808F50000E00320001BA8000D1
:1063A8007609B900A0BB20005415070001BA88007F
:1063B80000BA80006015070001BA8800F687470018
:1063C8007684570054150700208020002B00070012
:1063D8008807780021BA800030BA8000808F50008A
:1063E8000E00320021BA80007609B900A0D1200041
:1063F8004215070021BA880020BA80004E15070010
:1064080021BA8800F68747007684570042150700AE
:10641800208E2000190007008807780041BA800004
:1064280050BA8000808F50000E00320041BA8000C0
:106438007609B900A0E720003015070041BA8800A6
:1064480040BA80003C15070041BA8800F68747002B
:1064580076845700301507000000EB00070007009E
:10646800880778004F0478000080FA0000000600D2
:10647800B6B2020000000000000006005A01FA004F
:10648800889FBE008A9FBE0080047800508D290036
:106498002B010900305F7800CE12B1002EB19700B1
:1064A8000080EB008080EB0002004000E0804800A4
:1064B80072042000820F5000E08F5800E0073E0071
:1064C8000060010047003700DD073700DC073700B0
:1064D8006E003700470037003001370049013700A8
:1064E80067013700A3003700D6003700FF003700E8
:1064F80099003700D2073700D10737007A003700F4
:106508008700370020023700D1013700E801370043
:10651800040237006101370081013700A602370005
:10652800BE023700DB023700F80237008403370069
:106538001803370020033700410337004F033700A3
:106548007003370084033700C7033700B5033700EB
:106558000304370008043700330437004C043700BD
:1065680055043700800437009A043700A804370020
:1065780066053700C9043700DD04370041023700DB
:106588007F023700FE043700C7033700E6033700F1
:10659800D70337000C0537001105370016053700FB
:1065A8005D05370081053700A5053700C9053700A7
:1065B800D3053700160537002A0537003E05370092
:1065C8001D063700220637003D06370058063700FB
:1065D8001907370099063700380737004E06370085
:1065E800B9063700BEB0970078804400D40707008A
:1065F80093073700495090000068A3000800320054
:1066080009007800D41207000004E00004003A00F2
:10661800BEB0970010A02900C907070088073700F7
:10662800494091000038A30004003A00BEB097002A
:1066380060A22900C207070081073700495090006F
:106648000018A30004003200BEB0970060A529001E
:10665800BB0707007A073700C949E2000400320087
:10666800BEB0970080A52900B5070700740737005A
:106678000900780006B3020000000000BEB09700D1
:1066880060A52900AE0707006D073700F6874700A9
:10669800768457007C0057000A000900301C7800F7
:1066A8006801B1006001B1000900780068070700BF
:1066B800880778000004E00061073200292990006B
:1066C800B92990008301D1000281D3000900780024
:1066D800FAB2020000000000BEB09700D0A829005E
:1066E80097070700560737000F0EB00000F22F007B
:1066F800008447006F000900391C7800080EB100BB
:10670800090EB1000E007800A90807008807780074
:10671800BEB097000E0078008907070048073700C9
:106728000F0EB00000F22F00008447006F00090030
:10673800391C7800080EB100090EB1000E0078006F
:10674800A007070088077800BEB097000E00780001
:106758007B0707003A07370009007800B6B2020045
:1067680000000000BEB09700F0A8290074070700D9
:1067780033073700F6874700768457007C005700B8
:106788000A000900301C78006801B1006001B100FE
:10679800090078002E070700880778000004E00049
:1067A8002707320061C0B30078005700FA100700CD
:1067B8000002BE0029289000B9289000800F5200DE
:1067C800818F5A0004003600BEB0970060A22900ED
:1067D8005B0707001A07370019009000A90090000E
:1067E800800F5200818F5A001200320049409100F8
:1067F8000048A3000B003200494091000038A30074
:1068080008003A0029299000B92990000401510094
:106818008581590009007800FAB2020000000000E2
:10682800040037000401BE0009007800FAB2020033
:1068380000000000BEB09700D0A82900400707005C
:10684800FF063700F6874700768457007C0057001C
:106858000A000900301C78006801B1006001B1002D
:1068680009007800FA060700880778000004E000AD
:10687800F306320019009000A9009000E00F5000C4
:10688800E08F5800EE063200494091000048A3000E
:106898000B003200494091000038A30008003A007C
:1068A80019019000A901900061014100E0814900AF
:1068B80009007800FAB20200000000000700370063
:1068C80019019000A901900061015100E08159006F
:1068D80009007800FAB2020000000000BEB097007C
:1068E800D0A8290016070700D5063700F687470005
:1068F800768457007C0057000A000900301C780095
:106908006801B1006001B10009007800D0060700F5
:10691800880778000004E000C906320019019000D9
:10692800A901900029289000B9289000800F5100F3
:10693800818F5900C2063100494091000048A300E8
:106948000B003200494091000038A30008003A00CB
:1069580019019000A901900061015100E0815900DE
:1069680009007800FAB202000000000007003700B2
:1069780019019000A901900061014100E0814900DE
:1069880009007800FAB2020000000000BEB09700CB
:10699800D0A82900EA060700A9063700F6874700AD
:1069A800768457007C0057000A000900301C7800E4
:1069B8006801B1006001B10009007800A406070071
:1069C800880778000004E0009D06320049409100E5
:1069D8000048A3000300320049409100E8406000ED
:1069E8000100320011C0B300090078002EB3020084
:1069F80000000000BEB09700D0A82900D00607000C
:106A08008F063700F6874700768457007C005700CA
:106A18000A000900301C78006801B1006001B1006B
:106A2800090078008A060700880778000004E0005B
:106A380083063200494091000048A3000800320054
:106A4800494091000038A30005003A0011C0B30086
:106A5800090078002EB3020000000000040037008F
:106A68008040EB00090078002EB30200000000000F
:106A7800BEB09700D0A82900B106070070063700FD
:106A8800090078005CB3020000000000BEB0970067
:106A980060A92900AA060700690637008EE8970052
:106AA80000C2B30080CF500004003C00BEB0970085
:106AB80060A22900A2060700610637000EF89700B9
:106AC8000004E00004003200BEB09700E0A92900ED
:106AD8009B0607005A06370078804400F8005700E4
:106AE8001C0A0200000000000F0EB00000F22F0088
:106AF800008447006F000900391C7800080EB100B7
:106B0800090EB1007AC00200000000008807780072
:106B1800BEB0970010AC2900890607004806370068
:106B28000EE89700F1CBB30001404000F94F500048
:106B380004003600BEB0970060A229008006070056
:106B48003F0637001EE89700F1CBB3000140400034
:106B5800F94F500004003600BEB0970060A229002B
:106B6800770607003606370069D891005ADB02001D
:106B7800000000000EEA9700E45498001EE8970011
:106B8800F0549800E9D8910020C3B30080CF50009A
:106B980008003A000041EB00C1478000A0A525008D
:106BA800808F50000100320012C0B300024078000C
:106BB800AEFD07000F0EB00000F22F000084470062
:106BC8006F000900391C7800080EB100090EB100E9
:106BD8007AC00200000000008807780009007800E9
:106BE800FDFC0700494091000038A3000C0032006A
:106BF80029289000B92890008100D1000080D30096
:106C0800E0049800F1049800090078008711070053
:106C18000900780006B302000000000005003700F4
:106C28006000B80090049800A1049800B00498008F
:106C3800C104980069D8910068DB020000000000D8
:106C4800BEB0970010AC29003D060700FC053700D0
:106C58008EE89700F0CBB30000C04000E44F50002E
:106C680004003600BEB0970060A229003406070071
:106C7800F305370081C498000F0EB00000F22F0012
:106C8800008447006F000900391C7800080EB10025
:106C9800090EB1007AC002000000000088077800E1
:106CA800BEB0970010AC290025060700E4053700A0
:106CB8008EE8970010C3B30080CF500009003A0057
:106CC800495090000048A30004003A00BEB0970065
:106CD80050AC29001A060700D905370010C0B300C8
:106CE800010037000040EB00A0D498000F0EB00060
:106CF80000F22F00008447006F000900391C78005B
:106D0800080EB100090EB1007AC0020000000000B0
:106D180088077800BEB0970010AC29000806070065
:106D2800C70537008EE8970010C3B30080CF500026
:106D380004003A00591090000080A000D014980078
:106D480003003700591090000080A100D01498006B
:106D58000F0EB00000F22F00008447006F000900FA
:106D6800391C7800080EB100090EB1007AC0020083
:106D78000000000088077800BEB0970010AC29001A
:106D8800EF050700AE0537000EE89700F1CBB3001A
:106D980001404000E44F500004003600BEB09700A8
:106DA80060A22900E6050700A50537001EEC97003C
:106DB80000C3B300804F54000D00320065405000FE
:106DC800804F54000A00320066404000804F540053
:106DD8000700320064405000804F54000400320025
:106DE800BEB0970060A22900D505070094053700BA
:106DF80041C0B30076005700670F07008000780095
:106E0800F0702200808F500004003400BEB097005C
:106E180060A22900CA05070089053700D0C2B3005F
:106E2800804F54000300320064404000804F5400FB
:106E380001003A008100EA000EE897000000FB001C
:106E4800000040000900400051909F000F0EB00064
:106E580000F22F00008447006F000900391C7800F9
:106E6800080EB100090EB1007AC00200000000004F
:106E780088077800BEB0970010AC2900B00507005D
:106E88006F0537000EE89700F1CBB30001404000D2
:106E9800E44F500004003600BEB0970060A22900FD
:106EA800A7050700660537001EEC970000C3B3006E
:106EB800804F54000D00320065405000804F540050
:106EC8000A00320066404000804F5400070032003C
:106ED80064405000804F540004003200BEB0970058
:106EE80060A22900960507005505370061C0B30068
:106EF80076005700280F070080007800F0FF270071
:106F0800808F500004003A00BEB0970060A22900AC
:106F18008B0507004A053700D0C2B300804F5400E4
:106F28000300320064404000804F540001003A00E2
:106F38008100EA000EE897000000FB000000400016
:106F48000900400021989F000F0EB00000F22F00AA
:106F5800008447006F000900391C7800080EB10052
:106F6800090EB1007AC0020000000000880778000E
:106F7800BEB0970010AC2900710507003005370036
:106F88000F0EB00000F22F00008447006F000900C8
:106F9800391C7800080EB100090EB1000E00780007
:106FA8008B0A070088077800BEB097000E007800AB
:106FB80063050700220537008EE8970010C3B30069
:106FC80080CF500004003A00494091000004A0001E
:106FD800C044990003003700494091000004A10013
:106FE800C04499000F0EB00000F22F000084470043
:106FF8006F000900391C7800080EB100090EB100B5
:107008007AC002000000000088077800BEB0970030
:1070180010AC29004A050700090537007804570015
:1070280008007800540B0200000000008040E900CE
:1070380008007800D80E070080007800F00F2000C4
:10704800808F500004003400BEB0970060A2290071
:107058003B050700FA043700E1F498000F0EB00072
:1070680000F22F00008447006F000900391C7800E7
:10707800080EB100090EB1007AC00200000000003D
:1070880088077800BEB0970010AC29002C050700CF
:10709800EB04370031C0B30078005700BE0E07007C
:1070A8008000780040062000808F500004003600E1
:1070B800BEB0970060A2290021050700E004370050
:1070C8008000FD002BE8B7000BE9B7008000FD0049
:1070D8000F0EB00000F22F0000844700218020002E
:1070E8006F000900311C7800080EB1007AC0020058
:1070F800000000008807780066FC0700BEB0970013
:1071080010AC29000E050700CD04370061C0B3009C
:1071180078005700A00E07000005BE004940910006
:107128000038A30004003200BEB0970060A2290016
:1071380003050700C204370029289000B9289000E9
:10714800800F5500818F5D0004003600BEB09700A7
:1071580060A22900FA040700B904370069D8910031
:107168005ADB0200000000009A049800AB04980063
:10717800BA049800CB04980009007800C2C1020044
:107188000000000069D8910068DB020000000000E0
:10719800AB0437000900780062C20200000000005A
:1071A800090078008CFB0700BEB0970010AC2900DE
:1071B800E3040700A20437008EE8970000CDB3006F
:1071C80000C140001EE897000000FB0001FD2F00F1
:1071D80001004000E10F400015003400E14F51006C
:1071E8000F003E00F8A520000200FB004400DD006F
:1071F80008004000F70057001C0A020000000000C9
:1072080008007800540B0200000000007FEAB70075
:10721800BEB0970010AC2900C904070088043700E5
:10722800BEB0970060A22900C50407008404370097
:10723800BEB0970060A22900C1040700800437008F
:107248008EE89700F0CBB30000C04000E44F500038
:1072580006003E000100780080EAB700BEB0970043
:1072680010AC2900B604070075043700BEB09700BB
:1072780060A22900B2040700710437008EE8970065
:1072880000CDB30000C140001EE897000000FB00DD
:1072980001FD2F0001004000E10F400015003400FF
:1072A800E34F51000F003E0018A820000200FB0029
:1072B8004400DD0008004000F70057001C0A0200E7
:1072C8000000000008007800540B020000000000D5
:1072D800C1EAB700BEB0970010AC290098040700B7
:1072E80057043700BEB0970060A229009404070035
:1072F80053043700BEB0970060A22900900407002D
:107308004F0437008EE89700F0CCB30000C040006F
:10731800E34F500006003E0001007800C2EAB700C3
:10732800BEB0970010AC290085040700440437005C
:10733800BEB0970060A2290081040700400437000E
:107348000E0078002D070700BEB097000E007800E9
:107358007B0407003A043700404BE2002D0032005E
:107368007F4AE20002003200804AE20004003A004C
:10737800BEB09700D0AF2900710407003004370071
:1073880001A820009140780010C4B30080CF5000BD
:1073980006003200C14AE20004003A00BEB097007D
:1073A800D0AF2900660407002504370001A8200093
:1073B8009140780040C4B30080CF500005003200EF
:1073C80001A82000914078000040E80080CF5000DC
:1073D80006003A00804AE20004003A00BEB0970076
:1073E800D0AF2900560407001504370052AC20001E
:1073F80074B32900050009003459780010C0B3009F
:1074080041EBB700BEB0970010AC29004C04070050
:107418000B043700BEB09700D0B32900480407001A
:107428000704370010C0B30044EBB700404BE2003C
:107438000900320051AC200092B62900080009006A
:10744800B258780041EBB700BEB0970010AC2900E5
:107458003B040700FA033700BEB09700D0B32900F9
:1074680037040700F6033700404BE2000A003200F9
:1074780054AC200020B7290005000900305A7800D4
:1074880010C0B30041EBB700BEB0970010AC2900A4
:107498002B040700EA033700BEB09700D0B32900D9
:1074A80027040700E6033700B6A802000000000022
:1074B8000000E0000A00320051AC200082B7290029
:1074C80004000900B258780010C0B30041EBB700BF
:1074D800BEB0970010AC290019040700D803370084
:1074E800BEB09700D0B7290015040700D4033700B1
:1074F800B6A80200000000000000E000060032000C
:107508000E00780027060700BEB097000E0078002E
:107518000B040700CA033700BEB09700D0B7290094
:1075280007040700C6033700B6A8020000000000E1
:107538000000E0000600320010C0B30043EBB700C3
:10754800BEB0970010AC2900FD030700BC0337004C
:10755800BEB09700D0B72900F9030700B803370079
:107568000E007800B0070700BEB097000E00780044
:10757800F3030700B20337000EE897000000FB0092
:10758800F1FC2F0001044000E30F540022003E00EC
:10759800C01220000E0040001EEA97000448780040
:1075A800AEE89700516F9A003EE99700626F9A0023
:1075B80004142000841F470011BA2900811F780095
:1075C8006E0B0200000000008E209100E487570037
:1075D800F00F2000808F50000B003E00C09C200060
:1075E8000174780000C0EB00D4E9B700D5E9B70012
:1075F800D6E9B700D769EF00BEB0970010AC2900F4
:10760800CF0307008E033700BEB0970060A22900A1
:10761800CB0307008A033700BEB0970060A2290099
:10762800C7030700860337000EE897000000FB0039
:10763800F1FC2F0081004000E38F500010003E0055
:10764800C81220000E044400C05A2100614078008E
:107658000080FB00801F780012BA2900821F780082
:10766800080078004C0D020000000000BEB0970032
:1076780008007800B2030700E4875700700337005A
:10768800BEB0970060A22900AD0307006C03370065
:107698000EE89700E14F500002003A00D8E9B70021
:1076A80001003700D869EF00BEB0970010AC290080
:1076B800A3030700620337000EE897000000FB00F1
:1076C800F1FC2F0001044000E30F540022003E00AB
:1076D800C01220000E0040001EEA970004487800FF
:1076E800AEE89700516F9A003EE99700626F9A00E2
:1076F80004142000841F470011BA2900811F780054
:107708006E0B0200000000008E209100E4875700F5
:10771800F00F2000808F50000B003E00009D2000DD
:107728000174780000C0EB00D4E9B700D5E9B700D0
:10773800D6E9B700D769EF00BEB0970010AC2900B2
:107748007F0307003E033700BEB0970060A2290000
:107758007B0307003A033700BEB0970060A22900F8
:1077680077030700360337000EE897000000FB0098
:10777800F1FC2F0001004000E30F500011003E0013
:10778800C81220000E044400E4004000C05A210042
:10779800614078000080FB00801F780012BA290041
:1077A800821F7800080078004C0D020000000000DD
:1077B800BEB097000800780061030700E48757000F
:1077C8001F033700BEB0970060A229005C030700C2
:1077D8001B033700C81220000E044400D8C9BF009C
:1077E8000080FB00801F780014BA2900841F7800ED
:1077F800080078004C0D020000000000BEB09700A1
:10780800080078004E030700E48757000C03370090
:10781800A6EC0200000000000000E0001B0032009F
:10782800BEB0970010AC2900450307009001200066
:1078380068EF0200000000000F0EB00009F22F00F0
:1078480009844700208020006F000900301C780060
:10785800080EB1007AC00200000000008807780016
:107868000F0EB00009844700218E20006F00090028
:10787800311C7800080EB1007AC002000000000038
:107888000000FE0088077800ED023700BEB09700C0
:1078980060A229002A030700E90237008EE8970052
:1078A800E1C06000C408DD00494091000044A10027
:1078B80001407000C04499000F0EB00000F22F0084
:1078C800008447006F000900391C7800080EB100D9
:1078D800090EB1007AC00200000000008807780095
:1078E800BEB0970010AC290015030700D40237007A
:1078F80061C0B30078005700A70C07000001BE0064
:10790800494091000038A30007003A00C22C9800B3
:10791800D32C980049289000D9289000A02C9800D2
:10792800B12C98000800370011C0B3000900780096
:107938004CDE02000000000029289000B9289000C1
:10794800C02C9800D12C98000F0EB00000F22F0028
:10795800008447006F000900391C7800080EB10048
:10796800090EB1007AC00200000000008807780004
:10797800BEB0970010AC2900F1020700B002370032
:1079880061C0B30078005700830C0700A03498004A
:107998000F0EB00000F22F00008447006F000900AE
:1079A800391C7800080EB100090EB1007AC0020037
:1079B8000000000088077800BEB0970010AC2900CE
:1079C800DF0207009E0237000E007800ED0807006E
:1079D800BEB097000E007800D90207009802370061
:1079E8000E007800E0090700BEB097000E0078008E
:1079F800D3020700920237000E007800EF0A070052
:107A0800BEB097000E007800CD0207008C02370048
:107A1800A11420008E8040007800570036BB020079
:107A2800000000000000E0000A0032005E20910023
:107A3800EE2091005AEC0200000000000000E00077
:107A480004003200BEB0970010AC2900BC02070049
:107A58007B023700BEB0970060A22900B802070079
:107A680077023700411420008E80400078005700CC
:107A780036BB0200000000000000E0000A003200EF
:107A88002E209100BE20910078EC0200000000003A
:107A98000000E00004003200BEB0970010AC2900DE
:107AA800A702070066023700BEB0970060A229004F
:107AB800A302070062023700011320008E804000F5
:107AC8007800570036BB0200000000000000E0000C
:107AD8000A0032000E1891009E1891008EEC0200E8
:107AE800000000000000E00004003200BEB0970073
:107AF80010AC29009202070051023700BEB097006F
:107B080060A229008E0207004D02370016ED020020
:107B1800000000004A023700411320008E80400018
:107B28007800570036BB0200000000000000E000AB
:107B38001A0032002E189100BE1891006EEC020057
:107B4800000000000000E000140032002E18910030
:107B580001B320009140780030EBB7004800DE0008
:107B680011B320009140780031EBB7003E18910026
:107B780021B320009140780032EBB7004800DE00C6
:107B880031B320009140780033EBB700BEB09700C6
:107B980010AC29006A02070029023700BEB097001E
:107BA80060A2290066020700250237008113200021
:107BB8008E8040007800570036BB020000000000AD
:107BC8000000E0001A0032004E189100DE18910003
:107BD8008CEC0200000000000000E00014003200FD
:107BE8004E18910041B320009140780034EBB70063
:107BF8004800DE0051B320009140780035EBB70013
:107C08005E18910061B320009140780036EBB70010
:107C18004800DE0071B320009140780037EBB700D0
:107C2800BEB0970010AC29004502070004023700D7
:107C3800BEB0970060A22900410207000002370089
:107C4800C11320008E8040007800570036BB020028
:107C5800000000000000E0001A0032006E189100D9
:107C6800FE189100A2EC0200000000000000E000F5
:107C7800140032006E18910081B320009140780002
:107C880038EBB7004800DE0091B32000914078003F
:107C980039EBB7007E189100A1B32000914078001D
:107CA8003AEBB7004800DE00B1B3200091407800FD
:107CB8003BEBB700BEB0970010AC290020020700CC
:107CC800DF013700BEB0970060A229001C02070040
:107CD800DB0137008040EB000EE89700E14F5000D1
:107CE80001003A0080407800010078003CEBB700C2
:107CF800BEB0970010AC290011020700D001370070
:107D0800454BE2004800320003B32000934178005D
:107D18008381FB0012B32000124178004811DD0076
:107D28000300710023B32000934178008381FB0096
:107D380032B32000124178004811DD008300710041
:107D48006EEC0200000000000000E00004003A00B1
:107D5800BEB09700D0AF2900F9010700B80137007D
:107D680043B32000934178008381FB0052B3200085
:107D7800124178004811DD000300710063B3200050
:107D8800934178008381FB0072B320001241780090
:107D98004811DD00830071008CEC02000000000037
:107DA8000000E00004003A00BEB09700D0AF290000
:107DB800E3010700A201370083B320009341780054
:107DC8008381FB0092B32000124178004811DD0046
:107DD80003007100A3B32000934178008381FB0066
:107DE800B2B32000124178004811DD008300710011
:107DF8008CEC0200000000000000E00004003A00E3
:107E0800BEB09700D0AF2900CD0107008C01370024
:107E180010C0B30042EBB700BEB0970010AC290009
:107E2800C701070086013700BEB09700D0B7290008
:107E3800C3010700820137000E007800A206070080
:107E4800BEB097000E007800BD0107007C01370026
:107E58000000EB000027990001142000811F470053
:107E680042BA2900821F7800780057006E0B020082
:107E780000000000E4875700E10F500002003A00BC
:107E88000E229100544E88000F0EB00000F22F0011
:107E980000844700208020006F000900301C780013
:107EA800080EB1007AC002000000000088077800C0
:107EB800BEB0970010AC2900A1010700600137008F
:107EC8008EE8970000C2B30080CF500004003C0049
:107ED800BEB0970060A22900990107005801370039
:107EE8003EE897000004E00004003200BEB09700AE
:107EF800E0A929009201070051013700F800570056
:107F0800509C20001C0A020000000000BEB0970030
:107F180010AC29008A0107000E007800B905070097
:107F2800BEB097000E0078008501070044013700B5
:107F38008EE8970000CDB30080C44000715D8000DA
:107F480010902800808F500004003A00BEB09700BF
:107F580070BA29007A010700390137001EE8970036
:107F68000000FB0001FD2F0001004000E10F400070
:107F78002E003400E3CF540028003E00A81420004F
:107F88000E044400F7005700080078001C0A02009D
:107F980000000000401420000E004000018D290060
:107FA80004000900315878005000B1000900FB00B6
:107FB8004300DD00E1B5200081044000AA1520003F
:107FC8000E0545001841780062C79A0018429000D3
:107FD80074C79A000001EB008000EB0040142000F9
:107FE8000E0040009C0C020000000000805C78003D
:107FF8000884E8008A0F5400F2FF3A0010A8200015
:10800800540B020000000000C1EAB700BEB09700A0
:1080180010AC29004A01070009013700BEB09700DB
:1080280060A229004601070005013700BEB097008D
:1080380060A229004201070001013700715D80003C
:1080480010902800808F500004003A00BEB09700BE
:1080580070BA29003A010700F90037006000B8003B
:10806800002799001127990000142000801F47005D
:1080780051BC2900811F7800780057006E0B020060
:1080880000000000E4875700E10F50000A003A00A2
:108098000E2091009E2091006011B80064B5200068
:1080A800009ABE000292BE00BEB0970010AC290034
:1080B80023010700E2003700BEB0970060A2290044
:1080C8001F010700DE003700985D8000A95D800071
:1080D800D3050700800F5400818F5C0004003A002C
:1080E800BEB0970070BA290015010700D400370008
:1080F800715D800010902800808F500013003200BE
:1081080064B820003400BE002401BE00F40F2D0026
:1081180075692A00F6FF2F00F7FF2F0000004200C4
:1081280081804A0002014B0083814B00E44F260006
:10813800D5DC21006033B8000400E1000588E100C7
:108148000690E1000798E10004003E00BEB09700E9
:1081580070BA2900FA000700B90037006000B800BB
:10816800002799001127990000142000801F47005C
:1081780051BC2900811F7800780057006E0B02005F
:1081880000000000E4875700E10F500026003A0085
:1081980068B520000E2091009E2091006011B80063
:1081A800009CBE000294BE007E6BEF00E0C7B300E7
:1081B8007FEBB700229C2000124178000201FB00EF
:1081C800400620000091B900C3C9BF000000FB00B1
:1081D8006A00B90000014100C4C9BF000000FB00EB
:1081E8000001410000B32E0000014100025C88003C
:1081F800000420000100200054E1020000000000FB
:1082080001032000080078007AE102000000000065
:1082180098E1020000000000BEB0970010AC2900F1
:10822800C700070086003700BEB0970060A229008B
:10823800C300070082003700715D8000109028009D
:10824800808F500004003A00BEB0970070BA290031
:10825800BB0007007A0037006000B80000279900CB
:108268001127990002142000821F470054BC2900DE
:10827800841F7800780057006E0B02000000000091
:10828800E4875700E10F500008003A000E209100E3
:108298009E209100105C8800215C8800BEB0970089
:1082A80010AC2900A600070065003700BEB0970093
:1082B80060A22900A200070061003700715D8000FC
:1082C80010902800808F500004003A00BEB097003C
:1082D80070BA29009A0007005900370064B52000D9
:1082E8003400BE002401BE0004102D0075692A0068
:1082F800F6FF2F00F7FF2F000000420081804A00A0
:1083080002014B0083814B0004A02C00A5B9230077
:108318006033B8000400E1000588E1000690E10040
:108328000798E10004003600BEB0970060A229005B
:1083380083000700420037006022B8006033B800AD
:10834800E8B52000E9B72000384078000080FB003D
:108358000100200002002000030020000402400069
:10836800858248000603490087834900888F5400A6
:10837800F5FF3A00E00F5200E08F5A00E00F5B0073
:10838800E08F5B0004003A00BEB0970060A22900AD
:108398006B0007002A003700185C8000295C800009
:1083A8001F050700800F5400818F5C000400320015
:1083B800BEB0970060A229006100070020003700C6
:1083C80010C0B3007EEBB70090C8B3007FEBB700D6
:1083D800229C2000124178000201FB004006200088
:1083E8000091B900C3C9BF000000FB006A00B900D2
:1083F80000014100C4C9BF000000FB0000014100AA
:1084080000B32E0000014100025C88000004200037
:108418000100200054E102000000000001032000D8
:1084280060B520007AE102000000000098E1020037
:1084380000000000BEB0970010AC29004000070003
:108448004F05BE004F04BE000080FA000000060081
:108458000000FA00889FBE00000478009FB49700CF
:10846800405090000068A30009003200080078001E
:10847800390B07000004E00005003A008900780085
:1084880010A029002E0007000000EB00290037008B
:1084980008007800300B07000004E00003003200F9
:1084A800485090000068A30019003200484091002D
:1084B8000038A30003003200485090000028A300B1
:1084C80016003200C949E200050032008900780030
:1084D80080A529001A0007000000EB0015003700EE
:1084E800485090000068A3001100320048509000E6
:1084F8000004E0000E003D0018009000A800900065
:10850800C2122000820F5000E08F58000800360089
:10851800485090000024A100405498008900780039
:1085280090BC2900060007000000EB00010037009E
:10853800100020004F04BE000080FA000000060072
:10854800E38F50001300320005003E00E18F500019
:1085580008003200E28F500019003A000900370085
:10856800E48F50000F003200E68F500014003A00EC
:108578001000370011C0B300EEE202000000000056
:108588000F00370011C0B300BAE402000000000079
:108598000B00370011C0B3008AD8020000000000A9
:1085A8000700370011C0B3005AAC020000000000F9
:1085B8000300370011C0B300528D02000000000014
:1085C800000006000C00FA00889FBE008A9FBE00CB
:1085D800800578008000EB0074805700011878004F
:1085E80001087800F0845700B0BF29000600090090
:1085F800B05C78007900B100A0C0B300C0EF9F0064
:1086080021C029000B0078001A0B020000000000AE
:10861800FA80570000F22F00008440008180E900B2
:108628000B0078001A0B020000000000F4805700CD
:108638000B0078001A0B02000000000091C029000E
:108648000B0078001A0B020000000000F80044003C
:108658000B0078001A0B020000000000F48057009D
:108668000B0078001A0B02000000000051C129001D
:108678000B0078001A0B0200000000002829900067
:10868800B8299000F069280011002000800F5100DF
:10869800818F590006003E0028289000B8289000D5
:1086A80053C0B30009017800F5080700050037003A
:1086B8005F289700EF28970063C0B30070815700C8
:1086C800EF080700708457006D0C07001A0B0200B2
:1086D80000000000F48057000B0078001A0B02001D
:1086E8000000000011C229000B0078001A0B0200DC
:1086F80000000000A0F12F00F480570080844000A3
:10870800F6804400220020000B007800280D0200AB
:1087180000000000F48057000B0078001A0B0200DC
:1087280000000000D1C229000B0078001A0B0200DB
:10873800000000007285570029D09000DC0B07006C
:108748001A0B020000000000F48057000B007800AC
:108758001A0B02000000000091C329000B007800EA
:108768001A0B02000000000069109000470C070077
:1087780074080700420C07001A0B020000000000F2
:10878800F48057000B0078001A0B0200000000006C
:1087980051C429000B0078001A0B020000000000E9
:1087A80079109000390C070066080700340C0700A0
:1087B8001A0B020000000000F48057000B0078003C
:1087C8001A0B02000000000011C529000B007800F8
:1087D8001A0B020000000000091890002B0C07007B
:1087E80058080700260C07001A0B020000000000BA
:1087F800F48057000B0078001A0B020000000000FC
:10880800D1C529000B0078001A0B020000000000F7
:10881800191890001D0C07004A080700180C0700DB
:108828001A0B020000000000F48057000B007800CB
:108838001A0B02000000000091C629000B00780006
:108848001A0B020000000000291890000F0C070006
:108858003C0807000A0C07001A0B02000000000081
:10886800F48057000B0078001A0B0200000000008B
:1088780051C729000B0078001A0B02000000000005
:108888000104200089804000120020000B007800BD
:10889800280D020000000000F48057000B0078004B
:1088A8001A0B02000000000011C829000B00780014
:1088B8001A0B02000000000049409100720B0700EB
:1088C8001A0B020000000000F48057000B0078002B
:1088D8001A0B020000000000D1C829000B00780024
:1088E8001A0B02000000000069F090000080FB00F5
:1088F80032C0B3008800780012080700E00B0700B8
:108908001A0B020000000000F48057000B007800EA
:108918001A0B02000000000091C929000B00780022
:108928001A0B020000000000196890000080FB008C
:108938000100200033C0B300080178005008070088
:10894800CF0B07001A0B020000000000F48057004C
:108958000B0078001A0B02000000000051CA290021
:108968000B0078001A0B020000000000591090005C
:108978004800DE00440B07001A0B0200000000004C
:10898800F48057000B0078001A0B0200000000006A
:1089980011CB29000B0078001A0B02000000000020
:1089A8004F05BE004F04BE000080FA00000006001C
:1089B8001000FA00889FBE008A9FBE0080057800DC
:1089C800A0C0B30080EF9F000040EB0090EF9F0035
:1089D800F6845700B0CB290005000900B05C780088
:1089E8006900B1007080570051CB290005000900CB
:1089F800315878006000B1000000EB00B0BF9F0064
:108A080011CC29000B0078001A0B020000000000AE
:108A18007E84570000F22F00000544008880E9009A
:108A28000B0078001A0B020000000000F8805700C5
:108A38000B0078001A0B02000000000081CC29000E
:108A48000B0078001A0B0200000000004870960026
:108A58000048A300080032001A0078008900780056
:108A680095070700890078000B0078001A0B0200B0
:108A780000000000090037000B007800540B0200CA
:108A8800000000000B004000E1C4B300015878006A
:108A980081C0E800015878000048EB00F8805700D2
:108AA8000B0078001A0B02000000000041CD2900DD
:108AB8000B0078001A0B0200000000007E825700AD
:108AC800750B07000A003200414091000038A300EE
:108AD80007003A0021299000B1299000141097004E
:108AE800A41097000002510081825900020037004B
:108AF8002F029700BF0297006C0B070005003E008D
:108B080053C0B300708157000400BE00DC070700A3
:108B18000400370063C0B300708157000400BE0032
:108B2800D7070700F08057000B0078001A0B0200E7
:108B380000000000F88057000B0078001A0B0200B4
:108B48000000000001CE29000B0078001A0B02007B
:108B5800000000007E8257004F0B07000A00320019
:108B6800414091000038A30007003A0021299000F5
:108B7800B129900034109700C410970000025100EA
:108B880081825900020037004F029700DF029700E8
:108B9800460B070005003E0053C0B3007081570024
:108BA8000400BE00B60707000400370063C0B30026
:108BB800708157000400BE00B1070700F08057001D
:108BC8000B0078001A0B020000000000F880570024
:108BD8000B0078001A0B020000000000C1CE29002B
:108BE8000B0078001A0B020000000000FE845700FA
:108BF8000AF22F000A85440049709600614060001F
:108C08006A845700010B07001A0B020000000000DD
:108C1800F88057000B0078001A0B020000000000D3
:108C280081CF29000B0078001A0B02000000000019
:108C3800497096000000D100A20A07001A0B020032
:108C480000000000F88057000B0078001A0B0200A3
:108C58000000000041D029000B0078001A0B020028
:108C680000000000497096004200DE00950A0700E7
:108C78001A0B020000000000F88057000B00780073
:108C88001A0B02000000000001D129000B00780037
:108C98001A0B020000000000497096004600DE0032
:108CA800880A07001A0B020000000000F88057002D
:108CB8000B0078001A0B020000000000C1D1290047
:108CC8000B0078001A0B02000000000049709600A3
:108CD8006F0A07001A0B020000000000F880570016
:108CE8000B0078001A0B02000000000081D2290056
:108CF8000B0078001A0B0200000000004970960073
:108D08004500DE006F0A07001A0B02000000000091
:108D1800F88057000B0078001A0B020000000000D2
:108D280041D329000B0078001A0B02000000000054
:108D3800497096004300DE00620A07001A0B020021
:108D480000000000F88057000B0078001A0B0200A2
:108D58000000000001D429000B0078001A0B020063
:108D6800000000004A409100490A07001A0B02005F
:108D780000000000F88057000B0078001A0B020072
:108D88000000000011CB29000B0078001A0B02002C
:108D9800000000004F05BE004F04BE000080FA002E
:108DA800000006004200FA00889FBE000004780018
:108DB800A0C0B300A07F9F000040EB00B07F9F00E1
:108DC800C1D42900080078001A0B02000000000036
:108DD800A1FB2F008F804000080078001A0B0200CA
:108DE80000000000D6CABF00C1FB2F0081844700E5
:108DF8000080FB00801F780060D52900801F780064
:108E0800090078004C0D0200000000000800BE00B8
:108E18001A0B02000000000061FB2F008F80400049
:108E2800080078001A0B020000000000D8CABF0032
:108E38000080FB00801F780041D62900811F780040
:108E4800090078004C0D0200000000000800BE0078
:108E58001A0B02000000000021FB2F008F80400049
:108E6800080078001A0B020000000000D7CABF00F3
:108E78000080FB00801F780020D72900801F780021
:108E8800090078004C0D0200000000000800BE0038
:108E98001A0B020000000000E1FA2F008F8040004A
:108EA800080078001A0B02000000000001D8290011
:108EB800080078001A0B02000000000091AD2000A5
:108EC800080078001A0B020000000000E1FA2F00E9
:108ED8008F804000080078001A0B02000000000094
:108EE800F9CABF000080FB00801F7800C1D82900A4
:108EF800811F7800090078004C0D02000000000076
:108F08000800BE001A0B020000000000A1FA2F00A2
:108F18008F804000080078001A0B02000000000053
:108F2800FACABF000080FB00801F7800A0D9290082
:108F3800801F7800090078004C0D02000000000036
:108F48000800BE001A0B02000000000061FA2F00A2
:108F58008F804000080078001A0B02000000000013
:108F6800FBCABF000080FB00801F780081DA29005F
:108F7800811F7800090078004C0D020000000000F5
:108F88000800BE001A0B02000000000021FA2F00A2
:108F98008F804000080078001A0B020000000000D3
:108FA80043CBBF000080FB00801F780060DB2900F6
:108FB800801F7800090078004C0D020000000000B6
:108FC8000800BE001A0B020000000000E1F92F00A3
:108FD8008F804000080078001A0B02000000000093
:108FE8000D0A07001A0B020000000000FC8757005A
:108FF8004F04BE000080FA00000006002400FA00BA
:10900800889FBE008A9FBE0000057800A0C0B300FC
:10901800C0D79F000040EB00D0D79F0040FD2F0035
:109028000F0040008085E800800DEB0064044000DC
:1090380041DC29000F000900315C78000801B1000B
:10904800F88457006000B800808CBE007481570017
:109058000089BE00708157000099BE000089BE00DB
:10906800DAC9BF00804C7800E0C2B30090EF9F00DF
:10907800B19D200091407800A1EF9F00B0EF9F00C4
:10908800DCC9BF00C0EF9F0041DD29000A0078005D
:109098001A0B02000000000041FD2F008F804000E5
:1090A8000A0078001A0B020000000000D1DD290038
:1090B8000A0078001A0B020000000000D909070016
:1090C8001A0B02000000000041FD2F008F804000B5
:1090D8000A0078001A0B02000000000091DE290047
:1090E8000A0078001A0B020000000000C9C9BF007E
:1090F800CF0907001A0B02000000000041FD2F00F5
:109108008F8040000A0078001A0B0200000000005F
:1091180051DF29000A0078001A0B02000000000045
:10912800C35A2100C6090700D25A2100E4090700E2
:1091380003007100E35A2100C1090700F25A210017
:10914800C2090700B1070700B60907001A0B020099
:109158000000000041FD2F008F8040000A007800C9
:109168001A0B02000000000011E029000A00780034
:109178001A0B020000000000D8D5BF004600DE0030
:1091880061006000AA0907001A0B02000000000035
:1091980041FD2F008F8040000A0078001A0B020062
:1091A80000000000D1E029000A0078001A0B020034
:1091B800000000003FCBBF009D0907001A0B02000A
:1091C8000000000041FD2F008F8040000A00780059
:1091D8001A0B02000000000091E129000A00780043
:1091E8001A0B02000000000045CABF0090090700E2
:1091F8001A0B02000000000041FD2F008F80400084
:109208000A0078001A0B02000000000051E2290051
:109218000A0078001A0B020000000000890078009C
:109228000A0078001A0B02000000000041FD2F0020
:109238008F8040000A0078001A0B0200000000002E
:1092480011E329000A0078001A0B02000000000050
:1092580040CBBF00760907001A0B0200000000008F
:1092680041FD2F008F8040000A0078001A0B020091
:1092780000000000D1E329000A0078001A0B020060
:1092880000000000119E20000A0078001A0B02005E
:109298000000000041FD2F008F8040000A00780088
:1092A8001A0B02000000000091E429000A0078006F
:1092B8001A0B020000000000D39D2000600907007F
:1092C800E29D20007E09070003007100F39D200045
:1092D8005B090700029E20005C0907004B07070096
:1092E800500907001A0B02000000000041FD2F0082
:1092F8008F8040000A0078001A0B0200000000006E
:1093080051E529000A0078001A0B0200000000004D
:10931800024AE20003003A0010C4B300804D78000E
:109328001700370002CABF00E84F500003003A0098
:1093380020C4B300E0D79F001100370002CABF0065
:10934800E74F500003003A0030C4B300E0D79F0055
:109358000B00370002CABF00E14F500003003A007B
:1093680040C4B300E0D79F000500370002CABF0021
:10937800E24F500002003A0050C4B300E0D79F000B
:1093880060FD2F0000844700260907001A0B020021
:109398000000000041FD2F008F8040000A00780087
:1093A8001A0B02000000000011E629000A007800EC
:1093B8001A0B02000000000041FD2F008F804000C2
:1093C8000A0078001A0B020000000000D1E629000C
:1093D8000A0078001A0B02000000000044CABF000F
:1093E80001C3B300014C40000E0907001A0B02002C
:1093F8000000000041FD2F008F8040000A00780027
:109408001A0B02000000000011CB29000A007800A6
:109418001A0B0200000000004F05BE004F04BE00FA
:109428000080FA00000006004200FA00889FBE0093
:1094380000047800A0C0B300004F78000040EB00A3
:109448001047980091E72900080078001A0B0200DD
:1094580000000000010907001A0B020000000000CC
:10946800804D8000814680008E84E800801F78004F
:10947800811F780060E82900801F780009007800C3
:109488004C0D0200000000000800BE001A0B02008C
:1094980000000000F10807001A0B0200000000009D
:1094A800904D800091468000801F7800811F7800D1
:1094B800B0E92900801F7800090078004C0D0200EF
:1094C800000000000800BE001A0B020000000000A7
:1094D800E20807001A0B020000000000B5C9BF002F
:1094E800518D2000914078000080FB00801F78009B
:1094F8008180FB00811F780020EB2900801F780005
:10950800090078004C0D0200000000000800BE00B1
:109518001A0B020000000000D00807001A0B020016
:1095280000000000B8C9BF00818D2000914078007C
:109538000080FB00801F78008180FB00811F78007D
:1095480060EC2900801F7800090078004C0D0200AB
:10955800000000000800BE001A0B02000000000016
:10956800BE0807001A0B020000000000D9C8BF009F
:109578000080FB00801F780080ED2900801F7800A4
:10958800090078004C0D0200000000000800BE0031
:109598001A0B020000000000B00807001A0B0200B6
:1095A80000000000E0B98000F1B98000A2002000AE
:1095B80046080700809FBE0070EE2900801F7800D3
:1095C800090078004C0D020000000000E0FD2F00AB
:1095D800808747000800BE001A0B02000000000048
:1095E8009E0807001A0B0200000000008A08070006
:1095F8001A0B0200000000004F04BE000080FA00B1
:10960800000006004200FA00889FBE008A9FBE0044
:1096180080047800A0C0B300E0779F000040EB0012
:10962800F0779F0031EF2900090078001A0B02003B
:109638000000000061FB2F008F80400009007800C7
:109648001A0B02000000000080FB2F000084470076
:1096580061B820005101BE004100BE00809FBE00DD
:10966800829FBE00F2EF2900821F78000800780070
:109678004C0D020000000000160807001A0B02003B
:1096880000000000C1FA2F008F8040000900780018
:109698001A0B02000000000001F1290009007800FF
:1096A8001A0B020000000000E8B82000EA87570003
:1096B80083FB2F0003854700EBBA20003880FB00AE
:1096C800801F780080F12900801F78000A00780048
:1096D8004C0D020000000000010807001A0B0200F0
:1096E80000000000E4875700888F5500F3FF3A0018
:1096F80061FB2F008F804000090078001A0B0200E0
:1097080000000000AECBBF000080FB00801F780087
:10971800D1F12900811F78000A0078004C0D020061
:1097280000000000EE0707001A0B0200000000000E
:1097380021FB2F008F804000090078001A0B0200DF
:1097480000000000AFCBBF000080FB00801F780046
:10975800B2F22900821F78000A0078004C0D02003E
:1097680000000000DE0707001A0B020000000000DE
:10977800E1FA2F008F804000090078001A0B0200E0
:1097880000000000B00BF80053F32900831F780095
:109798000A0078004C0D020000000000D007070006
:1097A8001A0B020000000000A1FA2F008F80400071
:1097B800090078001A0B020000000000905D80008C
:1097C800A15D8000809FBE0021F42900811F7800E0
:1097D8000A0078004C0D020000000000C0070700D6
:1097E8001A0B02000000000041FA2F008F80400091
:1097F800090078001A0B02000000000011CB2900B4
:10980800090078001A0B020000000000F2875700D8
:109818004F05BE004F04BE000080FA00000006009D
:109828003600FA00D9D5BF00A0CF9F00DAD5BF0017
:10983800B0CF9F00B15D210091407800C1CF9F005B
:10984800C25D210012417800D2CF9F00DDD5BF0054
:10985800E0CF9F00E15D210091407800F1CF9F00AB
:1098680090C0B30080D79F0080C0B30090D79F00FE
:1098780030C0B300A0D79F0020C0B300B0D79F006E
:10988800C0D79F00D0D79F0070C0B300E0D79F001B
:109898000040EB00F0D79F00A2FC2F000F01410011
:1098A8006E0041000600090032187800E000B1009F
:1098B800E200B100710020000CEE02000000000080
:1098C8000080FA00000006004800FA00889FBE00E9
:1098D80000047800A0C0B300C0779F000040EB00F0
:1098E800D0779F00E1F42900080078001A0B0200E5
:1098F8000000000041FB2F008F8040000800780026
:109908001A0B02000000000060FB2F008084470053
:10991800CA09F800A1F52900811F7800090078001C
:109928004C0D0200000000000800BE001A0B0200E7
:109938000000000001FB2F008F8040000800780025
:109948001A0B020000000000EE845700800CEB00A8
:10995800B91478000000EB00B0BF9F00C5C9BF0074
:10996800804C7800E0C2B300B0F79F00619C2000F3
:1099780091407800C1F79F00D0F79F00C7C9BF008A
:10998800E0F79F0081F62900080078001A0B020012
:10999800000000000800BE001A0B020000000000D2
:1099A80001FB2F008F804000080078001A0B02008E
:1099B80000000000980707001A0B020000000000D2
:1099C800E48757004F04BE000080FA00000006003C
:1099D8000C00FA00889FBE008A9FBE000004780031
:1099E8000000EB00F4845700801C7800800C78009D
:1099F8007085570040F7290006000900305D78009F
:109A08007A00B100A0C0B300C0EF9F00B1F72900F1
:109A1800080078001A0B020000000000FA805700C6
:109A28000BF22F008B8540008180E9000800780048
:109A38001A0B020000000000F480570008007800AC
:109A48001A0B020000000000D1C2290008007800AB
:109A58001A0B0200000000002BD0900001C3B300D5
:109A6800814C40000800BE001A0B020000000000F4
:109A7800F4805700080078001A0B0200000000006C
:109A880051C72900080078001A0B020000000000E6
:109A9800010420008B80400012002000080078009C
:109AA800280D020000000000F4805700080078002C
:109AB8001A0B02000000000051CA290008007800B3
:109AC8001A0B0200000000005B1090004800DE0046
:109AD8006140600001C3B300814C40000800BE0033
:109AE8001A0B020000000000F480570008007800FC
:109AF8001A0B02000000000091C32900080078003A
:109B08001A0B0200000000006B109000F706070017
:109B18008C030700F80607001A0B0200000000007B
:109B2800F4805700080078001A0B020000000000BB
:109B380051C42900080078001A0B02000000000038
:109B48007B109000E90607007E030700EA0607007D
:109B58001A0B020000000000F4805700080078008B
:109B68001A0B02000000000011C529000800780047
:109B78001A0B0200000000000B189000DB0607001B
:109B880070030700DC0607001A0B02000000000043
:109B9800F4805700080078001A0B0200000000004B
:109BA800D1C52900080078001A0B02000000000047
:109BB8001B189000CD06070062030700CE060700B9
:109BC8001A0B020000000000F4805700080078001B
:109BD8001A0B02000000000091C629000800780056
:109BE8001A0B0200000000002B189000BF060700A7
:109BF80054030700C00607001A0B0200000000000B
:109C0800F4805700080078001A0B020000000000DA
:109C180051F82900080078001A0B02000000000023
:109C28003B189000B706070046030700B206070076
:109C38001A0B020000000000F480570008007800AA
:109C48001A0B02000000000011F929000800780032
:109C58001A0B0200000000004B189000A90607002C
:109C680038030700A40607001A0B020000000000D2
:109C7800F4805700080078001A0B0200000000006A
:109C8800D1F92900080078001A0B02000000000032
:109C98005B1890009B0607002A030700960607003A
:109CA8001A0B020000000000F4805700080078003A
:109CB8001A0B02000000000091FA29000800780041
:109CC8001A0B0200000000006B1890008D060700B8
:109CD8001C030700880607001A0B0200000000009A
:109CE800F4805700080078001A0B020000000000FA
:109CF80051FB2900080078001A0B02000000000040
:109D08007B1890007F0607000E0307007A060700FD
:109D18001A0B020000000000F480570008007800C9
:109D28001A0B02000000000011FC2900080078004E
:109D38001A0B0200000000002B30900001002000E8
:109D480053C0B3000A0178004D0307006A060700F4
:109D58001A0B020000000000F48057000800780089
:109D68001A0B020000000000AB0607001A0B0200E5
:109D7800000000004F05BE004F04BE000080FA003E
:109D8800000006005200FA00889FBE008A1F780073
:109D98005F06070010FE29003B000900B05C780050
:109DA800C903B100D1012A00080078001A0B02008B
:109DB80000000000A90607001A0B020000000000BE
:109DC800AFD5BF000080FB00801F7800AED5BF0074
:109DD8000080FB00801F7800ADD5BF000080FB002D
:109DE800801F7800ACD5BF000080FB00801F780082
:109DF80090022A00801F7800090078004C0D0200AC
:109E0800000000000800BE001A0B0200000000005D
:109E1800920607001A0B020000000000B3D5BF002D
:109E28000080FB00801F7800B2D5BF000080FB00D7
:109E3800801F7800B1D5BF000080FB00801F78002C
:109E4800B0D5BF000080FB00801F780000042A0006
:109E5800801F7800090078004C0D02000000000007
:109E68000800BE001A0B0200000000007B06070075
:109E78001A0B020000000000B7D5BF000080FB00ED
:109E8800801F7800B6D5BF000080FB00801F7800D7
:109E9800B5D5BF000080FB00801F7800B4D5BF0097
:109EA8000080FB00801F780070052A00801F780062
:109EB800090078004C0D0200000000000800BE00F8
:109EC8001A0B020000000000640607001A0B0200CB
:109ED80000000000BBD5BF000080FB00801F780099
:109EE800BAD5BF000080FB00801F7800B9D5BF003D
:109EF8000080FB00801F7800B8D5BF000080FB0001
:109F0800801F7800E0062A00801F7800090078008A
:109F18004C0D02000000000080FD2F0080874700E4
:109F28000800BE001A0B0200000000004B060700E4
:109F38001A0B020000000000BFD5BF000080FB0024
:109F4800801F7800BED5BF000080FB00801F78000E
:109F5800BDD5BF000080FB00801F7800BCD5BF00C6
:109F68000080FB00801F780050082A00801F7800BE
:109F7800090078004C0D0200000000000800BE0037
:109F88001A0B020000000000340607001A0B02003A
:109F980000000000C3D5BF000080FB00801F7800D0
:109FA800C2D5BF000080FB00801F7800C1D5BF006C
:109FB8000080FB00801F7800C0D5BF000080FB0038
:109FC800801F7800C0092A00801F780009007800E7
:109FD8004C0D0200000000000800BE001A0B020031
:109FE800000000001D0607001A0B02000000000018
:109FF800C7D5BF000080FB00801F7800C6D5BF0012
:10A008000080FB00801F7800C5D5BF000080FB00E2
:10A01800801F7800C4D5BF000080FB00801F780037
:10A02800300B2A00801F7800090078004C0D0200D0
:10A03800000000000800BE001A0B0200000000002B
:10A04800060607001A0B020000000000D8D5BF0062
:10A058004600DE00E11F6000A00C2A00801F780087
:10A06800090078004C0D020000000000E0FD2F0000
:10A07800808747000800BE001A0B0200000000009D
:10A08800F60507001A0B020000000000805C2100A2
:10A09800801F7800800D2A00801F78000900780052
:10A0A8004C0D0200000000000800BE001A0B020060
:10A0B80000000000E90507001A0B0200000000007C
:10A0C800EA0320000E054500D0FC29001300090012
:10A0D800305D78004A01B100D9D5BF000080FB008F
:10A0E800A15D210091407800C808DD0080807000E3
:10A0F800DBD5BF000080FB00C25D2100F005070032
:10A1080000017100DDD5BF000080FB00E35D210088
:10A1180085050700380507008A1F7800600E2A00A9
:10A12800801F7800090078004C0D02000000000034
:10A138000800BE001A0B020000000000C705070057
:10A148001A0B020000000000B30507001A0B0200FA
:10A1580000000000E88757004F0578004F04BE0054
:10A168000080FA00000006005200FA00889FBE0036
:10A178008A1F78006605070080102A003B00090046
:10A18800B05C7800C903B10041142A0008007800C7
:10A198001A0B020000000000B00507001A0B0200AD
:10A1A80000000000FFCABF00E1AF20009140780026
:10A1B800D2AF200012417800C3AF20005F0507002E
:10A1C800801F78008180FB00811F78000281FB00DE
:10A1D800821F78008381FB00831F780090022A0089
:10A1E800801F7800090078004C0D02000000000074
:10A1F8000800BE001A0B02000000000097050700C7
:10A208001A0B02000000000003CBBF0021B02000A1
:10A218009140780012B020001241780003B020006D
:10A2280046050700801F78008180FB00811F7800A9
:10A238000281FB00821F78008381FB00831F780066
:10A2480000042A00801F7800090078004C0D0200E5
:10A25800000000000800BE001A0B02000000000009
:10A268007E0507001A0B02000000000007CBBF00A4
:10A2780061B020009140780052B02000124178006F
:10A2880043B020002D050700801F78008180FB0067
:10A29800811F78000281FB00821F78008381FB0008
:10A2A800831F780070052A00801F78000900780055
:10A2B8004C0D0200000000000800BE001A0B02004E
:10A2C80000000000650507001A0B020000000000EE
:10A2D8000BCBBF00A1B020009140780092B02000C5
:10A2E8001241780083B0200014050700801F780011
:10A2F8008180FB00811F78000281FB00821F7800AB
:10A308008381FB00831F7800E0062A00801F780005
:10A31800090078004C0D02000000000080FD2F00AD
:10A32800808747000800BE001A0B020000000000EA
:10A338004A0507001A0B0200000000000FCBBF00FF
:10A34800E1B0200091407800D2B02000124178009E
:10A35800C3B02000F9040700801F78008180FB004B
:10A36800811F78000281FB00821F78008381FB0037
:10A37800831F780050082A00801F780009007800A1
:10A388004C0D0200000000000800BE001A0B02007D
:10A3980000000000310507001A0B02000000000051
:10A3A80013CBBF0021B120009140780012B12000EA
:10A3B8001241780003B12000E0040700801F7800F4
:10A3C8008180FB00811F78000281FB00821F7800DA
:10A3D8008381FB00831F7800C0092A00801F780052
:10A3E800090078004C0D0200000000000800BE00C3
:10A3F8001A0B020000000000180507001A0B0200E3
:10A408000000000017CBBF0061B120009140780028
:10A4180052B120001241780043B12000C704070060
:10A42800801F78008180FB00811F78000281FB007B
:10A43800821F78008381FB00831F7800300B2A007D
:10A44800801F7800090078004C0D02000000000011
:10A458000800BE001A0B020000000000FF040700FD
:10A468001A0B02000000000028CBBF004600DE00E7
:10A47800E11F6000A00C2A00801F78000900780006
:10A488004C0D020000000000E0FD2F00808747000F
:10A498000800BE001A0B020000000000EF040700CD
:10A4A8001A0B02000000000028CBBF004700DE00A6
:10A4B800E11F600010152A00801F7800090078004D
:10A4C8004C0D0200000000000800BE001A0B02003C
:10A4D80000000000E10407001A0B02000000000061
:10A4E80080B12000801F7800800D2A00801F78002E
:10A4F800090078004C0D0200000000000800BE00B2
:10A508001A0B020000000000D40407001A0B020016
:10A5180000000000EA0320000E054500400F2A0055
:10A5280013000900305D78004A01B10029CBBF0053
:10A538000080FB00A1B2200091407800C808DD002F
:10A54800808070002BCBBF000080FB00C2B22000CF
:10A55800DB040700000171002DCBBF000080FB0069
:10A56800E3B2200070040700230407008A1F780064
:10A57800600E2A00801F7800090078004C0D020048
:10A58800000000000800BE001A0B020000000000D6
:10A59800B20407001A0B0200000000009E04070026
:10A5A8001A0B020000000000EC8757004F057800E6
:10A5B8004F04BE000080FA00000006003E00FA00CA
:10A5C800889FBE008A1F780080047800000FEB0087
:10A5D800A0C0B300004F78000E84E800F0152A00F0
:10A5E8003B000900305C7800C803B100CFC9BF0048
:10A5F8000080FB00801F7800CEC9BF000080FB00F0
:10A60800801F7800CDC9BF000080FB00801F780044
:10A61800CCC9BF000080FB00801F7800B0192A0059
:10A62800801F7800080078004C0D02000000000030
:10A63800280407001A0B020000000000420407006B
:10A648001A0B020000000000D3C9BF000080FB0005
:10A65800801F7800D2C9BF000080FB00801F7800EF
:10A66800D1C9BF000080FB00801F7800D0C9BF009F
:10A678000080FB00801F7800401B2A00801F7800A4
:10A68800080078004C0D02000000000011040700CB
:10A698001A0B0200000000002B0407001A0B02002E
:10A6A80000000000D7C9BF000080FB00801F7800B1
:10A6B800D6C9BF000080FB00801F7800D5C9BF0045
:10A6C8000080FB00801F7800D4C9BF000080FB0019
:10A6D800801F7800F01C2A00801F7800080078008E
:10A6E8004C0D020000000000FA0307001A0B0200DC
:10A6F80000000000140407001A0B0200000000000C
:10A70800D8C9BF000080FB00801F7800801E2A0087
:10A71800801F7800080078004C0D0200000000003F
:10A72800EAFD2F008A874700EA0307001A0B020098
:10A7380000000000040407001A0B020000000000DB
:10A7480033CBBF0021B320009140780012B3200022
:10A758001241780003B32000F8030700801F780037
:10A768008180FB00811F78000281FB00821F780036
:10A778008381FB00831F7800A01F2A00801F7800B8
:10A78800080078004C0D020000000000D10307000B
:10A798001A0B020000000000EB0307001A0B02006E
:10A7A8000000000037CBBF0061B320009140780063
:10A7B80052B320001241780043B32000DF030700A2
:10A7C800801F78008180FB00811F78000281FB00D8
:10A7D800821F78008381FB00831F780040212A00B4
:10A7E800801F7800080078004C0D0200000000006F
:10A7F800B80307001A0B020000000000D20307008C
:10A808001A0B0200000000003BCBBF00A1B32000E0
:10A818009140780092B320001241780083B3200061
:10A82800C6030700801F78008180FB00811F780025
:10A838000281FB00821F78008381FB00831F780060
:10A8480000232A00801F7800080078004C0D0200C1
:10A85800000000009F0307001A0B02000000000020
:10A86800B90307001A0B0200000000003CCBBF0030
:10A878000080FB00801F7800A0242A00801F780039
:10A88800080078004C0D0200000000008A8747008D
:10A89800900307001A0B020000000000AA0307003B
:10A8A8001A0B0200000000004F0578004F04BE009C
:10A8B8000080FA00000006000002BE000000E00070
:10A8C80004003D00D0C2B300804878000402EA00CA
:10A8D80002003700B0C2B30080487800420620006A
:10A8E800110009000202D80001C3B30081414000F1
:10A8F800934298000280B90000005200A200200094
:10A90800801F7800110009000200D80000017800BB
:10A918004F00780001C3B30001424100A4429800EF
:10A92800E4C2B300B44298006A11B90002005000B2
:10A9380001404000C04298000040EB00D04298001F
:10A9480000000600889FBE000004BE000000E00072
:10A9580004003D000004EA00D0C2B300804878003B
:10A9680002003700B0C2B30080487800E34F5100BE
:10A978001200320005003C00E14F51000B0032008C
:10A98800E24F510007003A000A003700E54F510036
:10A998000C0032001400200023003500E64F51005F
:10A9A8000A00320011002000310037001100200099
:10A9B8002B003700140020001F003700140020006F
:10A9C8001B003700110020000C0037006140B9005F
:10A9D800026A280013002000880502000000000019
:10A9E80003C3B3000341400092449800026A280060
:10A9F8000202B80004045400210020000371220060
:10AA0800811F7800110009000304D800CF007800E6
:10AA180004C3B3000441400082F07C000102E80056
:10AA28000380B90000045400833E20004903070056
:10AA38004306200047030700A20020001100090078
:10AA48000204D8000001780003C3B30003404100AA
:10AA580000F27C008400E8006A11B9000204540086
:10AA680004C3B3000440440080F07C008100E80087
:10AA78000040EB0080F478004F04BE0000000600A0
:10AA8800889FBE008A9FBE000004BE0002057800B1
:10AA9800E3CF51001200320005003C00E1CF510025
:10AAA8000B003200E2CF510007003A000A003700DD
:10AAB800E5CF51000C0032008005EB001D00350089
:10AAC800E6CF51000A0032008000EB002D0037006D
:10AAD8000002EB00270037008005EB001D0037005F
:10AAE8008005EB00170037008005EB000D003700EC
:10AAF800026A2800130020007403070002C3B30091
:10AB0800024D4000026A28000202B8000503400016
:10AB18000289B900820243000404540085845C0061
:10AB28001B0020000271220013030700027122009B
:10AB380014030700823E20000F030700823E200016
:10AB480010030700420620000B03070042062000FE
:10AB58000C030700A2002000430307000B02E800D3
:10AB68006A01B8006A08B900830140000204540071
:10AB780083845C0001C3B3000140440000727D007F
:10AB88008400E8000040EB0000F578004F05BE00A7
:10AB98004F04BE00000006000200FA00A2002000D8
:10ABA8008F80E9008A0B0200000000000080FA0094
:10ABB80000000600889FBE008A9FBE008C9FBE00D2
:10ABC80092ED0200000000000006BE006ABA800094
:10ABD8007BBA80000002BE006033B8000A00BE00E5
:10ABE8006011B800C009B0000180B0000280B00058
:10ABF8000380B0000020E10001A8E10002B0E100FC
:10AC080003B8E10040003600E8B98000F9B98000D7
:10AC18000A0256008B825E00027122000220B800F0
:10AC28009D0207000001BE00C41220000800BE00FB
:10AC38005D020700E0B98800F1B98800D702070073
:10AC4800C0010700DB020700BE010700D3020700AE
:10AC580018020700D70207001602070080882000A4
:10AC6800ACD402000000000080962000ACD40200A2
:10AC7800000000006CBA88007DBA8800004080009F
:10AC8800E20F50001200320005003E000000E00014
:10AC980009003200E10F500006003A0009003700B1
:10ACA800E40F5000100032000D003900E50F50008D
:10ACB800100032000028EF00208020002800070044
:10ACC8000F00370020802000830007000C003700A9
:10ACD8002080200050E60200000000000800370035
:10ACE800208E20001E000700208E20007A0007001A
:10ACF80003003700208E200050E60200000000000C
:10AD08000028EC00050037008A0F56008B8F5E0084
:10AD1800020031006CBA88007DBA880020802000CB
:10AD2800B4AE020000000000208E2000B4AE020085
:10AD3800000000004F06BE004F05BE004F04BE00D5
:10AD48000000060020802000B4AE020000000000D1
:10AD5800208E2000B4AE02000000000000000600B3
:10AD6800889FBE008A9FBE008C9FBE00800478002A
:10AD780030809000E20F50000600320049509000E9
:10AD88000044A100910207000000EB00B09C98006D
:10AD98004D00370049809000E10F500047003A000D
:10ADA800399E9000EE0F560018003C0049A590000F
:10ADB800D9A5900029A19000B9A190000A00BE0071
:10ADC800A6050200000000000000E0003E0032007E
:10ADD800AAA49800BBA498000C0446008809B000F7
:10ADE80002002400C36124000A00BE00AA05020074
:10ADF80000000000120602000000000000B47C0001
:10AE08000C00E800B09C98002F0037008A09200049
:10AE1800090545006066B8008005EB001A04780053
:10AE28006140B900CC030200000000000800E00007
:10AE380004003D000200200003782400A80402005A
:10AE4800000000000001BE000C00BE00A8040200C3
:10AE5800000000000006BE008B05E8000A85E80037
:10AE6800EF8F5500EDFF3A000000EB00B09C980012
:10AE780002002000031724000C00BE002204020078
:10AE88000000000048060200000000004200DD004B
:10AE9800A2002000110009000280D800E2922000E0
:10AEA80000015100D29C9800820C78004950900013
:10AEB8000044A000450207000300370049509000F5
:10AEC8000044A100C05498004F06BE004F05BE00C4
:10AED8004F04BE0000000600881F780000047800B8
:10AEE80040809000E20F5000060032004850900069
:10AEF8000054A100405498000000EB00609C9800AA
:10AF080040003700485090000054A000405498007A
:10AF1800485090000018A3003A003A006898900042
:10AF2800E10F50002C003200E20F50002F003200D9
:10AF3800E8A09000E0232000808F500010003E0021
:10AF4800484091000048A3000700320048409100A3
:10AF58000038A30004003A0008007800DCB20200C0
:10AF6800000000000300370008007800C0B20200AB
:10AF78000000000010002000609C980021003700AD
:10AF8800502D2000808F50001E0036004840910050
:10AF98000048A30007003200484091000038A30091
:10AFA80004003A0008007800C0B202000000000067
:10AFB8000300370008007800DCB20200000000003F
:10AFC80008007800DCB20200000000002000200029
:10AFD800609C98000B003700E8A09000E023200058
:10AFE800808F50000700360004003700E8A090006A
:10AFF800502D2000808F500002003E000000EB0022
:10B00800609C98004F047800000006000400FA00D5
:10B01800889FBE008A9FBE008C1F78000005BE0076
:10B02800020478000046EB000C4978000080FB0021
:10B03800EE80570096BC020000000000EE8057002A
:10B04800080078001A0B02000000000008007800D1
:10B05800540B02000000000008004000E9C2B300E1
:10B06800094878001C4098004850DE00EE805700E0
:10B0780096BC020000000000EE805700080078002F
:10B088001A0B02000000000008007800540B0200B0
:10B098000000000008004000094878001C409800A3
:10B0A8000B80FB00EE80570096BC020000000000F9
:10B0B800EE805700080078001A0B0200000000001C
:10B0C80008007800540B020000000000080040004F
:10B0D800094878001C4098004858DE00EE80570068
:10B0E80096BC020000000000EE80570008007800BF
:10B0F8001A0B0200000000004F0678004F05BE0042
:10B108004F04BE000080FA0000000600000178002D
:10B11800E0509000F0C4B30080CF50000C003A001B
:10B12800F25090006B40500080CF50000600320073
:10B138006540400080CF5000030032000040E80026
:10B1480080CF500002003A001000200001003700B4
:10B158000000EB000000060080017800E05090003D
:10B16800F0C4B30080CF500016003A00F3509000AE
:10B178006B40500080CF500006003A0082512100F9
:10B18800C1DA200003007800100007000080FB00EF
:10B198000D00370090C4B30080CF50000300320088
:10B1A800A0C4B30080CF500006003A0082B5210049
:10B1B800C157210003007800040007000080FB004D
:10B1C800010037000000EB00000006008001780055
:10B1D80050D09100EB4F50000A003E0073A0900041
:10B1E800810F50000300360073A09000820F5000BA
:10B1F8000B00390073A0900080A998000001EB00B3
:10B208000800370013009000A30090000001EB0035
:10B21800331F2000830F5000E08F580001003E00CC
:10B22800120020000200780000000600889FBE007F
:10B238008000780020802000808F50001A003A009B
:10B24800C2C2BF000080FB0048C0B300C704DE00D4
:10B258001000200068EF020000000000C2C2BF001A
:10B268000080FB004700DE00890F500003003A0011
:10B278000844E9002A003200F5FF370016E8A90063
:10B2880016C8A8002D00370016E8A80016C8A800A0
:10B298002A00370016E8A90016C8A900D0C0B300D4
:10B2A800D7E8B70025003700208E2000808F500097
:10B2B80022003A00CBC2BF004300DE000044EB008E
:10B2C800E10460001000200068EF020000000000A8
:10B2D8000844E800CBC2BF004300DE006100600004
:10B2E800890F500003003A00E44F54000F00320069
:10B2F800F4FF3700F6E8A900F6C8A8000F003700E9
:10B30800F6E8A800F6C8A8000C003700F6E8A9007F
:10B31800F6C8A900D0C0B300B7E9B70007003700E6
:10B32800C242E200D8FF3500DAFF3700CBC2BF00C7
:10B338000038A300F2FF3A00F4FF37004F04BE00C4
:10B3480000000600889FBE008A9FBE008C9FBE003A
:10B358008E1F78000004BE0092ED0200000000007D
:10B368000006BE0058AA9000E8AA90000402500007
:10B3780085825800823E20000220B8000007EB00BA
:10B38800C50007000005BE0008D891000080FB003A
:10B39800890F5000100032008A00D0002ED4990086
:10B3A8005ED49900F0F32100800F5500E08F5D0016
:10B3B80006003E0078A090006109B8000100200056
:10B3C800040320007800070070A498005CAC980083
:10B3D8006DAC980009DC990058A89000E8A8900086
:10B3E800800F5600818F5E002800390002E8230094
:10B3F800820F5500E08F5D00290036000900E0004B
:10B408001500320028D091000004E0002400350027
:10B4180028D091000040E80020D49900A8D09100DD
:10B4280038D0910080CF50001D003600EB00070097
:10B438001B003600485090000018A300030032009B
:10B4480028D0910040D499001500370028D19100E8
:10B4580032D499001200370058D091000004E0005F
:10B468000F00350058D091000040E80050D49900F2
:10B47800D8D0910068D0910080CF500008003600E5
:10B4880058D0910060D49900050037005CAC980052
:10B498006DAC980078D091000040E80070D4990015
:10B4A8004F0778004F06BE004F05BE004F04BE0090
:10B4B80000000600881F78000004780020D0910062
:10B4C800EB4F50000F003600485090000074A00069
:10B4D800C80007000DFF07000004E000300032003C
:10B4E800485090000018A3002D003A0048509000E2
:10B4F8000008A3002A003200B80007002800360020
:10B508002100370058D09100EB4F500011003E0049
:10B51800485090000074A100B6000700FBFE070029
:10B528000004E0001E003200080078000AFF07004F
:10B538000004E0001A003A00485090000008A300F8
:10B548001700320008007800B6B2020000000000C0
:10B5580013003700485090000074A1004054980030
:10B56800485090000064A1004054980008007800FA
:10B57800E6FE07000004E000090032004850900091
:10B588000008A3000600320008007800B6B20200E6
:10B5980000000000485090000024A100405498008A
:10B5A8004F04780000000600889FBE008A9FBE00F6
:10B5B8008C9FBE000004BE000200BE006125B800DA
:10B5C8000A01BE00380007000006BE000A01BE00DE
:10B5D800BE000700000454000C0144006000B800DD
:10B5E800010033006110B9004F06BE004F05BE00D0
:10B5F8004F04BE00000006000600FA00889FBE0047
:10B608008A9FBE008C9FBE0000057800F1B79F009E
:10B6180082BF9F0093BF9F008004EB0089057800DC
:10B6280072865700ADC3B300040037000B00E0007A
:10B63800020032008D747D008904E8003C447800E3
:10B64800084078001ABD02000000000000F57C00E8
:10B65800084078002EBD0200000000008900450067
:10B66800904098008984E8008B05E800E68F550033
:10B67800EEFF3A004F06BE004F05BE004F04BE0065
:10B688000080FA00000006006140600008003700F2
:10B698004400DE000B00370002A9B9008100410018
:10B6A800C2092000090037006805040000000000F6
:10B6B80001C3B300014D40008A0078000B007800F8
:10B6C8000000060061006000500037000300200001
:10B6D800F5FF3700880078000900780000000600B0
:10B6E8008A007800090078000000060042C0B30014
:10B6F8008A007800000006008A00780008007800B8
:10B708000000060052C0B3008A007800000006005E
:10B7180000047800000FEB00A0C0B300004F7800D1
:10B728008E84E8000000060093417800C819DD0007
:10B73800808171000A0078000000060093417800BB
:10B748000080FB00000006008E00780009007800E9
:10B7580000000600110009000304D80001C3B3006B
:10B768000141400002F27C000402E8000380B900B5
:10B7780000045400000006003B0007008B05E800A9
:10B78800000006000202B8000289B90085024100E3
:10B798000404540085845C0000000600212C20006D
:10B7A800914078008180FB00C708DE0020802000DF
:10B7B80000000600B12C200091407800C308DE008C
:10B7C800E1806000208E200000000600570007007E
:10B7D8000054A100C0549800000006001800900012
:10B7E800A8009000421F2000820F5000E08F5800F0
:10B7F8000000060040549800485090000064A000E3
:10B8080040549800080078000000060001C3B30007
:10B81800014C40001A00370011CB290008007800BD
:10B8280000000600880078000A0078000000060082
:10B8380001C3B300814D40000A00BE0000000600AD
:10B84800934178008381FB00000006001C0007007C
:10B858008300710008017800000006008E0078005F
:10B868000800780000000600030020001700070009
:10B8780003C3B3000341400082757D000000060049
:10B88800880078000B0078000000060042C0B30072
:10B89800880078000000060000F22F0080004200B7
:10B8A800414091000048A30000000600F06928000C
:10B8B80011002000800F5200818F5A0000000600FE
:10B8C800124178004811DD00000006000800BE00A3
:10B8D80075FF3700000141000A000900331978009C
:10B8E8006201B1006301B100000006000000E80039
:10B8F80011000700838F500000000600020040007E
:10B908000A000900301F78006E01B1006001B10023
:10B918008100E800000006000A0009003E1C7800CB
:10B928006801B1006E01B10000000600C054980023
:10B938004950900000000600020120001100090093
:10B948000200D8000000060080407800AED7BF0093
:10B95800814F50000F003200E24F400004003200D7
:10B96800D00A07000E00090030197800E201B10082
:10B9780001007800AEF7B700E2CF400005003200C2
:10B9880001407800C70A07000E0009003218780045
:10B99800E201B10000000600AFD7BF00E17A210044
:10B9A800914078000104E10017003200E24F4000A6
:10B9B8000C003200E2C1B3000440BC007C0341002B
:10B9C80065FE200062807A0081FD2F0001004000A2
:10B9D8008402200013C0B300A2092100E6C07A0047
:10B9E8002C0A0700AED7BF00AFF7B70082FD2F00C3
:10B9F800F18780000101410084022000CC0A070081
:10BA0800A0092100230A070000000600889FBE0045
:10BA18008A9FBE008C1F7800B017E20007003A002A
:10BA28008ABA020000000000F27F200002006000D5
:10BA3800024020000200400080BD8800C2032000B0
:10BA48008000EB00200C21002C0A020000000000FE
:10BA580048F920000005EB0059EA2A000A4078005E
:10BA6800B9FF07000900E8009000780063804400EF
:10BA7800100178001904E00008003A000280400034
:10BA880008004000AB0220008085450000ED210041
:10BA9800808F550002003600FFFF3700FFFF370098
:10BAA8001A71EF008002200008004000F08788002B
:10BAB800008040000000E800008888000000410085
:10BAC80010888800D0002000A08888001671A9007E
:10BAD800B1FF070079F89700C1F0B700BC0607006E
:10BAE8000A05E800E6844400E60F5500020032002B
:10BAF8000B047800D9FF37004F0678004F05BE00C9
:10BB08004F04BE00000006000400FA00889FBE0033
:10BB18008A9FBE008C1F780090BF9F00A1BF9F0026
:10BB28008245780003067800044578000004EB009D
:10BB3800884478000840780083FF0700A0888000C8
:10BB4800ED0F500050003A0093FF07000A407800BC
:10BB5800C150E3004C003A0080212000F0858800A5
:10BB68000B04E00006003A005C8588001671A80006
:10BB780040002000A0888800CC888800400037005A
:10BB880000C02F00B017B40081F82000810F5000CA
:10BB9800020036000040200080BD880080BD800083
:10BBA800508588000000E80080BD88004C8588002A
:10BBB80092ED02000000000060888800718888000B
:10BBC8001691A800E3CF550003003200E4CF5500DA
:10BBD8002B003A00120037002FB897009FB8970043
:10BBE8000100400000004600518580000100680007
:10BBF800C08888001FB89700AFB897008085880074
:10BC080091858800C070EF0081092000D1848800E8
:10BC18009C30EF0020002000A08888001800370022
:10BC28001FB99700224090000080FB00B2409000AE
:10BC3800C808DD00808070009281FB0012409000EF
:10BC48004800DD000300700080804000810046004D
:10BC58005085800080806800C1888800000B210022
:10BC68000900090032587800A200B10050002000F5
:10BC7800A088880011C0B30020C0B3004D0407009D
:10BC88000980FB00040037000804E800E60F5400B0
:10BC9800A7FF3A00E00F20004F0678004F05BE00CE
:10BCA8004F04BE000080FA000000060011002000CA
:10BCB800E54F500009003E0023FF0700B1888000CF
:10BCC800000021000080600002003A008000780037
:10BCD800020037001791A900110020000100780028
:10BCE800000006008000EB00E54F500005003E0014
:10BCF80015FF07008000EB00F009070001003A007B
:10BD080011002000F5FF3700E54F500031003E00DC
:10BD18000DFF07004088800050888800A0888000B8
:10BD2800E50F50002A00320006003E000000E00047
:10BD3800270032000080E900E10F500021003E009A
:10BD480023003700EB0F50001100320003003E00C3
:10BD5800E70F50001B003E0003003700EE0F5000B5
:10BD680018003A001400370011C0B30010C1B30026
:10BD780010040700AC10E20002003200D2090700EC
:10BD8800F9FF3A0080002000A088880011003700E1
:10BD980011C0B30010C1B30006040700AC10E200E4
:10BDA80002003200C8090700F9FF3A00C00020006D
:10BDB800A088880007003700D0002000A0888800ED
:10BDC800040037008040EB0040C1B300F9030700CE
:10BDD800FF05070000000600881F7800004478006F
:10BDE800E54F500004003E00D7FE07001671A90079
:10BDF80008407800C4FF07004F04780000000600E0
:10BE08008000EB00E54F500009003E00CEFE070021
:10BE1800E1FE0700A0FD2000010B21000900090038
:10BE28003158780040858000207F8800A1FD2000DF
:10BE3800AAFF3700E54F500006003E00C2FE07008B
:10BE4800D5FE0700A009070002003200A20907007A
:10BE5800D803070000000600E54F500012003E001E
:10BE6800B9FE070014D1BF00E74F500002003200AE
:10BE7800EB4F50000C003A00228880003188800087
:10BE8800810F510005003900960907008280500093
:10BE9800010040000000E900040037000280500063
:10BEA8000000E900010037000000EB000000060078
:10BEB8000200FA00889FBE0000447800A1FF9F009E
:10BEC800E54F500031003E009FFE07000840780013
:10BED800E1FF0700800478000000E0002B0032003A
:10BEE800E10F500002003A0008407800D1FF070037
:10BEF8001711AB0007003A007A0907000000D100CB
:10BF0800808F540003003E0008407800C9FF0700F6
:10BF18001711A8008009070020888000140020005D
:10BF28008441780066815700DA080700218880007C
:10BF38008100E8002188880000888000808F5000F8
:10BF480002003900F087800020888800E18F5400C3
:10BF580004003A0008407800B6FF0700090078009E
:10BF68000B0037001000200016B1AB0008003A00A3
:10BF780016B1A800AAED02000000000078004000F9
:10BF88008088880010002000010037000000EB00C6
:10BF98004F04BE000080FA0000000600889FBE0023
:10BFA8008A9FBE008C9FBE0000447800010678007E
:10BFB800820578000000EB00E54F54003F003E008A
:10BFC8000840780060FE070008407800A2FF0700DC
:10BFD800000578000000E00004003A0008407800FE
:10BFE80094FF07000A007800340037008B0F5000D8
:10BFF800020036008B0478000100370080047800C6
:10C008001711AB0007003A00360907000000D100FD
:10C01800800F550003003E000840780085FF0700A8
:10C028001711A80025888000018880000580440039
:10C038008006EB00810F50000B0039008586500008
:10C04800350907000D02780013C0B3000C01780011
:10C05800050078008F0807000D0646008D845400FF
:10C06800F0878000208888002B090700208880003E
:10C078000902780013C0B3000C0178008508070096
:10C08800090078000431B4008B0F550003003E000E
:10C098000840780067FF07000700370016B1AB00BB
:10C0A80005003A0016B1A800AAED02000000000041
:10C0B8007800400080888800098046004F06BE004E
:10C0C8004F05BE004F04BE0000000600889FBE005A
:10C0D800804478000104780001007800540B0200C5
:10C0E800000000000001780088007800094078000E
:10C0F800AAFF0700000044004F04BE00000006002D
:10C10800889FBE00804478000000EB00E5CF540013
:10C1180009003E00094078000BFE0700F887800000
:10C1280000888000080450000804E90009407800ED
:10C1380049FF0700000054004F04BE00000006003D
:10C14800881F7800004478000A0007000000E0001B
:10C158000600320008407800FBFD07004088800098
:10C1680050888800DC080700120307004F04780095
:10C17800000006008000EB00E54F50000B003E0079
:10C18800F1FD0700DA0807000200390081005100BC
:10C198000600370010888000810050000088800069
:10C1A80000005100808040008100E800CBFE37008D
:10C1B800889FBE008A1F7800004478000105780037
:10C1C800ECFF0700800478000000E0001500320052
:10C1D80008407800DCFD07000A00E0000600320095
:10C1E8005288800014002000CE08070084407800A0
:10C1F8000A00780027080700518880008100E800BD
:10C208005188880010888000808F50000200360016
:10C218000088800050888800E18F540003003A00AD
:10C228001751A80009007800090037001000200005
:10C2380016B1AB0006003A0016B1A800AAED02003C
:10C2480000000000A007B0008088880010002000CF
:10C258004F0578004F04BE0000000600889FBE000E
:10C268008A9FBE0080447800810578000204780027
:10C27800C0FF0700000578000000E0002C00320035
:10C2880009407800B0FD0700880F55000100310013
:10C298000A04780052888000118880000200440057
:10C2A8008004EB00810F50000B0036000280500024
:10C2B8008004E8000B00E000040032000902780066
:10C2C80039080700F3070700898545000904540069
:10C2D80000888000508888000B00E00003003200CE
:10C2E8005288800022080700EA0707000800780043
:10C2F8000A31B4000884440008005500800F540037
:10C30800030039001751A80008007800080037001A
:10C3180016B1AB0005003A0016B1A800AAED02005C
:10C3280000000000A007B00080888800080078009E
:10C338004F05BE004F04BE0000000600889FBE00E7
:10C34800804478000000EB00E5CF540008003E0070
:10C35800094078007CFD070008888000108880006C
:10C36800080450000940780082FF070000005400CC
:10C378004F04BE0000000600889FBE008A9FBE00D2
:10C38800004478008105780002057800830478006D
:10C39800E54F500022003E000200E000200032007D
:10C3A80069FD07000840780072FF070080007800E8
:10C3B80009004500808F50000100310009855000B8
:10C3C800508880000081440011888000810F51004E
:10C3D80001003600F7070700028050000004E8005B
:10C3E800880F550005003E000A027800EE07070096
:10C3F800A80707000A0078000A003700DC070700D2
:10C40800A4070700028880000B00440008025500BA
:10C41800470807009F0707000A0078000100370057
:10C428000000EB004F05BE004F04BE0000000600F0
:10C438000200FA0081017800120020008F80E900D4
:10C44800CDFF0700EFF897000180FB000080FA009D
:10C45800000006000F03B000889FBE008A9FBE0040
:10C468008C9FBE008E1F780000447800E1B79F00C3
:10C47800F2B79F00830578008404780085BF9F0089
:10C48800E54F5000A1003E000200E0009F0032008E
:10C498002DFD07000840780036FF07000B07500005
:10C4A8007FB097008E0F50009A003E000900E00010
:10C4B80003003200890F5700010036000907780091
:10C4C800508880000081450011888000810F51004C
:10C4D80001003600B7070700028050000000E8009E
:10C4E800C0B79F00EFB09700A1B79F00B144780094
:10C4F800A1B79F000FBA97000400E00006003200C1
:10C50800F0C9B30000C04400F94F500002003E00DB
:10C5180000CEB30080C444007FB59700BBB79F002E
:10C52800D2B79F002FB697008006EB000BC2B3006E
:10C538004FB09700FF0F500001003E008FED9700AD
:10C548000B80FB00800F5700010031008E457800FA
:10C558000B84FB0008027800F20707005FB1970020
:10C5680011C0B30040FC2F000F004000490707002E
:10C5780088027800DFB0970088804000D1B79F001C
:10C588004FB2970008025200C4B79F0004003A0057
:10C5980000888000D0B79F008080EB00C1B79F0063
:10C5A8000FBA97000400E0005F003A005B00370014
:10C5B8000042EB0043FC2F008F814100F6C9B30015
:10C5C80007CEB3003FB09700FFB0970001045000BA
:10C5D800030178009340780006C04000F94F5000EE
:10C5E80001003E0087C9400092CF54000E003A0077
:10C5F8000A05E90004003A000480FB00000044003A
:10C608000000E8004B003700BC44780006C0440036
:10C618001D002000F94F500010003E0087C4440060
:10C628001D0020000D0037000D00E00002003A0058
:10C638007FB59700090037006FB0970090447800E5
:10C6480006C04400F94F500001003E0087C4440072
:10C658007FB597002FB697008006EB000442E800EC
:10C668008301E80084CF550021003200D8FF37004D
:10C678000041EB008000EB003FB297007FB09700CD
:10C688008001520044FC2F000F02420064C0780071
:10C6980080CF540009003A000A05E90004003A0076
:10C6A8000280FB00008041000000E8002100370004
:10C6B800BC4478001D002000090037000D00E00090
:10C6C80002003A007FB59700050037006FB0970069
:10C6D800904478007FB597002FB697008006EB004E
:10C6E8000241E8008100E80082CF5500E5FF3A00EA
:10C6F800050757008E0F550006003E00BFB0970093
:10C7080085804000B1B79F0088FF37000000EB002C
:10C71800080037000080EB00060037000B04E0003B
:10C72800D3FF3A00F2FF37000B04E000A0FF3A0005
:10C73800EFFF37004F0778004F06BE004F05BE00D9
:10C748004F04BE000F03B100000006000200FA000B
:10C75800E1FF9F00840278000302780082017800DC
:10C76800120020008F80E9003AFF07000080FA00DD
:10C7780000000600889FBE008A9FBE008C9FBE00F6
:10C788000005EB000D0C21000A4678000A407800ED
:10C798006DFC0700B0888000016020000100600087
:10C7A800310032000A840200000000000000E000AE
:10C7B8002D003200B08880004A00DE00E1056000EC
:10C7C80009C1B3002A00370073FC07007440B900A0
:10C7D80080017800220C210002004000010B21009A
:10C7E80009000900B0587800A000B100EA804100B3
:10C7F800E100790041858800EC804100828040009A
:10C80800160020000700200031024300A1824B00DF
:10C81800148588002585880081858000978580009B
:10C8280087804000428580008280400052858000D9
:10C8380082806800C188880061002000A188880083
:10C84800620214007422B900610D210001814100C7
:10C8580013C0B300834078008E060700FA30EF005B
:10C8680029C1B300310037008044EB008005EB009C
:10C8780016B1AB000700320088888000AAED0200DC
:10C8880000000000000454004240A90001003C00E0
:10C8980009C1B30016D1AB000700320098888000A8
:10C8A800AAED020000000000000454004240A90064
:10C8B80001003C0009C1B300A0888000EB0F5000C4
:10C8C80009003A0098888000AAED020000000000E4
:10C8D800000454004240A90003003C00C0002000AE
:10C8E800A088880019C1B300A0888000E40F500018
:10C8F8000C003A00C28880000004EB00210D2100E2
:10C90800110078000000E00006003200820F50009D
:10C91800ADFF32000804E800F4804000E30F540043
:10C92800F7FF3A000904E0000400320011C0B30028
:10C938008BC05000094078001E0107001691AB001B
:10C948001D003A00DD060700A3003A0092ED020040
:10C95800000000009C0607009F003300B18880009B
:10C9680067806000E60F50000B003A00430CDE00C1
:10C97800614464000C407800E3FC07000C40780038
:10C98800E1FC07000804E00093003A00E000200002
:10C99800A088880090003700FFFB070021C0B30083
:10C9A80000C1B3000301070092ED0200000000007F
:10C9B800D30607008800370092ED0200000000004F
:10C9C8008106070084003300F3FB0700A08880007D
:10C9D8000100200062005000E0805800EA0F50007B
:10C9E800E08F580059003E00006001000A0037003F
:10C9F80012003700550037002B003700360037008B
:10CA08003E00370045003700540037004700370024
:10CA18003A00370049003700AAED02000000000084
:10CA280080888800000B210036DD0200000000002D
:10CA380030002000A088880044003700410B210006
:10CA4800000B210062DD0200000000000000E00091
:10CA580010003A00AAED0200000000008288800061
:10CA680002005000D2848000820F50003700360048
:10CA7800C0D0BF00E54F500003003E000040E80072
:10CA8800C0F0B7005506070020002000A0888800E5
:10CA98002E00370050002000A08888000004EB001A
:10CAA80029C0B3004600370029C0B30010C0B30046
:10CAB8009D4F10006E00360020C0B300C0F0B700D4
:10CAC800414B2C00D184880041002000E18488007B
:10CAD800804478006600370012C0B3009D4F1100F3
:10CAE8005E003600B0888000680060001B003A00D5
:10CAF80029C0B300000478001A00370024C0B3002E
:10CB08009D4F12005700360080002000A088880042
:10CB180019C1B3000004EB001200370025C0B300B0
:10CB28009DCF1200510036000C00370026C0B3001C
:10CB38009D4F13004B0036000800370027C0B30094
:10CB48009DCF130049003600040037000004EB00B5
:10CB58000904E00003003A001F00370049C1B30090
:10CB6800180020000B00E00015003200C070EC0037
:10CB78001A060700308580003388800003015000C2
:10CB8800830F5000020031005606070000014100E3
:10CB9800F08480000185800002005000E080580089
:10CBA8005A06070002007800AC30B40033858800CC
:10CBB8008040EB00094078007E0007000300370042
:10CBC80011C0B300094078007A0007000800E000AF
:10CBD800010032007E0207000A05E800E60F550052
:10CBE800E9FE3A008004EB002A0C21007448B900E1
:10CBF800000478007000400060007D000000E00044
:10CC08001D003200AAED020000000000720144007D
:10CC180062017D000200500072722000820F5000F5
:10CC28000A003600628214007422B900620D2100E5
:10CC3800020144000A00440013C0B3008340780096
:10CC480094050700FA30EF008904E9008904E80038
:10CC5800E28F540008003E00E4FF370029C1B3000A
:10CC68000300370009C1B3000100370019C1B30040
:10CC78000004EB00BDFF37004F06BE004F05BE00A5
:10CC88004F04BE00000006002000FA00889FBE0086
:10CC98008A1F780080047800020578001082FB0063
:10CCA800104090004800DD00040170002942900007
:10CCB8000482FB00394090004800DD0084017000C8
:10CCC80072845700028CBE001101BE0092BF9F0003
:10CCD800A3BF9F000040EB00E0F79F0060C0B300D7
:10CCE800F0F79F00CABF9F000A00780090BD0200BD
:10CCF80000000000C0BF9F00C100200008007800AD
:10CD0800D0BD020000000000000478000A0078008E
:10CD180082870200000000008880EA00808F5000AF
:10CD28001D003A000000EB00DAEB020000000000F2
:10CD380041012000A0FD2F000F004000B68902002D
:10CD480000000000A0FD2F000F004000FC010700BC
:10CD58003FB097004400DE006F4060004200DD00F5
:10CD6800744050000080FB0000005500740450001F
:10CD780089007800A0FD2F000F0040005B0107002C
:10CD88000000E0000400320088007800A0FD2F00B9
:10CD98000F0040007A020700208402000000000013
:10CDA800100020004F0578004F04BE000080FA00F4
:10CDB800000006002600FA00889FBE008A9FBE0079
:10CDC8000044780001457800F3FA07000808A3003A
:10CDD800020032001771A8000804A10016B1A900CA
:10CDE80016D1A90016F1A9001731A9001751A900F9
:10CDF8001711A9000A840200000000000000E000EA
:10CE0800FCFF3200660064008004EB004E003A002C
:10CE180020888000328580008004EB00820F50005B
:10CE28003E0032001100360002005000618580008B
:10CE3800810F50000100360001007800F98580005C
:10CE4800890F500002003E0080047800010037007E
:10CE58001751A80009027800670507000D050700AB
:10CE680009007800A630B4002C0037000188800043
:10CE780082815000B3BF9F0083004000F08780008C
:10CE88000080500061858000810F5000010036004D
:10CE980001007800F9858000890F500002003E00EB
:10CEA80080047800010037001751A800838F5400D0
:10CEB80001003100B9BF9F003FBA97004E05070037
:10CEC800F40407003FB8970000825400B4BF9F00E5
:10CED80008003200F2878000308580000011B5001C
:10CEE800919D2000010040008E0507008040EB0066
:10CEF800E804070030858000808044003185880080
:10CF080002888000828F500004003900F08780007A
:10CF18000000510000805000308588001771AB0078
:10CF28000700320060858000808F540004003200C2
:10CF3800F0858000808F5400010032000804A000B2
:10CF48000900E00002003A006300640011003200AA
:10CF580009007800AC30B5000900E000010032009B
:10CF68000834A0000A08A30005003200C070EF00D2
:10CF7800D1122300D184880011002000E1848800A8
:10CF880092ED020000000000FB0407001691A800C3
:10CF9800250037000A18A3000E003200B088800070
:10CFA8008040E800E780600082FF2F0002006000F8
:10CFB80001007000B0888800F0848000018580003E
:10CFC80061005000E080580050050700190020005B
:10CFD80015003700B08880007000600002003A0039
:10CFE80080047800100037000A08A3000A003A00FD
:10CFF800C0D0BF00080032000040E900C0F0B70010
:10D00800D0848000E18480008100D1000080D300BA
:10D01800D0848800E184880092ED020000000000BE
:10D02800D50407008004EB0041FD2F000180470074
:10D038005285800002087800418580001100980020
:10D04800F284800003858000C2AF9F00D3AF9F00A9
:10D05800ED040700E0AF9F00F1AF9F000FB097000D
:10D06800F1FF23000100600001FF2F0001006000B4
:10D0780080B79F0098E79F000000EB00B0B79F00C3
:10D0880009014100E0814900F28488000385880095
:10D098008880FB000100D1006100600080457800B5
:10D0A8000004E000130032000148A30003003A0026
:10D0B8006000B800E0AF9F00F1AF9F00BC30AB004C
:10D0C800070032004FA89700DFA8970061005000C2
:10D0D800E0805800C0AF9F00D1AF9F000500370027
:10D0E80061014100E0814900F284880003858800DD
:10D0F800BC30A8000808A30001003200BC10A8003A
:10D10800FB04070006003900008880000211B50002
:10D11800810051000100500090B79F0003003700C4
:10D12800028050000000E90090B79F004A84020086
:10D13800000000008000780090AF9F00F0032000FE
:10D14800808F500003003E008000EB0091AF9F00ED
:10D158000300370000FC2F000080400090AF9F00C4
:10D168009FA897001FB09700810F5000010036005C
:10D1780091B79F0042FD2F0002804700F000070092
:10D1880074854400F2F02F000FB097008200600011
:10D198000105B30081B79F000B04E0000A003200CC
:10D1A8007885440020C0B30080EF9F0040C0B300E2
:10D1B80090EF9F0020802100D0B79F000280600080
:10D1C8000006B30080B79F00C15A21009140780043
:10D1D8008180FB00ADD5BF004800DD000101700073
:10D1E800E15A2100914078008180FB00AFD5BF0053
:10D1F8004800DD008101700074845700028CBE0075
:10D20800808580009185800080BF9F0091BF9F002E
:10D218000040EB00C0F79F0069C0B300D9F79F003A
:10D22800BABF9F000A00780090BD0200000000000D
:10D23800B0BF9F00C100200008007800D0BD0200E8
:10D24800000000000080EA00A0B79F00109B2000AB
:10D25800DA860200000000000A01780089407800A0
:10D26800000B210052EB02000000000041012000E9
:10D2780042FD2F0002804700568A0200000000008D
:10D288000B04E000040032004100200078805700C1
:10D29800568A020000000000509C2000048702000B
:10D2A800000000000A0078008287020000000000E9
:10D2B80090AF9F00509D2000DA8602000000000019
:10D2C8002100200020FD2F000F004000568A020098
:10D2D80000000000B6850200000000004F05BE00F7
:10D2E8004F04BE000080FA0000000600889FBE00C0
:10D2F8008A9FBE008C1F78008005780001067800A0
:10D30800900190000300E000880032002140900066
:10D318000080FB00B1409000C808DD0080807000EC
:10D328001C81FB001C4090004800DD0002007000DA
:10D33800808040009B80400001856900E9CFB300F0
:10D348000004EB00084078007FF90700A0888000FF
:10D35800ED0F500018003200E40F500006003A00AC
:10D368009B009000C0888000810F500012003A0096
:10D378008844780010003700C0888000800F55006E
:10D388000D003A0084F907009B009000508580004A
:10D39800808F500008003A00408580009B0F1000E5
:10D3A80005003A001B0407008085800091858000F5
:10D3B80022040700150032000804E800E60F5400B4
:10D3C800E0FF3A00E2CF4400310032000940780023
:10D3D8005DF9070070F90700CA888800000B210072
:10D3E800090009003C587800AC00B1001B01780026
:10D3F800428588009B0590005B858800F387800044
:10D4080033858800100020004900370010002000F4
:10D4180047003700AAED0200000000007449B90077
:10D4280072014100240C210000317A000000EB0059
:10D438003F003700744CB9002A0C21000A00440050
:10D44800090009003C587800A000B100AC00B10008
:10D458006A0044001B307D000A0044002B01900044
:10D46800BB019000620098007300980070004400AF
:10D478009B0590000B307D00AAED02000000000023
:10D488007204440000347D000000EB0028003700DF
:10D498006B0090000098A30024003200FA10E2000C
:10D4A80022003A008004EB00240D2100940078004B
:10D4B8000100E000100032001B009000808F500037
:10D4C80009003A0054B897009B0F500006003A0034
:10D4D800D003070004B8970094B89700820F500053
:10D4E800838F5800CBFF32008904E80074024200A1
:10D4F800E38F5400EDFF3A000004EB000840780089
:10D5080011F907001671AB000500320022F9070077
:10D518009B00900050858000810F5000C5FF3200AD
:10D528000804E800E60F5400F4FF3A000000EB009E
:10D538004F0678004F05BE004F04BE0000000600ED
:10D54800881F7800000478001000780090BD020061
:10D5580000000000000C78001800900090BD020048
:10D56800000000001004980028009000B800900007
:10D57800A2BD0200000000002004980031049800B9
:10D5880048009000D8009000A2BD020000000000F2
:10D5980040049800510498007800900090BD020063
:10D5A80000000000700498000808900090BD020078
:10D5B80000000000000C98001808900090BD0200C0
:10D5C80000000000100C98004F04780000000600CE
:10D5D800F1F8070050858000C0888800F087800037
:10D5E800208888003088880000888000408888006B
:10D5F80050888800400020001671AB0001003A00F6
:10D60800D0002000A08888001611A9001631A900B2
:10D618001651A9001691A90016B1A90016D1A900A2
:10D6280016F1A9001711A9001731A9001751A9006F
:10D638001771A9001791A800BC10A900BC30A90057
:10D64800BC70A900BC90A900F087800030858800D4
:10D6580050BA020000000000F084880050BA0200AE
:10D668000000000000858800BAB0EF00100020001C
:10D6780060858800000006000200FA00889FBE004E
:10D68800C0002000DAEB020000000000A0890200C0
:10D6980000000000000FB2004280DE00F444500099
:10D6A80033003200710020000000EB00B689020050
:10D6B800000000002B003700A089020000000000D5
:10D6C8000004E0002A003200E14F5000250032003B
:10D6D800E24F500017003A00E2CF54002400360011
:10D6E8000000EB00D0BF9F00A089020000000000EE
:10D6F800E44F500006003A00A08902000000000034
:10D70800B0FF9F00A089020000000000A0FF9F005A
:10D71800DFB8970070212000808F50001400360079
:10D72800D039B000808F500012003E000100780010
:10D7380010003700E1CF54000D003600A089020028
:10D748000000000000447800894F500008003E00A7
:10D758008080FB000000EB00B6890200000000009A
:10D7680088C454008944E900E1CF4400D2FF3A005C
:10D77800802120004F04BE000080FA00000006004F
:10D78800F0874700889FBE008A9FBE008C9FBE001E
:10D798008E1F78000005780001077800504C900033
:10D7A80040069000D0069000B00090002000900045
:10D7B800D0B79F00E1B79F001611A9001631A90044
:10D7C8001651A9001691AB0003003A0092ED020031
:10D7D800000000004A030700A4888000E40F5200FC
:10D7E80003003200E50F520045003A0016003700EA
:10D7F8000880FB000028A30038023A000048A30074
:10D8080006003200FC8488000D8588008040EB000B
:10D8180040C0B30067FD0700300237000018A300BE
:10D828002E0232005FB19700EFB19700610141000D
:10D83800E081490012858800238588008EFF070053
:10D84800F0858800280037008880FB000128A300A5
:10D8580026023A004408DE00610060008045780036
:10D868000004E0000A003200F88480000985800086
:10D87800880F5600898F5E0005003200F20207000B
:10D888004CFD0700F88488000985880017023700D6
:10D898000118A300150232005FB29700EFB297009B
:10D8A80061024200E0824A001485880025858800CC
:10D8B8007A0590006A8588006FFF0700F085880068
:10D8C8000B04E000080032000303070039FD0700DD
:10D8D80070002000A088880092ED0200000000007F
:10D8E800DE0207000102370011C0B30020C1B300F7
:10D8F80030FD070060002000A0888800FB01370089
:10D908008882FB00E18562008BF79F000B04E00032
:10D9180002003A00CEB79F00020037008E00E800F0
:10D92800C1B79F000884FB000818A3000300320059
:10D938004FB197000201E800C2B79F00EC02070050
:10D9480005003900008880000211B50081005100EF
:10D958008104500002003700028050008004E90072
:10D96800A90207005FB19700EFB1970000005100CE
:10D97800818059000001BE00F0B79F004FB39700A7
:10D988000600E0001E0032000900E0002700320017
:10D99800E00F5000E08F5800040035006148B800DF
:10D9A800820F5000838F580009003E004FB3970044
:10D9B80006004100E08049004240A900060034000A
:10D9C80006805400CF80DE009C02070002003C0065
:10D9D80016002000010037000003EB006148B80082
:10D9E800960207000F003D00FFB097004FB1970067
:10D9F800028040004240A9000F003C0009003700A7
:10DA0800E00F5000E08F58000B003200070035008F
:10DA18006148B800820F5000838F580006003E000E
:10DA2800020037000600E00003003A000828A300BF
:10DA3800AE013A00AB01370066806200A7013A00E8
:10DA48000848A300A9013200EB0F520005003E0070
:10DA5800E70F520015003100E60F5200BB003A00F4
:10DA680003003700EC0F5200B8003A00AF0037004F
:10DA7800F484800005858000A4B79F00B5B79F0097
:10DA8800840F5600858F5E00060032006E02070084
:10DA9800C8FC07002FB09700BFB097009B02070093
:10DAA8009201370070002000A0888800348580002B
:10DAB800228880008400510002003B008902070090
:10DAC80080804000F28480000385800001004100CE
:10DAD800E08049000000560081805E004240A900B5
:10DAE8000B003400BC10AB0003003200E10F500003
:10DAF800E08F5800040032008040EB0000C1B30002
:10DB0800ACFC07007901370061065600E0865E002C
:10DB18003588800005005200CF80DE0000035100E8
:10DB280081835900850F5200020039000600BE00AB
:10DB3800030037006B02070000005300E0805B0021
:10DB48000001560081815E004240A900280034008F
:10DB580064020700010020003802070024003E008C
:10DB6800BC70A900BC90A9001711A90030888000DA
:10DB7800020240003488880031858000810F5000FF
:10DB880005003E00810F52000900360001005200D6
:10DB980035020700060037005202070000804000E7
:10DBA800800F520002003600000052002E020700CB
:10DBB80001888000810F520004003900F08780003E
:10DBC80000805000000052003088880032858000B4
:10DBD80001888000810F51001A003900F087800009
:10DBE8000080500000005100308588001500370083
:10DBF800850F520013003200E08580000038A30032
:10DC08000F0032000048A3000C003200F6848800A0
:10DC18000785880030858000808F52000500360017
:10DC280030020700CF80DE000000530081805B00D7
:10DC380036020700358588001751A800BC90A80057
:10DC4800BC70A8003188800020888000808F500038
:10DC58000C003A001771AB0004003A0092ED020084
:10DC680000000000FD01070006003700050207005C
:10DC780004003A00BC10AB00020032001691A90063
:10DC88001771A900F38480008C8051007A009000FD
:10DC980001005000AC10E20003003A000000E00070
:10DCA800010032001731A80060858800A088800034
:10DCB800E80F50000D003A00F201070023003A0077
:10DCC800BC10AB002100320092ED02000000000001
:10DCD80022BC2E00B3002000A90107001691A8005D
:10DCE80090002000A088880018003700E90F500035
:10DCF80009003A000B00E00014003A00FC84880098
:10DD08000D8588008B40780040C1B30029FC0700CE
:10DD18002FFE0700F5003700EA0F50000B003A000D
:10DD2800D8010700F1003A00EC003700F4848000C5
:10DD38000585800061004200E0804A00800F56009F
:10DD4800818F5E00E9003A00E40037000858A3001C
:10DD5800E6003A00A0888000EB0F5000E300320094
:10DD6800EA0F5000E1003200EC0F5000DF003200F3
:10DD78000E00E00094003200FFB597000B00E000B1
:10DD880044003C006A0090004200DE00C003B2007C
:10DD98000B005000DAEB0200000000007FB3970090
:10DDA800060547008A8F54000100310009057800F4
:10DDB800950107000A004000E080480010858800AF
:10DDC800218588004588800011888000050045006D
:10DDD800810F50000E003600058450000804E8004A
:10DDE8006C0107002B01070008045500CA01070051
:10DDF8000088800008027800A701070025010700B5
:10DE08000088800000044400488888000600370025
:10DE1800C10107000A027800600107001D01070020
:10DE28000A0078000831B400D0858000E10F400076
:10DE3800650032008A005000D18588007085800016
:10DE480000814000110033000100E0005E003C004A
:10DE58006D01070002004000E0804800108588003E
:10DE68002185880040888000800041004188880022
:10DE780010888000808F5000040036000011B50023
:10DE8800008040000000E90040888800BAB0EF0038
:10DE98004D003700FFB0970001004700808F540005
:10DEA80001003100018754006A0090004200DE0042
:10DEB800C003B200DAEB02000000000041888000D5
:10DEC8007FB1970081024100128880000500470059
:10DED800820F50001600360001005100FFB1970074
:10DEE800030050000004E80008003300290107007F
:10DEF800E800070088010700008880000802570032
:10DF080065010700E30007000D00370082010700E4
:10DF1800020078000011B500008042000000E9000E
:10DF28000E0278005C010700DA00070004003700E1
:10DF3800790107000E02780018010700D5000700D4
:10DF4800D0858000E10F400003003A00DB8588009F
:10DF58007E8588001C003700800078007FB297001B
:10DF6800800F52000E0031000401470070858000C8
:10DF780000804000800F510002003E00828F500058
:10DF8800020036007E85880003003700FFB2970044
:10DF98000500500070858800DB8588000A0037007E
:10DFA8007FB397000601470070858000008040001D
:10DFB800800F510004003600800F530002003E001D
:10DFC80001005100708588004FB097000000E00004
:10DFD8001200320039010700020032004188800037
:10DFE8005188880016F1AB00040032003A0107009E
:10DFF80070FB070068F607000800370016F1A80054
:10E0080016D1AB0005003A0016D1A800AAED02000F
:10E0180000000000D003B000908888000FF197003E
:10E028000204E0003100320014858000258580005C
:10E0380061014200E0814A004FB397005FB2970048
:10E04800EFB2970006004200E0804A00FB0007009C
:10E0580026003A00128588002385880017010700EA
:10E068000F00320003003E00E60F50001D003A008A
:10E0780005003700E80F500010003200E90F50008B
:10E0880018003A0012003700C0002000A08888005D
:10E0980011C0B30010C1B30046FB070013003700DE
:10E0A800B0002000A0888800AAED0200000000004F
:10E0B800A007B000908888000A003700F100070028
:10E0C80003003200A0002000A08888000500370067
:10E0D8008040EB0000C1B30036FB07003CFD0700A1
:10E0E80002003700FC00070032FB07004F077800EA
:10E0F8004F06BE004F05BE004F04BE000F01B10021
:10E1080000000600889FBE008A9FBE0001047800B8
:10E118008205780083447800E54F500058003E009F
:10E1280009F607000800E00001003A001800200086
:10E13800F08780000211B5000005E9000B044400D7
:10E14800880F55004E00390013F6070063806400FD
:10E1580001003A003940B300080055008981FB00EE
:10E168000318A30002003A008B007800060037006D
:10E178000308A300030032000000D100808045009E
:10E188000100370080804500F08780000080400053
:10E198000004E80044888000D1858000E18F4000B9
:10E1A80009003200708580000080400000024200B3
:10E1B80010888000800F5200030036000011B5005F
:10E1C800000042000002E90050888000800F5200E1
:10E1D80003003600800F54000A003600050037009F
:10E1E800800F52000500310000888000800F540025
:10E1F800070036000328A30021003A005888880049
:10E208004888880050888000800F52001000310034
:10E218000328A3000E00320002888000BE00070019
:10E2280002025200814178000800780019000700B6
:10E238004188800050888000808F500004003100A1
:10E24800080078000011B500008050004088880060
:10E2580008888800F087800030858800308888002A
:10E2680020888800110020009400070005003A006B
:10E2780099000700CFFA07001100200001003700BD
:10E288008000EB00010078004F05BE004F04BE007F
:10E2980000000600889FBE008A1F780000057800ED
:10E2A80082047800040478000304E00016003200B9
:10E2B800E1CF51002B003A000104E00008003200D1
:10E2C800E1CF500027003A00040178008900780067
:10E2D8000A007800600B02000000000021003700EF
:10E2E800E10F4500030032000A007800DA860200D8
:10E2F800000000008800780009007800568A0200B3
:10E3080000000000170037000104E0000C00320094
:10E31800E1CF500013003A00E10F41000300320042
:10E3280002007800048702000000000088007800DE
:10E338000A007800B68902000000000009003700D2
:10E3480004017800890078000A0078001288020029
:10E35800000000008A890200000000000000E000C0
:10E36800FCFF32004F0578004F04BE000000060095
:10E37800080278000C003700D2848000E384800013
:10E388000001410081814900628888007388880003
:10E398000000060060000700080278003E00070041
:10E3A8000500780000000600610007000B007800F7
:10E3B80000000600010078000011B50000004100CF
:10E3C8000001E90000000600628880007388800070
:10E3D800020050008380580000000600D0848000AE
:10E3E800E18480000000400081804800D0848800DB
:10E3F800E1848800000006004A0007008040EB0026
:10E40800909D200000000600108580002185800076
:10E41800000006009C80FB001C4090004800DD00C6
:10E4280001017000AC4090008180FB003C409000EE
:10E438004800DD008101700000000600800F5100D7
:10E44800818F590000000600FC8488000D85880033
:10E4580011C0B30040C0B300000006002800070048
:10E468001691A90000000600F28480000385800050
:10E4780000004100E080490024000700348588003E
:10E4880000000600F084800001858000800F56009F
:10E49800818F5E00000006008041EB000081EB00E8
:10E4A80000000600E2C1B3000440BC0060FE20008A
:10E4B80000014100E00F210000000600A088800054
:10E4C800E70F50000000060021888000308580009A
:10E4D800808F50000000060011C0B30000C1B300D7
:10E4E80000000600F08780000011B500000006005B
:10E4F8004288800051888000810F5100000006008A
:10E5080042782D00730120009DFF3700F0848800B9
:10E518000185880000000600A111210091407800C3
:10E5280000000600A31121009341780000000600B6
:10E53800FCFF070011C0B3000000060042052000E0
:10E54800820F5000E08F5800B3003E0000600100C9
:10E5580054003700B000370055003700AE003700D0
:10E56800AD003700AC003700AB003700AA00370019
:10E57800A9003700A8003700A7003700A600370019
:10E58800A5003700A4003700A3003700A200370019
:10E59800A1003700A00037009F0037009E00370019
:10E5A8009D0037009C0037009B0037009A00370019
:10E5B8009900370098003700970037009600370019
:10E5C8009500370094003700930037009200370019
:10E5D80091003700900037008F0037008E00370019
:10E5E8008D0037008C0037008B0037008A00370019
:10E5F8008900370088003700870037008600370019
:10E608008500370084003700830037008200370018
:10E6180081003700800037007F0037007E00370018
:10E628007D0037007C0037007B0037007A00370018
:10E638007900370078003700770037007600370018
:10E64800750037001D003700200037002300370011
:10E6580026003700290037002C0037002F0037002C
:10E668003200370035003700380037003B003700EC
:10E678003E0037004100370067003700430037008D
:10E6880046003700490037004C0037004F0037007C
:10E6980052003700550037005F0037005700370039
:10E6A80059003700E0252A00AC0607006000370053
:10E6B80090262A00A90607005D00370010002000F8
:10E6C800A29202000000000059003700100020004C
:10E6D800BE92020000000000550037002000200014
:10E6E800A292020000000000510037002000200024
:10E6F800BE920200000000004D003700100020000C
:10E708001C93020000000000490037002000200090
:10E718001C93020000000000450037001000200094
:10E728006C93020000000000410037002000200028
:10E738006C930200000000003D003700100020002C
:10E748004A93020000000000390037002000200032
:10E758004A93020000000000350037001000200036
:10E768009E930200000000003100370020002000C6
:10E778009E930200000000002D00370010002000CA
:10E78800C693020000000000290037001000200096
:10E79800F093020000000000250037001000200060
:10E7A8001C94020000000000210037001000200027
:10E7B80042940200000000001D00370020002000E5
:10E7C800C693020000000000190037002000200056
:10E7D8001C94020000000000150037001000200003
:10E7E8006E94020000000000110037002000200095
:10E7F8006E940200000000000D0037008A940200A9
:10E80800000000000A0037002000200042940200A7
:10E8180000000000060037005E07070042002000E5
:10E8280041272A003B070700D25F020000000000D2
:10E838000000060057070700E1C7B300022E2100B9
:10E84800604079005C5F02000000000000000600E4
:10E85800889FBE008A9FBE000040EB00E6F2B7002A
:10E86800EB2D21008004EB006A0920000084FB00E6
:10E878004244DD000B0044000908780084C0B3005E
:10E8880003052000094178006000B800885D020097
:10E89800000000000884E80000F47D0000C0EB00E0
:10E8A8005CF2B7005DF2B700622E210012417800D9
:10E8B8000281FB000A91B90000ED2100020040002E
:10E8C800DA86020000000000000478008A00780060
:10E8D80080242100568A0200000000000800780009
:10E8E800DA86020000000000E652EC00E6F2B7000B
:10E8F800E14F5000DDFF360009007800E6F2B7006E
:10E908004F05BE004F04BE0000000600889FBE00F1
:10E918008A9FBE008C1F78008004EB00082E21001F
:10E92800EC2D21008945780008057800184078000A
:10E93800E24F4000270032005A5E0200000000004B
:10E948000000E000180032000940780029000700A4
:10E95800100707000C0040000008EB005CD2BF0065
:10E96800E14F400003003200FCB502000000000047
:10E978005CF2EF005DD2BF00E14F400003003200BF
:10E98800FCB50200000000005DF2EF0083060700FE
:10E9980043C0B3000001EB001100200060407E007E
:10E9A800867002000000000078B897000000E000C0
:10E9B80005003A001A407800BE600200000000001E
:10E9C8000000E000030032000B4078000900070057
:10E9D800320007008904E80064044400E28F540010
:10E9E800D0FF3A004F0678004F05BE004F04BE0026
:10E9F80000000600889FBE008A9FBE008C1F78001A
:10EA080080457800E6D2BF008B4F50001F003200CF
:10EA18000080FB00680920000880B9000CED210087
:10EA280000004600DA86020000000000800478003A
:10EA38008A242100880078000A007800568A02009B
:10EA48000000000009007800DA86020000000000DB
:10EA58000B80FB000880B900000046000487020014
:10EA68000000000080047800880078000A00780020
:10EA7800B68902000000000009007800048702003F
:10EA8800000000000B007800E6F2B7004F0678009F
:10EA98004F05BE004F04BE0000000600F687470081
:10EAA800889FBE008A9FBE008C9FBE008E1F780084
:10EAB800EE2D2100E6D2BF000081FB004210DD00F0
:10EAC80060007F000100200018002000EB0F5000BC
:10EAD800E08F580013033E00006001001500370066
:10EAE800360037001D0137007F0137009B013700D2
:10EAF800A1013700E4013700F9013700640237004B
:10EB0800D4023700E4023700F30237002306070077
:10EB1800220020008000EB0060407F00326102008C
:10EB2800000000009B0607003100200001307F0034
:10EB3800E0FF3700E92D21004210DD000080E800E9
:10EB480060C07C00BE600200000000000000E00021
:10EB5800F602320040262100C09288008D06070088
:10EB68001100200001B07C005FF2EF000044EB00D0
:10EB78000004FD005EF2B7000004FD0092ED020003
:10EB8800000000006606070054B2EF0056B2EF001E
:10EB98004832EF004A32EF0008007800DCF2B70094
:10EBA800FE05070053C0B3000001EB001100200070
:10EBB80060C07C008670020000000000E82D210083
:10EBC8005E06070060407C00AA63020000000000A7
:10EBD800E10F400013003A00C4050700A2610200DB
:10EBE80000000000180020000000E00004003A00C7
:10EBF800ED0507007200200002307F000004EB00E2
:10EC080092ED020000000000EA050700C50234008A
:10EC1800EE050700885E020000000000EE05070010
:10EC2800A4FF370092ED0200000000003C06070038
:10EC3800EC050700AA63020000000000E50F500081
:10EC480001003600500020000001E800E805070038
:10EC580032610200000000003200200021992A00E1
:10EC6800402621003A0A0200000000000000E000EF
:10EC780002003A00009388000D003700420020008F
:10EC880061992A00402621003A0A0200000000008B
:10EC98000000E00003003A001400200004938800FC
:10ECA8000300370070002000009388001E01370021
:10ECB800CC050700AA6302000000000000047800E9
:10ECC8003C0607008801780004017800F1C3B3000E
:10ECD80060407F00AA63020000000000080178007D
:10ECE800800F54000100360000017800B0062000B3
:10ECF800800F510003003600500020000093880068
:10ED080067013700BA050700326102000000000001
:10ED180041262100010040000048EB000100780076
:10ED28009303070040262100540B02000000000056
:10ED38000004780072002000B1992A0050262100B2
:10ED48003A0A0200000000000000E0000D003A004E
:10ED5800502621008A8D0200000000005FF2B700F3
:10ED68006012E20003003A0080002000009388004F
:10ED78000200370090002000009388009F050700DC
:10ED88004CFF37008804E9003026210000004400C9
:10ED9800F1C2B30090CF10000400320050262100C9
:10EDA800C2B40200000000005CF2B700C0252100D8
:10EDB80000C2EB00904F120014003A007C8044001F
:10EDC8008224210002004000F1C2B30090CF10005D
:10EDD800030032007C004400017079000804E80058
:10EDE8004026210000004400219A2A000C00090056
:10EDF80031587800D000B1006C044400502621003E
:10EE0800C2B40200000000005CF2B7003026210006
:10EE18008000440040262100808F50000700320007
:10EE2800E0C2B300914F1000040032008100E900F5
:10EE380040262100808F5000F9FF3A000104E800C5
:10EE48000000EB0010938800E92A2A000000400027
:10EE5800E0807C000800780040BD0200000000004F
:10EE68000004E000040032006212EC0010938800F5
:10EE7800EA0F5000F5FF3600502621008A8D020067
:10EE8800000000005FF2B7005CD2BF00E14F400015
:10EE98000B003200F6B80200000000000018A300C2
:10EEA800070032005CD2BF00C0B9020000000000B9
:10EEB8000000E800A6B50200000000005DF2B700FF
:10EEC800E92D2100A305070060C07C00AA630200A9
:10EED800000000004D0507001600320010C0B30006
:10EEE8005EF2B7002D050700E1FD2F008F8040007E
:10EEF80060C07C00DC600200000000000801E9003E
:10EF080050072000800F510002003600420507001C
:10EF1800E8FE3700C892800035050700326102001C
:10EF2800000000000004440060C2B300005C7800E8
:10EF3800C89288008105070060407F00AA6302002C
:10EF4800000000000001E8008505070060407F0020
:10EF580032610200000000002805070018002000A8
:10EF6800ED2D2100F2FD2F000F01410082BF9F000F
:10EF78007205070060C07E00AA630200000000005E
:10EF880080047800E10F400014003A0026050700CD
:10EF9800A261020000000000800078000000E0008C
:10EFA80004003A00000507007400200004B07E0049
:10EFB8000104780092ED020000000000FD04070043
:10EFC800D801340018050700885E02000000000020
:10EFD8006605070001B07E00B6FE370092ED02001C
:10EFE800000000004E050700E18F5400C7FE320004
:10EFF800EB2D21006F0507008901780004017800D6
:10F00800A1C3B30060C07D00AA6302000000000035
:10F01800000578000084E800F00F54001300360063
:10F028000901E80003050700326102000000000042
:10F038000004EB00CEFF37000A40780022020700E8
:10F04800D6040700080278008801780008017800D3
:10F05800A1C0B30060C07E00AA63020000000000E7
:10F06800000678001800200019003700F404070093
:10F078008FB8970060C07E00326102000000000077
:10F088008A00E8000040EB000FB997008070790013
:10F09800088654000005EB00C9982A00FBFD2F00E4
:10F0A8008F854500990078000B0078006E0A0200F1
:10F0B80000000000D5040700DFFF32000A05E80061
:10F0C8008984E800E30F5500F6FF3A000004EB00DE
:10F0D8000C01E8002205070060C07E0032610200D2
:10F0E80000000000A2FF37005F52E2000600350072
:10F0F80030002000009388004210DD0074002000DA
:10F1080004307F006BFE3700C09280000048EB009F
:10F118004026210096020700C092880000938000D4
:10F12800E80F500003003A00C804070001307F00D0
:10F1380060FE3700170507008E00400040002000E1
:10F14800800878005E52E20002003A005000200079
:10F15800800878005E72EF0056FE3700D68D0200F8
:10F1680000000000E20F500070013200090507009E
:10F178005100200001307F0041040700BE600200FA
:10F18800000000006101B800B20407000A003A005C
:10F1980092ED02000000000086040700060034001B
:10F1A80052040700885E020000000000EF04070018
:10F1B80001307C003FFE370000938000E10F5000D3
:10F1C8000400320069005000E20F500005003600CC
:10F1D8002A003700708E020000000000E0DF9F0068
:10F1E800040037004A030700E0DF9F000004E00046
:10F1F8002B0032006FD89700E24F500008003A0009
:10F2080072040700BE600200000000000000E90070
:10F2180001002000A0928800B192880043013700C5
:10F22800E14F500015003A0015040700BE600200C7
:10F238000000000001002000A0928800B192880020
:10F2480092ED020000000000B5040700C9040700A1
:10F25800800407000500360024040700A2610200AC
:10F26800000000000000E00030013A0060002000CB
:10F27800009388007C0407000EFE3700C5040700D1
:10F288006100200001307F00C025210080C0EB0014
:10F2980090CF100006003A0040002000009388003C
:10F2A800BC0407007200200002307F0001FE370016
:10F2B8004832EF004A32EF005DD2BF00E14F400014
:10F2C80003003A004CB2EF004EB2EF0003003700E3
:10F2D800C124210008B702000000000062040700F2
:10F2E800E903070023C0B3000001EB001100200070
:10F2F80060407C00867002000000000000938000DF
:10F308000000400081942A00E0807800F70307009D
:10F318006A6002000000000000938000EC0F5000BB
:10F328000E003A00540407006A6002000000000062
:10F338001A040700F19A2A0060407C006A60020003
:10F34800000000004C0407006A6002000000000092
:10F358004C0407006A60020000000000009380006F
:10F36800E10F5000020036001B040700EF003700D1
:10F3780010938000EB0F50000F00320007040700C5
:10F38800219C2A0060407F006A60020000000000A3
:10F398001093800000004000E1322A00E0807800ED
:10F3A8000A0407006A600200000000003804070031
:10F3B8006A600200000000005CD2BF00F6B80200DC
:10F3C800000000000008A30005003200F303070056
:10F3D800119D2A0060407F006A6002000000000062
:10F3E800EE030700A19E2A0060407F006A600200C9
:10F3F8000000000000938000E10F5000050032007B
:10F408006092800071928000E10F4000E08F480018
:10F4180006003200E1030700A19F2A0060407F0038
:10F428006A600200000000000A003700DB030700E2
:10F4380031A02A0060407F006A60020000000000DE
:10F44800D6030700C1A02A0060407F006A6002005E
:10F4580000000000E82D21000A0407006A6002008D
:10F46800000000005E52E200040032004904070078
:10F478008100200001307C008EFD37000404070065
:10F488006A600200000000000404070089FD3700DC
:10F4980040262100D09288005E52E20069003200C6
:10F4A800E92D2100BD03070001A12A0060C07C00EE
:10F4B8006A600200000000002800370000C2B300A4
:10F4C80080CF500005003A00F703070060C07C00B9
:10F4D8005C5F02000000000020003700F0C2B300AB
:10F4E80080CF50000B00360060CCB30000C0400055
:10F4F800E64F50000700360050CAB30000C0400075
:10F50800E54F500003003600A0C7B30080CF50007D
:10F518000F003600E703070060C07C005C5F020054
:10F52800000000006FD897001ABD0200000000001C
:10F5380080407800E20307005C5F020000000000E2
:10F548006FD897002EBD02000000000080407800B0
:10F55800DB0307005C5F020000000000DB0307001C
:10F56800D6FF3A008D030700D1C3B30060C07C000A
:10F578005C5F020000000000E82D21002800370031
:10F5880000C2B30080CF500005003A00C603070050
:10F5980060407C005C5F0200000000002000370033
:10F5A800F0C2B30080CF50000B00360060CCB3002F
:10F5B80000C04000E64F50000700360050CAB300B4
:10F5C80000C04000E54F500003003600A0C7B3005C
:10F5D80080CF50000F003600B603070060407C0063
:10F5E8005C5F0200000000006FD897001ABD02009F
:10F5F80000000000804078003C0307005C5F0200C8
:10F60800000000006FD897002EBD02000000000027
:10F6180080407800350307005C5F020000000000AE
:10F62800AA030700D6FF3A00D503070060C07C0094
:10F638006A600200000000005E52ED005EF2B70052
:10F6480098FF3A00920307006A6002000000000079
:10F65800920307003B0007000000E00002003A00A8
:10F6680000047800060037005CD2BF00FCB5020039
:10F67800000000005CF2EF005703070018002000AC
:10F6880052030700305F0200000000000000E000A5
:10F6980024003A0025003700E82D21004210DD0043
:10F6A8000080E80060407C00305F0200000000003D
:10F6B800EF0F50001D00360080928000919280006C
:10F6C8009EFB07008703070018003A00AF030700F6
:10F6D80001307C00F7FC37005CD2BF00E14F4000EE
:10F6E80003003200FCB50200000000005CF2EF00ED
:10F6F8005DD2BF00E14F400003003200FCB50200BC
:10F70800000000005DF2EF0030030700885E020091
:10F71800000000009F0307000E0040000008EB00F7
:10F72800020037000800E000E2FC32004F077800D2
:10F738004F06BE004F05BE004F04BE006F01B1006A
:10F74800000006004200FA00889FBE008A9FBE00A3
:10F7580069030700305F0200000000004492800047
:10F7680055928000629280007392800004015100DB
:10F778008581590001002000800F5100818F5900B8
:10F78800010036000001BE00820478000200420039
:10F79800E0804A00D80207000200E00015003200AD
:10F7A8000A042000EB2D2100090178008A8F5400FB
:10F7B800010036000A0178005CD2BF0073FB2F00FD
:10F7C8008380470092B60200000000000F03070084
:10F7D800360032001A03070073FB2F0083804700AE
:10F7E80060C07D00D25F02000000000088845400E1
:10F7F800EDFF3A005F03070060928000719280007D
:10F80800800F5100818F59002A003A00BD0207007D
:10F81800A1002000013079005432EF005632EF0089
:10F828005CD2BF008000EB000EB6020000000000B2
:10F83800E8C7B3005CD2BF0061FB2F008F80400097
:10F848000EB60200000000000000E00004003200D4
:10F858008F020700EF70970088CF5000F5FF3A003D
:10F868008B0207005DD2BF000125210008B7020006
:10F87800000000005DD2BF00C124210008B70200CB
:10F8880000000000E10207000A003A004CB2EF0055
:10F898004EB2EF005DD2BF00FCB5020000000000D0
:10F8A8005DF2EF0008007800030037001000200028
:10F8B800010037000000EB004F05BE004F04BE00FA
:10F8C8000080FA00000006000004E00002003A0090
:10F8D8004C00070007003700E14F500002003A00D3
:10F8E8000500070003003700E24F500001003A000E
:10F8F80084000700000006002800FA00889FBE0068
:10F908008A1F78005F52E2003A0035005E02070065
:10F91800620020008000EB0060407C003261020041
:10F92800000000007A02070060407C002E6202009E
:10F93800000000006300400000047800C80FB20017
:10F9480040022000800F54000100360000047800B7
:10F958000800E00003003A0029FD2F008F844400CE
:10F968001300370029FD2F008F844400EA2D210061
:10F978008A020700420020008900780060407D006C
:10F988003261020000000000330020000901780005
:10F998004100200009007800EABB020000000000D6
:10F9A80064045400E38444000800E000F0FF3A00D7
:10F9B800804CEB0020FD2F000F004000A2C3B300D5
:10F9C800E6805700904F1100030032000000E80065
:10F9D800808F5000FBFF3A000058EB008000780051
:10F9E80020FD2F000F004000B28D02000000000033
:10F9F8005FF2B7004F0578004F04BE000080FA00A0
:10FA080000000600889FBE008A9FBE00E92D2100E5
:10FA18003F02070060C07C002E6202000000000068
:10FA280000047800A02D2100C19280000100500040
:10FA3800800F54002E003900770207002E0037008F
:10FA480037020700B1C3B300002E210065407800DB
:10FA5800AA6302000000000080047800CA928000B7
:10FA680008017800800F540001003600000178007A
:10FA7800EB2D2100490207008A00780060C07D0054
:10FA880032610200000000000000450061C2B300BE
:10FA980001587800C0928800890F54000E00360083
:10FAA80064020700DC600200000000000B0478001C
:10FAB8000300370022020700DC600200000000009B
:10FAC800A402070060407C00AA6302000000000056
:10FAD8000000E000F7FF32001C0207002E6202005F
:10FAE800000000004902070003003200D4FF37007D
:10FAF8000800E000D2FF3A004F05BE004F04BE00E8
:10FB0800000006000A00FA00100207002E62020038
:10FB18000000000080007800E90F50000500360062
:10FB280020002000009388004832EF004A32EF009E
:10FB38000D0037009702070001017800EA8057009E
:10FB48007402070032610200000000008040EB00F0
:10FB58006A00500001F07F006A8057007A0D0200A9
:10FB680000000000E40107000080FA000000060021
:10FB78000200FA00889FBE008A1F780000047800FF
:10FB8800540B020000000000800178000000E00033
:10FB9800280032000805780008017800020478007F
:10FBA800B84078008304E900D0C3B30080CF500088
:10FBB800030032007740500080CF500002003A0026
:10FBC800005DEB0017003700B0C2B30080CF5000D3
:10FBD80003003A006B405000005D780011003700C8
:10FBE80050C2B30080CF50000D003A00E18F54009E
:10FBF800110036001844780098FF9F0022409000BA
:10FC080080FF9F0063044100E38451004FB89700D0
:10FC1800D2BC020000000000005D7800010037003F
:10FC2800015D78000900E000030032000801BE0011
:10FC3800DAFF3700080578008040EB00015D7800A6
:10FC48000A007800014D78004F0578004F04BE0087
:10FC58000080FA0000000600889FBE008A1F780016
:10FC680000047800010578001004E0001800320054
:10FC7800880078000A0078006E0A02000000000080
:10FC88000000E00006003A000A007800540B020069
:10FC980000000000000044000000E8000D003700EC
:10FCA80008007800540B0200000000000000440027
:10FCB8000004E80008007800540B0200000000006F
:10FCC800000044000004E8001804E000E8FF3A00DF
:10FCD8000000EB004F0578004F04BE00000006004E
:10FCE800889FBE0000047800010178008000780039
:10FCF800D0C3B3002F000700800478000800E0009C
:10FD0800040032001804E000020032000800780005
:10FD180097FF0700090078004F04BE0000000600A6
:10FD2800889FBE008A9FBE008C1F7800000578005F
:10FD380001067800010178008000780060C2B300F5
:10FD48001C00070080057800E20F50000E003A0002
:10FD58004892800059928000E7010700BE600200C7
:10FD68000000000001002000800F5400818F5C001B
:10FD780005003A000C0178008A0078000040EB008A
:10FD88000C000700800578000A00E000040032003B
:10FD98001A04E000020032000A00780074FF07002D
:10FDA8000B0078004F0678004F05BE004F04BE00D8
:10FDB80000000600889FBE008A9FBE008C9FBE0080
:10FDC8008E1F7800004778008106780002067800C8
:10FDD8000004E0000800320051010700804078006C
:10FDE800002E210065407800AA6302000000000090
:10FDF8008005780004003700BF010700BE600200DC
:10FE080000000000800578002A002000E18F4500EE
:10FE180039003200E10F560008003E000D00E000F6
:10FE2800080032001F0107003261020000000000D4
:10FE38001F0107001A002000260037000D00E0000F
:10FE480006003A00170107003261020000000000B6
:10FE5800170107000005EB001E0037000C81E900C0
:10FE6800828F550012003600160107008D007800B9
:10FE780060407D0032610200000000000C010700B4
:10FE88000C8155000281E800B501070060407D0043
:10FE98003261020000000000050107008C80460066
:10FEA8000040EB00E0F89F001A002000090037002E
:10FEB800320107008D0078009601070032610200C8
:10FEC80000000000FA0007000040EB0080F57E000B
:10FED8000005EB000E04E000070032008A0107006D
:10FEE8008000EB00022E210060407900DC600200F7
:10FEF80000000000EE0007000A0078004F077800B5
:10FF08004F06BE004F05BE004F04BE0000000600AD
:10FF18001000FA00889FBE008A1F780000938000B6
:10FF2800EA0F500058003200EB0F50003F0032003B
:10FF3800E90F500084003A00E82D21001201070063
:10FF480042002000D1A12A0060407C002E620200FD
:10FF58000000000080007800E10F40002900320016
:10FF68000E010700010178008000EB0060407C0072
:10FF78003261020000000000D6000700DB00070025
:10FF8800BE60020000000000E90F50006E0036005D
:10FF980002010700A2002000F680570060407C00A4
:10FFA8003261020000000000CA000700A200200021
:10FFB80021A22A00768057003A0A020000000000B9
:10FFC8000000E0000B003A00A00020000093880029
:10FFD800D8B70200000000005CF2B7006200200001
:10FFE800F280570018B8020000000000200020002E
:10FFF80056003700B0002000009388002000200041
:020000040001F9
:10000800520037009E000700BE600200000000009A
:1000180064015000CA0007003261020000000000BD
:10002800AC0007001000200048003700A5000700BA
:1000380060407D00BE600200000000009C000700D8
:10004800D600070060407D00A460020000000000A8
:10005800C0F92F00F1FF2F00460107000200400001
:1000680083804800C2F92F00F3FF2700820F500059
:10007800838F580034003600F400070001307D00FB
:100088000000EB00310037001B010700BE600200D2
:10009800000000000004780036010700010020007D
:1000A800820F5000838F5800010036000204780048
:1000B8000800E00017003200EA2D2100080178004E
:1000C800F00F54000100360002012000B3000700C1
:1000D800F680570060407D00326102000000000099
:1000E8000001780040928000519280000200500088
:1000F800E080580080000700020454005CD2BF0072
:10010800F680570018B80200000000000800E00060
:10011800EAFF3A004092800051928000E00F5000C0
:10012800E08F580008003A00100020007CB8020058
:100138000000000073000700710020000130790002
:100148000000EB0001003700100020004F05780088
:100158004F04BE000080FA00000006004000FA00CC
:10016800889FBE008A9FBE008C1F7800000178001F
:10017800DC00070010003A0002007800C2B4020058
:100188000000000000457800E14F400037003200D1
:10019800C0B9020000000000A092880011003700DA
:1001A8000A407800FCB50200000000005432EF005D
:1001B8005632EF002D003700A0928000A6B502004D
:1001C8000000000000457800E14F400027003200A1
:1001D800B292800003002000210020001AB702001C
:1001E80000000000C4000700305F020000000000AB
:1001F800800478000000E000150032000B042000A5
:10020800EC2D2100090178008B8F54000100360085
:100218000B01780061FB2F008F8040000A407800B6
:1002280092B602000000000078000700DCFF3200F0
:100238008300070061FB2F008F80400060407E0034
:10024800D25F02000000000088845400EDFF3A00ED
:100258000A407800AAB9020000000000B0928800A5
:100268000A407800FCB50200000000004F06780044
:100278004F05BE004F04BE000080FA0000000600D3
:10028800E82D210019003700E82D21004300370030
:10029800409280005192800061004000E080480058
:1002A80015003700350007008000EB009900370083
:1002B80000045400E0845C00489288005992880049
:1002C800000006004892800059928000EA2D210023
:1002D80032003700A700070000015100E0815900F3
:1002E8004292880053928800000006002B00070005
:1002F80060407C000000060040928800519288000F
:1003080000000600A3000700E22D210000000600FF
:100318001D0007002200200091272A000000060087
:10032800652E2100954278008582FB00C22ADD00F7
:100338000002EB0084017800040178000000060048
:100348008700070060407C0000000600662E210040
:10035800164378000683FB004233DD008002EB0081
:1003680005027800850178002200200091272A00E4
:10037800002E210066407800000006006200070099
:100388000B01780000000600040007008002EB0063
:100398000502780085017800000006007D0007004E
:1003A8000080E8000000060050002000009388004C
:1003B80078003700829280009392800002005000FB
:1003C800838058004240A90000000600F3FF0700A0
:1003D80060407F00000006006400070001307F00D5
:1003E800000006005B00070060407F000000060078
:1003F8005500070060407F00000006006500070008
:100408002100200001307F00000006000004780071
:100418000000E00000000600E3FF07007100200074
:1004280001B07C0000000600DCFF070060C07E0011
:10043800000006004A00070060C07D0000000600BA
:10044800D6FF0700080178000000060051000700E9
:1004580071000500A0928000B1928000800F5100C9
:10046800818F5900000006004A0007007400200030
:1004780004307F00000006003300070060407C0065
:10048800000006003E00070060407C0000000600F7
:100498003B00070060407F00000006003B000700AB
:1004A80001307F0000000600BCFF0700B1C2B300A6
:1004B80000000600B9FF070051C2B30000000600A3
:1004C800B6FF070060C07C0000000600D0928000E4
:1004D800B0407800A1DF9F00D09288000104E000BE
:1004E80000000600A0928000B1928000E00F50004A
:1004F800E08F58000000060026000700012E2100AA
:1005080060C0780000000600489280005992800080
:1005180020003700032E210060C07900000006008B
:10052800229D2400B306200000014100818149007A
:100538008292880093928800000006001900070044
:10054800A1C0B3000000060094FF07004126210067
:10055800000006001300070001C2B30000000600F7
:100568008EFF07008000EB0000000600090007006E
:10057800B1000500429280005392800000000600FE
:1005880086FF070091272A000000060001000700E7
:1005980091000500E6D2BF000080FB004200DD00AC
:1005A80000000600030007008401780004017800B9
:1005B8000000060079FF07000002EB0000000600BB
:1005C8000200FA00889FBE00CD22A800C922A90017
:1005D8008000EB0001128800F00020001012880053
:1005E800211288004302A80042A2A80041E2A80004
:1005F800F1030700D1C1B300668057000204070069
:10060800AFF897000180FB000038A300F8FF3A001C
:100618000080EA00E1046000F5FF3A0018002000BD
:10062800F8BB8800D9BB88008940780080C0B30037
:10063800430407008940780090C0B30040040700D5
:1006480011CAB300C0C0B3003D04070091C0B30095
:10065800D0C0B3003A04070011CAB300A0C0B30069
:100668003704070091C0B300B0C0B30034040700DA
:1006780021CAB30040C0B3003104070091C0B300E1
:1006880050C0B3002E04070021CAB30020C0B30035
:100698002B04070091C0B30030C0B3002804070042
:1006A8000940780070030700002020007604070046
:1006B800D1C0B300094078002104070021C3B3006A
:1006C80020C0B3001E04070021C1B30040C0B3001E
:1006D8001B04070001C4B30030C0B30018040700AE
:1006E800F1C3B30090C0B3001504070021C1B300E3
:1006F80060C0B30012040700C1C0B30070C0B300EB
:100708000F040700E1CEB300A0C0B3000C0407003B
:1007180051C0B300B0C0B300090407004030200046
:1007280059040700915D21009140780040C0B30052
:1007380003040700A15D21009140780050C0B30078
:10074800FF030700B15D21009140780020C0B3008D
:10075800FB030700C15D21009140780030C0B30061
:10076800F7030700D15D2100914078000940780027
:10077800F3030700E15D210091407800084078000C
:10078800EF0307008940780050C1B300EC0307006D
:1007980021C1B300658057009B0307003FF897000D
:1007A80080F7B7000110200000C1B3001A04070049
:1007B8002147230040C1B3001704070089007800CF
:1007C8000940780014040700090078002E04070087
:1007D80041C0B300F0C1B300FE0307004F04BE00E0
:1007E8000080FA00000006000200FA0011C0B30001
:1007F8000F80E900A60307007FB897004200DE00DB
:10080800610060000080FA00000006000200FA00A3
:10081800F1C1B3000F80E9007B030700EFF89700F0
:100828000180FB004300DE000000A20061006000C0
:100838000080FA0000000600881F78007E17E2009A
:1008480010003A0010002000F0BB8800D8BB8000E0
:100858000804E9006104070001003600000478007C
:1008680001C4B300E0C1B300DA0307008840780090
:10087800C0C0B300B2030700C840DE00D0C0B30058
:10088800AF0307004F047800000006000600FA00D6
:10089800889FBE008A9FBE0090112000FA030700BF
:1008A8000AF02F00FB0F200091C1B3006E805700A3
:1008B800550307002FF49700E0002000F20307001B
:1008C800E1C0B3006D8057004F0307003FF0970069
:1008D8000080FB008A84640080847400F1C0B30047
:1008E8006C805700480307004FF097004800DD0070
:1008F8008B8464008084740090112000E203070058
:1009080091C1B3006B8057003F0307005FF0970069
:10091800804F5400E4FF3A00C0002000DA030700CB
:10092800C1C0B3006A805700370307006FF0970013
:100938000080FB000A04640000047400D1C0B30006
:1009480069805700300307007FF097004800DD00FA
:100958000B04640000007400808F5400040036000B
:1009680080805400109A20000101500005003700D3
:10097800129A2000808F54000200320009005000B3
:100988000001E900020078004F05BE004F04BE00D8
:100998000080FA00000006001600FA00889FBE00DA
:1009A8008A1F7800800478000105780090112000E3
:1009B800B503070091C1B300688057001203070010
:1009C8000FFC97000000EB00AF0307000000EB00EE
:1009D8000804E0003A0032007E17E20003003A0003
:1009E80095FF07000000EB0035003700D0BB800002
:1009F800E0BB8800C1772100914078000040EB00FF
:100A08004F030700D17721009140780010C0B30050
:100A18004B030700410120007C805700510207006A
:100A28003FB8970090BD020000000000B0BF9F00D3
:100A38002FB19700109A2000800F51000D003E0042
:100A4800CFE0970061C060000A003A00CFB197007C
:100A5800000128000080610006003A00BFB097003E
:100A6800E05E2000808F500002003E000378A30063
:100A780001003A000000FE00D2BB880070805700D9
:100A880005000900B05C78006900B1006000B100A1
:100A980000CDEB007FF09700E84F500006003A00C9
:100AA8006FF097000004E00002003200E64F5000AB
:100AB80001003A00004D78007E37EF00100020005A
:100AC8004F0578004F04BE000080FA0000000600C1
:100AD8000200FA00889FBE00000478008144780074
:100AE800D2BF9F0031CAB30020C0B300140307006F
:100AF80091C0B30030C0B30011030700009B200071
:100B0800DFB8970080804000D1BF9F00AFF8970002
:100B180060C0B3000A030700BFF8970070C0B300B5
:100B28000703070061002000080078005D02070045
:100B380061002000905D21005A02070080C0B300C8
:100B48004902070060C0B3000904E00001003A0050
:100B580009407800440207004F04BE000080FA00F4
:100B6800000006001000FA00889FBE008A9FBE00A1
:100B78008C9FBE00AA03070016030700A8030700FE
:100B880003030700A1C0B300C0C1B30000030700FE
:100B9800A60307000F03070080D7BF006540500079
:100BA800E14F50006F003E000004EB00893E20003A
:100BB800C1C1B30074805700930207004FE8970043
:100BC8006A00600003003A000804E800890F540036
:100BD800F7FF3A00C1C1B300738057008A020700CB
:100BE8005FE897000018A30003003A00703E200059
:100BF800800F54005B0036008C030700E4020700F6
:100C08008040EB00728057007F0207006FE8970072
:100C18000080FB0009F02F0009056500000575003C
:100C280011C0B3007180570077020700FFEE9700EC
:100C38004868DD00F80F200008056500000575000C
:100C480061C0B300708057006F0207000FF0970073
:100C58000080FB00898464008084740071C0B30044
:100C68006F805700680207001FF097004800DD00FA
:100C780088846400808474000904E800884578004A
:100C8800884078000040EB00AD0207004844DE00D1
:100C9800884478008840780010C0B300A802070094
:100CA8007C865700810020000C007800AD01070009
:100CB8000044EB00C1C1B3006E8057005202070028
:100CC8002FF097000018A300200032003FB09700D3
:100CD80000D8A3001D00320051030700BD02070021
:100CE8004F030700AA020700A1C0B300C0C1B300A8
:100CF800A70207004D030700B6020700C1C1B300F1
:100D08006D805700400207003FF097006A006000BE
:100D1800FAFF3200450307009D0207008B40780068
:100D28000040EB00860207008940780010C0B3003D
:100D380083020700810020000C0078008901070069
:100D48000844E800F04F5400DAFF3A008A4078007F
:100D58000040EB007A0207008D40780010C0B30015
:100D6800770207004F06BE004F05BE004F04BE00C5
:100D78000080FA0000000600881F780009030700B9
:100D88000200360020672F00008440008840780069
:100D98000040EB006A020700C840DE0010C0B30044
:100DA800670207004F047800000006000400FA00FC
:100DB800881F7800668157000019780021C0B300A9
:100DC8000200780010020700FA02070031C0B300E1
:100DD800638057000C0207001703070020C0B30008
:100DE80057020700BFF8970030C0B300540207004D
:100DF800080078004F0478000080FA000000060020
:100E08000400FA00881F78006681570000197800EE
:100E18008040EB0002007800FB010700E5020700B4
:100E280011C0B30063805700F701070002030700F1
:100E38000040EB0042020700BFF8970010C0B30063
:100E48003F020700080078004F0478000080FA008D
:100E5800000006000200FA00889FBE008A9FBE00BC
:100E680081057800CF0207000200360020672F00B6
:100E7800008440008040EB006A805700E2010700D0
:100E88006A8057003081FB0001F02F0001056500E2
:100E98000205750011C0B300DB010700FFF49700DD
:100EA8004848DD000A85FB00000575008840780089
:100EB8000040EB0022020700C840DE0010C0B3006B
:100EC8001F0207000B0078000C00070000047800E0
:100ED8008A4078000040EB0019020700894078003A
:100EE80010C0B30016020700080078004F05BE00C6
:100EF8004F04BE000080FA0000000600FA87470091
:100F0800889FBE008A9FBE008C9FBE008E1F7800FF
:100F1800800578006044B8008040EB00708057007E
:100F2800B90107000FF09700D90207000106660013
:100F38000006760011C0B3006F805700B2010700A9
:100F48001FF797004870DD000C86FB00000676004E
:100F58000B00E00020003200C0FD2F008086470013
:100F68008B007800F48F5500010036004101200005
:100F7800D1AF9F000D007800FA000700DFA89700A6
:100F88008185550061806000050032000040EB005B
:100F980080F07E005FA997000201E800D2AF9F00B1
:100FA800DFA897000100E00009003200C0FD2F0013
:100FB800008147003200780000044400E0844C00BF
:100FC8000180E90080007800FAFF3A00D0AF9F0066
:100FD8000B00E000E2FF3A008C4078000040EB0094
:100FE800D70107008E40780010C0B300D401070075
:100FF8006148B80008044000E08448000900440043
:101008000080EA004F0778004F06BE004F05BE007B
:101018004F04BE00AF01B100000006001000FA0046
:10102800889FBE008A9FBE008C9FBE00A0B79F000D
:10103800B1B79F00C2B79F008005EB000B05780091
:10104800E10F4000020032000B0678000C00370068
:1010580021C0B300768057006B0107002FE8970086
:101068000080FB00A0B79F0031C0B3007580570017
:10107800650107003FE89700D0E79F001C002000AB
:101088008006EB003FB09700E10F40000C003A00EB
:101098008040EB00748057005B0107004FE8970021
:1010A8000080FB00B0B79F0011C0B30073805700E9
:1010B800550107005FE89700F0E79F001D0020003A
:1010C800CFB49700E18F540045003E000D00E000CA
:1010D8000E003A008D407800728057004A010700E0
:1010E8006FE897006A0207008185650080857500B2
:1010F80011C0B30071805700430107007FE89700D3
:101108004800DD008B85FB00808575000C00E00041
:101118000E003A0021C0B300708057003A01070062
:101128000FF097005A0207000105650000057500D9
:1011380031C0B3006F805700330107001FF09700DC
:101148004800DD000A85FB0000057500EFE0970008
:101158000040EB007A010700FFE0970010C0B300E1
:1011680077010700CFE0970020C0B30074010700A3
:10117800DFE0970030C0B300710107000900E0000C
:10118800060032000004EB006B000700B600070001
:101198000804E800888F5400FBFF3A000D00E000C7
:1011A80006003A008B4078000D4078006401070083
:1011B800C858DE0010C0B300610107000C00E00051
:1011C8004D003A008A40780020C0B3005C01070057
:1011D800C850DE0030C0B300590107004600370090
:1011E8000C00E000080032002FB097000085440092
:1011F8008A40780020C0B30051010700C850DE00C3
:1012080030C0B3004E0107003FB497000885440082
:101218008A04E900C9B79F00F1C1B3006E80570086
:10122800F90007002FF097000058A300FAFF3A00D2
:10123800EFE0970000C1B30041010700FFE097000D
:1012480010C1B3003E010700CFE0970040C1B300D2
:101258003B010700DFE0970050C1B30038010700E9
:10126800DE01070005003E00808F540003003600B1
:10127800D0652F0000004500C0B79F007885570053
:101288009A40780020C1B3002D010700F784570069
:101298009940780030C1B3002901070001C1B300AB
:1012A800F0C1B3003A01070001C2B300F0C1B300B6
:1012B800480107000D00E0000F0032004FB1970011
:1012C8008200E800C1B79F00C401070004003E0087
:1012D800808F50000200360000005100C0B79F0008
:1012E8009A4078000040EB0015010700994078000B
:1012F80010C0B300120107004F06BE004F05BE0024
:101308004F04BE000080FA00000006000200FA0048
:10131800F1C1B3000F80E900BB000700EFF89700A8
:101328000180FB004500DE000000A20061006000B3
:101338000080FA0000000600AB01070000A02300AF
:1013480040128800C2010700FEFF3A00C3010700EF
:10135800FCFF3200C4010700CD22A8000080FB007A
:10136800000006000200FA0080017800CD22A900E2
:10137800A0032000401288000300E00001003200B2
:101388008301E900B2010700FEFF3A00B30107003C
:10139800FCFF3200B70107000002EB00E18F5000AC
:1013A80013003600910107006022B800451288003A
:1013B8000482E800A6010700FEFF3A00A701070023
:1013C800FCFF3200421280000300E00004003200FB
:1013D8004810DE00904198008381E8008249780037
:1013E80004805000E10F5000F0FF3E00A401070008
:1013F800848F5000180036000001EB008002EB00DB
:1014080084805000451288000300E0000800320084
:101418008301E8008E010700FEFF3A008F010700F4
:10142800FCFF320040128000804978000600370037
:1014380087010700FEFF3A0088010700FCFF320021
:101448008C0107008001EB000201E800828F500048
:10145800ECFF3A0002024200CD22A8000400780006
:101468000080FA00000006000200FA005E01070092
:101478000080FB0001A027000100700040128800D6
:1014880073010700FEFF3A0074010700FCFF3200F9
:1014980075010700E0FF9F00CD22A8000080FA0038
:1014A800000006000200FA008001780001027800BE
:1014B800CD22A900A007200040128800640107007F
:1014C800FEFF3A0065010700FCFF320069010700D2
:1014D800E10F5200280036001380FB004800DD00B1
:1014E8000281FB00000171001340900068010700B1
:1014F80001016100000171008381E8003B010700E0
:10150800421288000482E900E10F520014003600FC
:10151800F10F200005F02F001380FB004800DD00CC
:101528000101610000017100134090000080FB0080
:1015380005016100000171008381E8004401070092
:10154800FEFF3A0045010700FCFF32004901070091
:10155800421288000482E900E10F5200EEFF3E00CB
:101568003B010700FEFF3A003C010700FCFF320088
:1015780040010700420107000400E0000B003200B0
:1015880003017800848041003280FB00401288000B
:101598002F010700FEFF3A0030010700FCFF320070
:1015A80034010700810F5100F7FF3A00CD22A8004F
:1015B8000080FA00000006000200FA0001C2B30031
:1015C800E0C1B300720007001000200068EF0200BD
:1015D80000000000CD22A900F00F20004012880072
:1015E8001B010700FEFF3A001C010700FCFF320048
:1015F800020107001000200068EF02000000000050
:101608000080FA0000000600000107001001070032
:10161800FEFF3A0011010700FCFF32004012800073
:101628004822EF000A010700FEFF3A000B010700FD
:10163800FCFF320040128000CD22A800004978004B
:101648000200780000000600F00007000001070013
:10165800FEFF3A0001010700FCFF32004012800043
:101668004822EF00FA000700FEFF3A00FB000700DF
:10167800FCFF3200401280004822EF00F40007000F
:10168800FEFF3A00F5000700FCFF3200E9FF3700D3
:101698000400FA00889FBE008004780001447800A6
:1016A80040212000780007008840780040C1B3003E
:1016B8002300070011C0B30020C1B30020000700B9
:1016C800A030200070000700A1C0B3006880570058
:1016D800DDFF07000FF8970061446000FAFF3A0049
:1016E80040212000680007008840780020C1B3002E
:1016F8001300070081C1B30067805700D2FF0700BD
:101708001FF89700AC00070091C1B300668057002E
:10171800CDFF07002FF897004800DD000884FB0084
:10172800000474000000EB0057000700880C7800E4
:10173800090078004F04BE000080FA00000006008F
:101748000200FA00CD22A9000064A0000080FB007E
:1017580040128800BE000700FEFF3A00BF000700E5
:10176800FCFF320098000700B9000700FEFF3A00AE
:10177800BA000700FCFF3200BE00070000000000AE
:1017880000000000CD22A8000080FA00000006003A
:101798000200FA00CD22A9000080FB00000AB30075
:1017A80040128800AA000700FEFF3A00AB000700BD
:1017B800FCFF320084000700A5000700FEFF3A0086
:1017C800A6000700FCFF32008C0007000080FA002A
:1017D800000006000200FA00CD22A9000074A00053
:1017E8000080FB004012880099000700FEFF3A00C5
:1017F8009A000700FCFF32007300070094000700FE
:10180800FEFF3A0095000700FCFF32007B0007004E
:101818000080FA00000006000400FA00881F780023
:1018280000447800D1BF9F00402120001600070027
:101838008840780040C1B300C1FF0700AFF89700A7
:1018480060C1B300BEFF0700BFF8970070C1B300C6
:10185800BBFF0700A03020000B000700A1C0B300A9
:101868006480570078FF07004FF897000008A3002E
:10187800FAFF3A000000EB00030007004F0478006D
:101888000080FA00000006000200FA00F0BF9F0086
:1018980031C0B300F0C1B300BDFF0700FFF89700E7
:1018A800F0C1B300CBFF07000080FA00000006007B
:1018B8000200FA0041C0B300F0C1B300B4FF070052
:1018C800D1C1B3000F80E9004FFF0700EFF8970080
:1018D80064C06000FAFF3A00F1C1B3000F00E900EC
:1018E80049FF07007FF897000038A300FAFF3A0085
:1018F80001C2B300E0C1B300B6FF07000080FA00E0
:10190800000006000200FA0001C2B300E0C1B30003
:101918009FFF0700D1C1B3000F80E9003AFF07001D
:10192800EFF8970061C06000FAFF320041C0B300D1
:10193800F0C1B300A7FF07000080FA00000006000E
:10194800881F78000044780050312000CEFF07003F
:101958008840780050C1B30079FF07000000EB0011
:10196800C9FF07004F047800000006000200FA00D3
:10197800881F780050312000C3FF070051C1B30011
:101988006480570020FF07004FFC97000000EB0021
:10199800BDFF07000880FB004F0478000080FA00B4
:1019A80000000600E1BB8000810040007484400014
:1019B8000A0037000FF8970035000700010464009B
:1019C800000474000000060040128000A0FF9F0081
:1019D8000180FB004012880000000600109A2000D9
:1019E800800F540000000600CD22A90041E2A900A2
:1019F8004342A80041E2A80000000600401280000F
:101A0800A0FF9F00CD22A80000000600000178007A
:101A1800CD22A9008180FB00411288000000060049
:101A280001C8B300F0C1B3000000060081C0B300D4
:101A3800F0C1B300000006001FF897004800DD0061
:101A48000884FB0000047400EFF097000000060013
:101A580040C2BF000018A3000000060040C2BF003B
:101A68000008A300000006000500070040128000DF
:101A78000000060040128000A0FF9F000000060042
:101A880041E2A9004342A90041E2A8000000060083
:101A98000080FB0001F02F0000000600889FBE00B8
:101AA8000004780081447800C21220008000EB0016
:101AB800C01121002C0A0200000000001840780024
:101AC8008000EB000004E000070032008000EB001B
:101AD800C2112100807079008100E80061407C001B
:101AE8000004E000FBFF3A000904E00004003200B3
:101AF8000101E800A1C0B300C01121000171780004
:101B0800100020004F04BE0000000600881F780067
:101B1800000478007200200041C02A003A0A02003E
:101B2800000000000000E000080032004200200031
:101B3800C1C02A00080078003A0A0200000000002C
:101B4800010820000000E00001003A008000EB00DE
:101B5800010078004F04780000000600881F780014
:101B68000104780011C12A006E0A0200000000007A
:101B78000000E00007003A0071C12A000800780060
:101B88006E0A020000000000010820000000E000CA
:101B9800010032008000EB00010078004F0478005B
:101BA800000006002E00FA00881F780081C32A0072
:101BB80040262100307E020000000000000178006D
:101BC8000000E00040003200C0C3B300924F100094
:101BD8000C003A009240900060C4B30080CF5000DF
:101BE80008003A00A2409000F0CCB30000C04000CA
:101BF800E14F50000700360080C4B30080CF50008A
:101C08000400320011C0B30000C42A00A3FF07007B
:101C18002D003700014478007A80570011C22A004D
:101C280016000900315878007001B100E301410045
:101C38008000EB006022B80013417800E0C3B300D5
:101C4800804F510018003A0000FD2F000F0040009F
:101C58000498BE000498BE000498BE000498BE0014
:101C68000498BE000008EB006000200090AF9F00C1
:101C780002FD2F000F0141007A8057001E950200D7
:101C8800000000000FA897000000E000DDFF320010
:101C980001FD2F008F80400008407800623102006B
:101CA80000000000080037000204E000D5FF320001
:101CB8007A80570002F078008100E8008301E8008C
:101CC800F68F5000DCFF3A000000EB004F0478006C
:101CD8000080FA00000006001400FA005CD2BF0081
:101CE80042012000F480570078B90200000000008B
:101CF80092002000E1C52A00748057003A0A0200C9
:101D0800000000000000E00003003A00400120004D
:101D18000000E900FEFF3A0022012000B1C62A00B7
:101D2800748057003A0A0200000000008000EB00AF
:101D38000000E00002003A0004000700800078007C
:101D4800010078000080FA00000006003600FA0062
:101D5800889FBE008A9FBE008C1F78004892800032
:101D680059928000EB2D210029030700BE60020074
:101D7800000000000005780025030700A2610200AA
:101D8800000000000000450001002000800F540002
:101D9800818F5C00DC003E001D030700BE6002006E
:101DA800000000006101B80014002000409280008B
